:020000040800F2
:10000000183600209D010008C7500008D53C0008A4
:10001000C5500008CF120008E17800080000000079
:1000200000000000000000000000000005010008C2
:10003000671700080000000049010008176F00085A
:10004000B7010008B7010008B7010008B7010008B0
:10005000B7010008B7010008B7010008B7010008A0
:10006000B7010008B7010008B7010008B701000890
:10007000F5160008011700080D17000819170008E9
:100080002517000831170008B7010008B70100085C
:10009000B7010008B7010008B70100087117000890
:1000A000B7010008B7010008B7010008B701000850
:1000B000B7010008B7010008B7010008B701000840
:1000C000B7010008B7010008B7010008595100083E
:1000D00065510008FD77000809780008B70100089D
:1000E00069170008B7010008B7010008DFF810D051
:1000F00000F03AFE0048004777860008AFF3008022
:1001000018360020224B19680868B0E8F00F80F319
:100110000988BFF36F8F4FF0000080F311884EF015
:100120000D0E70470000000006480068006880F36C
:10013000088862B661B6BFF34F8FBFF36F8F00DFE1
:1001400000BF00BF08ED00E0EFF30980BFF36F8F41
:100150000F4B1A6820E9F00F106008B54FF05000FF
:1001600080F31188BFF34F8FBFF36F8F0BF0B2FB9B
:100170004FF0000080F31188BDE808401968086856
:10018000B0E8F00F80F30988BFF36F8F704700BFAE
:1001900018000020EFF305807047000006488047F4
:1001A00006480047FEE7FEE7FEE7FEE7FEE7FEE75C
:1001B000FEE7FEE7FEE7FEE78F6F0008ED000008B0
:1001C0002DE9F05F0546002092469B46884606468C
:1001D000814640241BE0284641464746224600F01F
:1001E00020F853465A46C01A914110D3114618467A
:1001F000224600F099FB2D1A67EB01084F46224674
:100200000120002100F090FB17EB00094E41201E59
:10021000A4F10104DFDC484631462A464346BDE8E6
:10022000F09F202A04DB203A21FA02F000217047D7
:1002300021FA02F3D040C2F120029140084319464E
:10024000704740EA01039B0703D009E008C9121F69
:1002500008C0042AFAD203E011F8013B00F8013B80
:10026000521EF9D27047D2B201E000F8012B491EAC
:10027000FBD270470022F6E710B513460A46044643
:100280001946FFF7F0FF204610BD10B5044604E004
:100290000B7800F8013B03B1491C521EF8D22046EE
:1002A00010BD421C10F8011B0029FBD1801A7047B9
:1002B00030B505460020034600E05B1C934205D2A2
:1002C000EC5CC85C201A01D1002CF6D130BD2DE9C0
:1002D000F0410E460546002400E0641C285D00F055
:1002E00040FB0746305D00F03CFB381A02D1295D27
:1002F0000029F2D1BDE8F0810FB400B58DB010A98E
:1003000009900B9000914FF0FF300A9000200C9064
:1003100005480690054807906A4609A80F9900F01D
:100320003BFB0DB05DF814FBB5090008D3090008CC
:100330002DE9FF5F1D464FF0FF3BD5E90146914691
:100340005F464FF00008A9697F1C01988847296A19
:10035000824688470028F6D1BAF1FF3F0CD024F43A
:10036000C064002E19DD600614D5BAF12B0F09D038
:10037000BAF12D0F0ED103E0584604B0BDE8F09F4E
:1003800044F48064A9697F1C01988847761E8246E0
:10039000002E02DDBAF1300F03D0B9F1000F26D0E4
:1003A00032E0A969761E44F400747F1C01988847E6
:1003B0008246002E05DDBAF1780F06D0BAF1580F4B
:1003C00003D0B9F1000F10D01EE0B9F1000F02D038
:1003D000B9F1100F18D1A969761E24F400747F1C9E
:1003E000019888478246102002E0082000E00A2099
:1003F000814609E008FB0908A969761E44F40074E7
:100400007F1C019888478246002E05DD49465046EC
:1004100000F0ADFA0028EDDAE96901988847A005F7
:1004200002D46FF00100A8E7E00725D1600613D5DC
:10043000600502D5C8F1000000E0404629680A1DA9
:100440002A600968220501D5087015E0220701D548
:10045000088011E008600FE02868011D296000682D
:10046000210502D580F8008006E0210702D5A0F81A
:10047000008001E0C0F8008038467EE72DE9F047B3
:1004800091460F4680460446002614F8015B2DB1C4
:1004900000F05AFA0068405DC007F6D12B2D02D05B
:1004A0002D2D18D0641E4A463946204600F0A2FA87
:1004B00027B13968A14201D1C7F8008071054FF01A
:1004C00002040BD54042002803DD07F085FB0460E1
:1004D000A007BDE8F08746F48066E4E70028F8DA74
:1004E00007F07AFB04606FF00040F2E72DE9F05F5F
:1004F00093460F4680460446002607F06DFBD0F871
:100500000090824614F8015B2DB100F01DFA0068DE
:10051000405DC007F6D12B2D02D02D2D1AD0641EC0
:100520000021CAF800105A463946204600F062FA07
:10053000014627B13868A04201D1C7F80080DAF837
:100540000000022809D0CAF80090700505D548427D
:10055000BDE8F09F46F48066E2E70846F8E7F0B4AD
:1005600080EA0102D40F4200B2EB410F02D20246F0
:10057000084611464A0042D0C30DDDB2C1F3C7524E
:10058000AD1A202D35DAC1F3160141F4000204B191
:100590005242C5F1200602FA06F12A411044B3EB9B
:1005A000D05F23D0C4B1012DA0EBC35009DCF0BC57
:1005B0004FF0004202EAC352DBB200F5000000F047
:1005C00071BA400000F1807000EBC350A0F1807060
:1005D00040EAD170490009E0490841EAC071A0EB46
:1005E000C35000F50000400800EBC350F0BC00F021
:1005F00050BA6142012202EB4101001BF6E7F0BC58
:10060000704781F00041AAE780F00040A7E730B4CE
:1006100080EA010202F0004530F0004221F0004083
:1006200013D090B1C30DD40DC2F31601C0F3160060
:10063000E41A41F4000140F400027D34914201D3F8
:10064000641C00E04900002C02DA30BC0020704736
:100650004FF400000023914201D3891A034340085C
:100660004FEA4101F7D151B1914202D14FF000411F
:1006700005E002D24FF0010101E06FF0010103EB50
:10068000C450284430BC00F004BA2DE9FE4F81EA82
:10069000030404F0004421F0004100944FF0000BEB
:1006A00023F0004350EA01045ED052EA03045BD019
:1006B000C3F30A54C1F30A552C44A4F2F334019451
:1006C000A0FB0254C1F3130141F48011C3F31303DF
:1006D00043F4801301FB024400FB034E840A970A93
:1006E00044EA815447EA8357A4FB076802958D0AC0
:1006F00005FB07854FEA932C04FB0C542705029D4C
:100700004FEA065847EA1637B5EB08056EEB070CBB
:10071000870E920E47EA811742EA8312A7FB020175
:10072000B6EB0B0164EB00042B0D43EA0C335E18AF
:1007300044EB1C50DA465146E7FB0201C5F31304B3
:100740004FEA0B3343EA14534FEA0432019C43EA65
:100750000603A4F10C040294009CCDE900B400F05F
:10076000DEF903B0BDE8F08F00200146F9E72DE97E
:10077000F04D81EA030404F0004B21F000451446DB
:100780004FF0000A23F0004150EA050220D054EA5D
:1007900001021DD0C5F30A570246C5F31303C1F386
:1007A0001300C1F30A5640F4801543F48013A7EBFD
:1007B0000608101BD64608F2FD3873EB050002D37D
:1007C00008F1010801E092185B41B8F1000F03DA6B
:1007D00000200146BDE8F08D00204FF48011064650
:1007E00084460EE0171B73EB050705D3121B63EB62
:1007F000050306434CEA010C49084FEA3000921801
:100800005B4150EA0107EDD152EA030012D082EABF
:10081000040083EA0501084305D0101BAB4106D252
:100820000122002306E000224FF0004302E06FF0B7
:10083000010253101AEB06004CEB085110EB0A00B2
:1008400041EB0B01BDE8F04D00F05AB930B404465D
:1008500096230800214604D0B62330BC002200F0C5
:1008600021B920460021F8E70EB5C10F80EAE070FB
:100870000844CA07002140F233438DE80E000A46BF
:100880000B4600F04CF903B000BD0EB540F2334109
:1008900002910021CDE900110A460B4600F03FF914
:1008A00003B000BDC1F30A5210B5C1F3130140F209
:1008B000FF3341F480119A4201DA002010BD40F26A
:1008C00033439A42A2F2334203DC5242FFF7A9FCBF
:1008D00010BD904010BD00F0004230F000400AD042
:1008E000C10D01F56071C0F3160042EA0151C20862
:1008F00040071143704700200146704730B50B4652
:10090000014600202022012409E021FA02F59D423F
:1009100005D303FA02F5491B04FA02F52844151E13
:10092000A2F10102F1DC30BD202A04DB203A00FAFA
:1009300002F1002070479140C2F1200320FA03F336
:10094000194390407047000000487047C0F300080A
:1009500010B50446FFF7F8FF0068005D00F00100E5
:1009600010BDA0F14101192900D8203070473A2864
:1009700000D2303820F02002412A01D3A2F1370002
:10098000884201D34FF0FF307047000002681144E5
:100990001378016018467047D160044951610449D9
:1009A000116200211161114600F002BA8D090008A0
:1009B00051090008426842B1016811F8013B23B1B6
:1009C000521EC0E90012184670470121C160881EFE
:1009D000704742685AB1C368016843B983688B4263
:1009E00005D0491E521CC0E90012002070474FF08C
:1009F000FF3070472DE9F05F8246007800271546EA
:100A00008B460AF10104B946302801D09DB113E0AC
:100A100014F8010B0127782803D0582801D045B1DC
:100A20000AE00DB1102D07D10027102514F8010B95
:100A300002E0082500E00A250026B0460EE005FB8E
:100A4000080005FB06F1012701EB10461FFA80F8AC
:100A5000B6F5803F00D3B94614F8010B2946FFF7DD
:100A600086FF0028EBDABBF1000F05D00FB1641E42
:100A700000E05446CBF80040B9F1000F06D007F073
:100A8000ABF802210160C81EBDE8F09F48EA0640AD
:100A9000FAE70029A8BF7047401C490008BF20F0B2
:100AA0000100704710B4B0FA80FC00FA0CF050EA74
:100AB000010404BF10BC704749B1CCF1200421FAF5
:100AC00004F411FA0CF118BF012121430843A3EBF0
:100AD0000C01CB1D4FEA00614FEA102042BF0020FD
:100AE00010BC704700EBC35010440029A4BF10BCD9
:100AF0007047401C490008BF20F0010010BC70473F
:100B000010B5141E73F1000408DA401C41F1000115
:100B100092185B411A4301D120F0010010BD2DE96C
:100B2000F04D92469B4611B1B1FA81F202E0B0FA63
:100B300080F220329046FFF7F7FE04460F4640EA67
:100B40000A0041EA0B0153465A46084313D01146A6
:100B500053EA010019D0C8F140025046FFF761FB8B
:100B600005460E46504659464246FFF7DDFE08430D
:100B700005D0012004E020463946BDE8F08D002074
:100B8000054346EAE0762C4337430A986305E40AB6
:100B9000A0EB08000022FD0A44EA47540A3002D5BF
:100BA00000200146E9E7010510196941DDE9084522
:100BB00000196941BDE8F04DA2E72DE9FE4F8046DE
:100BC00081EA0300C00F0C46009021F0004123F0A1
:100BD0000045B8EB0200A94105D2404621469046A7
:100BE0001C460B46024623F00040104347D0270D19
:100BF000C7F30A00C3F30A510290401A019040283B
:100C00006BDAC3F3130040F4801B0098924620B1C6
:100C10000023D2EB030A63EB0B0B01985946C0F19A
:100C200040025046FFF780FE06460D4650465946A4
:100C3000019A00F0ABF810EB08006141002487EA4C
:100C4000115284EAE7731A4340D0009A62B3019AC2
:100C5000012A4FEA075215DC001B61EB02014FF03D
:100C6000004202EA0752CDE90042001C41F5801122
:100C700032462B46FFF753FF03B0BDE8F08F4046E6
:100C80002146F9E7001B61EB0201001C41F58013CE
:100C900000185B412018A2F5001747EB030140EA5A
:100CA000D570B6196D4111E06D084FEA360645EA78
:100CB000C0754FEA0752001B61EB0201001C41F5B1
:100CC000801149084FEA30000019514132462B4645
:100CD00003B0BDE8F04FFFF713BF009801224000BA
:100CE0000023D0EB020263EBE073009821464FEA49
:100CF000E074B8EB000061EB0401E9E783F0004326
:100D00005BE781F0004158E7C1F30A52C1F31301D8
:100D100040F2FF3341F480119A4202DA002001468A
:100D2000704740F233439A42A2F2334202DC52420D
:100D3000FFF777BAFFF7F8BD30B5041E71F1000474
:100D400004DB4FF00044404264EB0101141E73F1D8
:100D5000000405DB1C464FF00043524263EB0403E2
:100D6000994208BF904230BD064C074D06E0E0684E
:100D700040F0010394E8070098471034AC42F6D3E2
:100D8000FFF7B8F970FB000890FB0008202A06DB8B
:100D9000CB17203A41FA02F043EAE07306E041FA49
:100DA00002F3D040C2F12002914008431946704737
:100DB0002DE9F34F8BB04FF0000801F10C000C4609
:100DC0004FF0010B46460DF1080A019062690121BE
:100DD00001989047051E2DD0252D2CD0216A8847DB
:100DE000C0B16269012101989047216A88470028B3
:100DF000F7D1411E62690198904700E0761CA16915
:100E00000B988847216A88470028F7D1E1690B9839
:100E10008847DBE7A1690B9888470746A84201D1BC
:100E2000761CD3E7E1690B9888477F1C02D1B8F1A3
:100E3000000F6FD047E1002762693D4639460198AF
:100E400090472A2804D16269012101989047012521
:100E5000DFF888926269012101989047A0F1300182
:100E60000A290AD24F45E5DC07EB870100EB410771
:100E7000303FDFD445F01005ECE7E90601D46FF010
:100E800000476C280AD04C2814D0682815D06A284E
:100E90000DD074281CD07A281AD01DE06269012177
:100EA000019890476C2802D045F0040514E045F005
:100EB00002050DE045F020050AE062690121019874
:100EC0009047682802D045F0080505E045F4006524
:100ED0006269012101989047C4E9015765283DD016
:100EE00019DC58287AD00CDC452837D004DC2528BA
:100EF00026D0412831D131E046282FD047282CD1A7
:100F00002CE05B2877D0612828D063287CD0642827
:100F100023D15AE0D1E06F2848D008DC66281DD0E4
:100F200067281BD0692821D06E2816D127E07028A9
:100F300045D0732868D0752847D078280DD14DE06A
:100F4000A1690B988847054625283FF469AFE169F8
:100F50000B9888476D1C3FF46AAFB4E023466A469D
:100F60006FF001000B99AFF300809FE045F0400067
:100F70006060A80723464FF0000236D43EE0E80741
:100F80007FF447AF2068011D21600068290501D565
:100F900006701BE7290701D5068017E7A90703D5C7
:100FA000F117C0E9006111E706600FE745F0400066
:100FB0006060A80723464FF0080216D41EE040F6F2
:100FC0000E0125EA0100606016E045F04000606017
:100FD000A80723464FF00A0207D40FE045F040006F
:100FE0006060A80708D5234610226FF001000B9916
:100FF000AFF300805AE007E0234610226FF00100B3
:101000000B99FFF795F951E04FF000094F464B4619
:10101000632802D05B2807D041E02079C00601D4C4
:101020000120A06001273AE0626901210198904700
:101030005E2805D14FF00109626949460198904741
:10104000216939B900210A46534643F82120491C39
:101050000829FADBB0B3216969B9C11700EBD16285
:1010600053110AEB830122F01F02821A01200B6840
:10107000904003430B6062690121019890475D280D
:10108000E8D1B9F1000F09D00020514651F82020D5
:10109000D24341F82020401C0828F7DB02AB22464F
:1010A00000976FF001000B99AFF3008000280CDA75
:1010B000401C08D1BBF1000F05D04FF0FF300DB040
:1010C000BDE8F08FFFE74046F9E7E90701D108F1F5
:1010D000010806444FF0000B78E60000CCCCCC0CA5
:1010E00070B58C1810F8015B15F0070301D110F8EA
:1010F000013B2A1106D110F8012B03E010F8016B17
:1011000001F8016B5B1EF9D12B0705D40023521E99
:101110000DD401F8013BFAE710F8013BCB1A921C01
:1011200003E013F8015B01F8015B521EF9D5A142FF
:10113000D8D3002070BD000010B510B14FF0FF30C3
:1011400010BD054813460A4684880068214602F00F
:101150006FF9002010BD0000A0C3000810B510B149
:101160004FF0FF3010BD03488188006802F02AFA72
:10117000002010BDA0C3000818B1012803D0002032
:101180007047024870470248704700003001002055
:101190008801002010B5022806D2FFF7EDFF18B134
:1011A000BDE8104001F094BAFF2010BD32B1054BEC
:1011B00003EB401040F82120002070476FF0010041
:1011C00070470000841F002010B54FF0FF34022844
:1011D00006D2FFF7D1FF18B123B101F05FFE04E0A2
:1011E000204610BD142301F025FC0028F9D0012071
:1011F00010BD38B54FF0FF34049D022806D2FFF72A
:10120000BBFF18B125B101F0C1FD05E0204638BD96
:101210001424009401F0C1FC0028F8D0012038BD4E
:101220002DE9F04107F03CFE06460AF0E1FE4FF4DE
:101230007A78B8FBF6F14FF0E02400FB01F5A769DE
:101240000AF0D6FEB8FBF6F14843A169854206D103
:1012500041464F436169491CB7FBF1F106E04FF489
:101260007A7251436269521CB1FBF2F100EB400209
:10127000C2EBC010C1EBC000002100F57A70BDE8E0
:10128000F081000018B1012803D000207047024807
:101290007047024870470000800500203805002094
:1012A00010B5022802D34FF0FF3010BD31B12AB182
:1012B0003BB1FFF7E7FF02F091FC06E06FF00100A1
:1012C00010BDFFF7DFFF02F0C5FC40B210BDFEE726
:1012D00010B5074C08E000BF10F8013B5340DBB2EB
:1012E00034F8133083EA1222491EF5D2104610BD9D
:1012F000D4DD000800487047C02E002010B5382209
:101300000549064804F0A6F80348083000F0B6F88E
:10131000002800D0012010BDC02E002000F80008D9
:10132000F0B54B4801220223A0F86420A0F8662003
:10133000A0F868300324A0F86A4080F8602071218A
:10134000A0F86210027243490025C0E914150D216E
:1013500080F8581080F85950447280F85A3080F85C
:101360005B3080F85C5080F85D504C2380F847304B
:1013700080F84820202380F84930042680F83B601C
:10138000294680F83930102480F83A4080F83C1023
:10139000C02580F84150342580F84250072580F858
:1013A00043500C2580F82D5080F82E107F2580F8B2
:1013B0002F5080F83030402780F83170EF2780F8C8
:1013C0003E7080F83F20702280F8403080F8262060
:1013D000082780F8277080F8284080F8293080F8A6
:1013E0002A504FF0300C80F82BC000F82C1F4FF023
:1013F000EB0E80F818E0417684768271C671047233
:101400004372857280F80BC0077313A10B790E68C5
:1014100013A10A790D6814A10C68097940F8226CAF
:1014200000F81E3C40F81D5C00F8192C40F8184CE0
:1014300000F8141C0EA110A20B680EA11268096816
:1014400040F8133C40F80F1C40F80B2CF0BD000096
:10145000C02E002080D29990123456789A00000055
:1014600023456789AB0000003456789ABC00000021
:1014700012233445566778899AABBCCD70B5040009
:1014800075D0B4F85C00002871D04FF6FF75A84203
:101490006DD2D4E91201954A821A71F100027FD30C
:1014A000934B0022181A8A417AD394F950001230D3
:1014B000202875D294F85800022871D2B4F85A0046
:1014C000401E7B286CD294F8510010F01F0F67D19A
:1014D0004011072864D894F85200042860D294F888
:1014E000530008285CD294F85400052858D294F888
:1014F0005500052854D294F8350090B101281DD02C
:10150000032835D004284BD194F83F0007F086F823
:10151000002846D094F840000F2841D894F84100A4
:1015200042E094F8360007F079F8002839D094F8B2
:1015300037000F2834D894F8380035E094F8390093
:1015400010F00F0F2CD10011401F072828D894F855
:101550003A000A2805D0182803D0262801D03428BC
:101560001ED194F83B00401E072819D220E017E056
:1015700094F83C0086280FD008DC04280CD02828DA
:101580000AD0452808D069280AD105E0AA2803D046
:10159000C72801D0EB2803D194F83D00042801D9D5
:1015A000002070BD94F83E0007F05CF80028F8D0E9
:1015B000607FC8B1012849D0032861D00428EFD149
:1015C00094F833008028EBD894F831008028E7D8CD
:1015D00094F83200102801D00028E1D194F83400AA
:1015E00031E00828DCD173E0A07F10F00F0FD7D1D5
:1015F00000110728D4D8E07F0928D1D2DFE800F015
:1016000006050605060506050600C9E794F820004C
:1016100010F00F0FC4D100110728C1D894F8210091
:10162000202801D00028BBD194F822000028B8D08F
:1016300094F8230028B1102803D0202801D03028A6
:10164000AED194F824000028CBD141E094F82500D5
:101650000028A6D094F8260008B18028A0D194F8DC
:10166000270000289DD094F82800202801D00028C9
:1016700096D194F8290040282AD0002890D127E05C
:1016800094F82A0010F00F0F8AD10011072887D88C
:1016900094F82B0008B1042882D194F82C0010F0A3
:1016A0000F0FB2D100110728AFD894F82D002028D1
:1016B00001D00028A9D194F82E000028B7D094F8C2
:1016C0002F0028B1102803D0202801D030289CD129
:1016D0005FF0000004EB4001B1F85E10A94294D025
:1016E000401C0328F6DB012070BD000000180D8FA0
:1016F00000F90295014800F01FBA00002402002002
:10170000014800F019BA0000E0010020014800F093
:1017100013BA0000F4020020014800F00DBA0000E6
:1017200068020020014800F007BA0000C805002048
:10173000014800F001BA00000C06002030B590F816
:1017400040500124AC40C56B6C6004686360436822
:10175000102B036803D099600068C26030BD9A60A6
:101760000068C16030BD70474FF4805000F07ABB14
:1017700010B5202000F076FB402000F073FBBDE8A0
:101780001040802000F06EBB72B6FEE7044B0022D2
:10179000DA61044A136943F0010313610180704761
:1017A000500600200020024014480022C168CB06E9
:1017B000134904D5CA6942F00202CA611022C36803
:1017C0005B0705D5CB6943F00103CB6142F004020E
:1017D000C369DB0707D0CB6943F00403CB61C16960
:1017E00021F00101C161A2F58071013901D0C2600F
:1017F0007047C16921F00101C161704700200240BA
:101800005006002070B5054600F032FC0646114C2B
:1018100009E0681C07D025B100F02AFC801BA84213
:1018200001D9032070BDE068C007F2D1E0688006EE
:1018300001D52020E060E068C00605D4E069C0075B
:1018400002D1E068400703D5FFF7AEFF012070BD6D
:10185000002070BD00200240064A0021D1610649E7
:101860000A6942F002020A614861086940F04000DA
:1018700008617047102000200020024030B500248D
:101880002346146019E0401C0578C5B1202DFAD11B
:1018900010F8015F9DB1202DFAD0641C8C420CD150
:1018A00003461168491C116010F8011F09B1202975
:1018B000F7D1106818B9002301E08C42E4D3184630
:1018C00030BD00002DE9F0472F4C05469146606879
:1018D0008A4601264FF00008A0BB04F10C0010E07E
:1018E000006807683846FEF7DCFC0246A85C202842
:1018F00000D020B939462846FEF7DAFC28B16068E6
:10190000406860600028EBD134E0D4F804C0DCF813
:10191000000090F90C70002F10DB002029460246D1
:1019200003E0202B18D00022491C0B78002BF8D1A3
:101930000AB1401E40B2B84200D00026BCF1000FF0
:1019400018D07EB160682A464946006883685046D0
:10195000984706000BD013E0002AE5D1401C40B2A6
:101960000122E1E74A4609495046FEF78EFCC4F8D9
:10197000048005E04A4606495046FEF786FC0026EC
:101980003046BDE8F0870000F400002008F40008AD
:1019900060F4000870B5050011D0082007F080FF42
:1019A000040014D009F0C2FD0020C4E900500C4826
:1019B00001684C60046009F0D9FD012070BD502021
:1019C00080F31188BFF34F8FBFF36F8FFEE7502076
:1019D00080F31188BFF34F8FBFF36F8FFEE70000D6
:1019E000F4000020014600200A0A00D008204FF22F
:1019F000F002114201D040F004004CF6CC421142FA
:101A000001D040F002004AF6AA22114201D040F073
:101A100001007047704700F021BB000070B515460B
:101A20000C460846FFF7DEFF002B0FD0084941F8AF
:101A30002030204603F056F904460022294600F0E3
:101A400089FB2046BDE8704000F076BB70BD000009
:101A500030240020D2B200F006BB10B590F821105F
:101A60000022022905D00421816380F82020012072
:101A700010BD01680B6823F00E030B6001680B6852
:101A800023F001030B6090F84030C46B012101FA90
:101A900003F3636080F8211080F82020104610BD09
:101AA00010B590F821100024022903D0042181638D
:101AB00001243DE001680A6822F00E020A60016814
:101AC0000A6822F001020A601A4A0168914201D1B3
:101AD000012121E0174A1432914201D110211BE06B
:101AE000144A2832914201D1891515E0114A3C323D
:101AF000914201D189140FE00E4A5032914202D135
:101B00004FF4803108E00B4A6432914202D14FF425
:101B1000801101E04FF08071064A083A51600121BE
:101B200080F82110002180F82010416B01B1884716
:101B3000204610BD080002402DE9F05FC16B0C6823
:101B400001680B68D0F840C0042202FA0CF2494D3B
:101B5000DFF824A1494E4A4FDFF828B1DFF828E129
:101B600022422CD05A072AD50A68920603D40A6862
:101B700022F004020A600168A94201D1042219E09E
:101B8000514501D1402215E0B14202D14FF48062AB
:101B900010E0B94202D14FF480420BE0594502D126
:101BA0004FF4802206E0714502D14FF4800201E03B
:101BB0004FF080622F4908394A60C16A3BE04FF01C
:101BC000020808FA0CF818EA040F4FF000094FF069
:101BD000010235D05FEA837832D50B689B0605D4C5
:101BE0000B6823F00A030B6080F821200168A942EA
:101BF00001D1022219E0514501D1202215E0B14264
:101C000002D14FF4007210E0B94202D14FF40052F9
:101C10000BE0594502D14FF4003206E0714502D184
:101C20004FF4001201E04FF00072124908394A6087
:101C300080F82090816A00291AD0BDE8F05F08473B
:101C4000082505FA0CF5254212D01B0710D50B68A4
:101C500023F00E030B6090F84010C36B02FA01F101
:101C60005960826380F8212080F82090016BE2E7C0
:101C7000BDE8F09F080002401C0002403000024016
:101C800044000240580002406C00024030B528B3C6
:101C900008C8134914221944B1FBF2F18900C16349
:101CA00010498163022141771A6843F6F0718A4333
:101CB000D0E900142143D0E902452C4321430469B3
:101CC0002143446921438469214311431960002160
:101CD0004163012242770177084630BD012030BDC3
:101CE000F8FFFDBF0000024070B5044690F82000E8
:101CF000002501280CD0012084F8200094F82160F0
:101D00000020012E06D084F820000225284670BD50
:101D1000022070BD022684F82160A0632068066856
:101D200026F0010606602046FFF708FDE06A00285D
:101D30002068016802D041F00E0106E021F00401A4
:101D400001602068016841F00A01016020680168B3
:101D500041F001010160D9E770B5044600F088F94F
:101D60000546601C02D004480078044400F080F965
:101D7000401BA042FAD370BD08000020034801694F
:101D800041F0800101610020704700000020024006
:101D90002DE9F05F07461C4888460024017E154661
:101DA0001E46012909D00121814601764CF2503AA4
:101DB0005046FFF727FD18B122E00220BDE8F09F52
:101DC000012F02D0022F00D00427D346DFF83CA019
:101DD000220128463146FEF724FA81B208EB44007E
:101DE000FFF7D4FC5846FFF70DFDDAF8102022F07B
:101DF0000102CAF8102018B9641CE4B2BC42E7D34F
:101E0000002289F81820D9E750060020002002405F
:101E1000064900200A69120607D5054A4A60054AA4
:101E20004A600969090600D5012070470020024078
:101E300023016745AB89EFCD2DE9F0410024084F20
:101E40000646012505FA04F0304203D057F8240075
:101E500000B18047641CE4B2102CF3D3BDE8F081DC
:101E6000441F0020044910B50A68024202D00860ED
:101E7000FFF7E2FF10BD0000140401402DE9F84F08
:101E8000DFF8B8910024A9F1040B23460F2709F1CC
:101E9000040AABF1040EC9E00125A5402A40AA427C
:101EA0007DD1674ED1F804C0ACEB0608B44532D002
:101EB00014DCBCF1030F3AD009DCBCF1000F2AD0CE
:101EC000BCF1010F1CD0BCF1020F31D11DE0BCF1FF
:101ED000110F17D0BCF1120F2AD119E0B8F5881FE5
:101EE00019D006DCB8F5803F15D0B8F5801F1FD19A
:101EF00011E0B8F5001F0ED0B8F5041F18D10AE0A4
:101F0000CB6815E0CB681B1D12E0CB6808330FE0EF
:101F1000CB680C330CE08B682BB1012B4FF008031E
:101F200003D0456104E0042302E0056100E00023E2
:101F3000FF2A01D8064601E000F104064FEA8405B5
:101F400001D9A5F12005D6F8008007FA05FC28EA9A
:101F50000C0803FA05F548EA0508C6F800804D6844
:101F6000ED0062D5374DAE6946F00106AE61AD6950
:101F700024F0030605F001050095334D06EB050C32
:101F8000DCF80850A607360F07FA06F825EA080518
:101F9000DFF8B880404503D14FF0000817E044E077
:101FA000DFF8AC80404502D14FF001080FE0DFF8C8
:101FB000A480404502D14FF0020808E0DFF8988085
:101FC000404502D14FF0030801E04FF0040808FA41
:101FD00006F848EA0508CCF808804D68D9F8006092
:101FE000ED024D4601D5164300E096432E604D6844
:101FF000DAF80060AD02554601D5164300E096437D
:102000002E604D68DBF80060AD035D4601D51643D8
:1020100000E096432E604D68DEF80060ED037546E3
:1020200001D5164300E096432E60641C0D682A46D5
:10203000E5407FF431AFBDE8F88F000008040140AF
:102040000000111000100240000001400008014093
:10205000000C01400010014000140140806808405D
:1020600000D0012070470AB1016170470904FBE705
:10207000014880687047000008000020024881681D
:10208000027811448160704708000020074810B5AD
:10209000016841F010010160032000F07BF80F207F
:1020A00000F006F800F024F8002010BD00200240E7
:1020B00070B50D4D04464FF47A712878B1FBF0F0FD
:1020C0000A490968B1FBF0F000F0B4FF48B9102CE0
:1020D00007D200222146501E00F03CF800206C6020
:1020E00070BD012070BD0000080000201400002019
:1020F0000F4808B5816941F001018161816901F0F2
:1021000001010091C16941F08051C161C0690022A3
:1021100000F0805000900F21901E00F01BF8054841
:10212000416821F0E06141F00071416008BD0000AC
:102130000010024000000140002809DB00F01F02EF
:10214000012191404009800000F1E020C0F8001119
:1021500070470000F0B40E4B1B680C46C3F302231B
:10216000C3F10705042D00D90425191D072901D243
:10217000002300E0DB1E012606FA05F1491E21407E
:1021800099409E40761E16403143F0BC05F014BDC8
:102190000CED00E0064900F0070208684FF6FF0367
:1021A000184040EA0220034A1043086070470000CC
:1021B0000CED00E00000FA052DE9F0470F460500A0
:1021C00061D0434E306800F00700B84209D2306851
:1021D00020F0070038433060306800F00700B84254
:1021E00051D128683B4C810712D5400703D5606860
:1021F00040F4E06060602878000703D5606840F430
:10220000605060606068A96820F0F000084360607A
:102210002878C00728D06868012810D021680228D3
:1022200010D0890700292EDA616821F003010143EB
:102230006160FFF71DFF804641F288390DE021689B
:102240008903EFE78901EDE7FFF712FFA0EB080133
:10225000494502D90320BDE8F0876068696800F04D
:102260000C00B0EB810FEFD1306800F00700B842EE
:102270000BD9306820F0070038433060306800F038
:102280000700B84201D00120E5E72878400705D5CE
:102290006068E96820F4E06008436060287800071F
:1022A00006D56068296920F4605040EAC10060608A
:1022B00000F038F86168084AC1F30311515CC84066
:1022C0000649086006480068FFF7F2FE0020C2E7F2
:1022D000002002400010024086C3000814000020C5
:1022E0000C0000200448054900684968044AC1F30D
:1022F0000221515CC84070471400002000100240C9
:1023000096C300080448054900684968044AC1F3B7
:10231000C221515CC84070471400002000100240E8
:1023200096C300080F4A516801F00C00042803D03E
:10233000082803D00C4870470C4870470C48C1F37C
:102340008343C903C05C0AD55168094AC1F34041BF
:10235000921E515C054A5043B0FBF1F070470549AD
:10236000484370470010024000127A000024F40035
:1023700076C3000800093D002DE9F84F040070D035
:102380002078C04DC00749D06868C0F3810001289B
:1023900007D06868C0F38100022809D16868C003CB
:1023A00006D52868800339D560680028E7D035E075
:1023B0006068B0F5803F0BD010B1B0F5A02F11D000
:1023C000286820F480302860286820F4802002E00B
:1023D000286840F480302860606890B1FFF748FEBC
:1023E00006460AE0286840F480202860F0E700BF35
:1023F000FFF73EFE801B642873D828688003F7D55A
:102400000CE0FFF735FE064605E000BFFFF730FEA3
:10241000801B6428F0D828688003F7D420789A4E6F
:1024200080074FF001094FF0000839D5686810F0B7
:102430000C0F07D06868C0F38100022809D16868D2
:10244000C00306D42868800714D52069012808D164
:1024500010E02069B0B1C6F80090FFF709FE07460A
:1024600005E00AE1FFF704FEC01B0228C4D8286873
:102470008007F7D52868616920F0F80040EAC100BC
:1024800028600DE0C6F80080FFF7F2FD074604E083
:10249000FFF7EEFDC01B022823D828688007F7D479
:1024A000207800072CD57948A169D9B1C0F80090EF
:1024B000FFF7DEFD074604E0FFF7DAFDC01B022848
:1024C0000FD8686A8007F7D571484FF4FA51006851
:1024D000B0FBF1F0009000BF0098411E0091FAD2CD
:1024E0000EE080E0C0F80080FFF7C2FD074604E080
:1024F000FFF7BEFDC01B022875D8686A8007F7D4B5
:102500002078400760D5E8690027C00008D4E86952
:1025100040F08050E861E869012700F080500090A9
:102520005C480168C90513D40168834641F4807191
:102530000160FFF79DFD824606E000BFFFF798FDB2
:10254000A0EB0A0064284ED8DBF80000C005F5D5E2
:10255000E06801280AD008B1052813D0286A20F0C5
:1025600001002862286A20F0040002E0286A40F096
:1025700001002862E06841F2883B98B1FFF778FDDE
:1025800082460BE0286A40F004002862EEE700BFB4
:10259000FFF76EFDA0EB0A0159455AD8286A80075B
:1025A000F6D50CE0FFF764FD824605E0FFF760FD1D
:1025B000A0EB0A0159454CD8286A8007F6D41FB110
:1025C000E86920F08050E861E06988B36968C1F388
:1025D0008101022944D00228C6F8608004D0FFF7A8
:1025E00047FD044638E034E0FFF742FD074604E0CB
:1025F000FFF73EFDC01B02282BD828688001F7D4C6
:10260000206AB0F5803F05D16868A16820F40030E9
:1026100008436860D4E908010843696821F474112B
:1026200008436860C6F86090FFF722FD044606E0A4
:1026300025E000BFFFF71CFD001B022809D8286811
:102640008001F7D51BE000BFFFF712FD001B022839
:1026500002D90320BDE8F88F28688001F4D40EE089
:102660000128F7D06868226A00F48031914204D1D1
:10267000616A00F47010884201D00120EAE700206E
:10268000E8E700000010024000004242800442429D
:10269000140000200070004070B5044602F06CFE8B
:1026A000032811D0204602F067FE084D05EB4010CC
:1026B0008069002808D0204602F05EFE05EB40103D
:1026C0008069BDE87040004770BD0000841F002095
:1026D00090F851007047000038B504460068426821
:1026E0008168C9434B0606D5CB0704D1D3435B06AB
:1026F00001D4216C05E08B0708D4D3431B0605D415
:10270000616C01B02046BDE8304008478B0601D51A
:102710004B0646D4D3439B0643D44B060AD494F8C5
:102720005130032B3ED0636D43F004036365C368EF
:1027300083680093890609D4616D41F001016165E8
:1027400081680091016821F040010160606D0028FE
:1027500027D02068416821F0E0014160012084F821
:102760005100900722D02068416821F003014160A8
:10277000104DE06C40B14563E06CFFF791F918B182
:10278000606D40F040006065A06C002809D0456392
:10279000A06CFFF785F9002803D0606D40F0400081
:1027A000606538BDC1688068009038BD2046FFF77D
:1027B00073FF38BD7151000870B5040009D0606A1C
:1027C000002540B125616561A56294F8510040B1D2
:1027D0000CE0012070BD6068B0F5827FF4D0E56147
:1027E000F2E784F85050204600F040F8022084F8C8
:1027F00051002068016821F040010160A088218912
:1028000000F4827001F404410843A18901F40061DD
:102810000843217C01F002010843217D01F0010100
:102820000843218B01F400710843217F01F0380136
:10283000084394F8201001F080010843218D01F431
:102840000051084321680860A069042101EA104092
:10285000216848602068C16921F40061C161656533
:10286000012084F85100002070BD00002DE9F041E6
:1028700086B00024009401940294039406464A4DC5
:1028800003684A480221032210274FF08008AB4218
:102890004ED1836943F480538361836903F4805389
:1028A0000493836943F0040383618069404D00F021
:1028B00004000490A020CDE9000103926946284657
:1028C000FFF7DCFA4020CDE900046946284602946F
:1028D000FFF7D4FA384D3748C5E90007C5E9024883
:1028E0002C616C61AC6147462846EC61FFF7CEF97C
:1028F00008B1FEF749FFB5646E622F4D2D4844358F
:102900001438C5E90004C5E902472C616C61AC616B
:102910002846EC61FFF7BAF908B1FEF735FFF56418
:102920000022052123206E62FFF714FC232035E0EE
:10293000224DAB4234D1C36943F48043C361C369C0
:1029400003F480430493836943F00803836180693F
:10295000039200F0080004904FF42040CDE90001FC
:1029600069461748FFF78AFA134D12488835283010
:102970002860C5E90174C5E903846C61AC6128462F
:10298000EC61FFF783F908B1FEF7FEFEB5640022A3
:10299000052124206E62FFF7DDFB2420FFF7CCFB2E
:1029A00006B0BDE8F0810000003001400010024098
:1029B0000008014030000240E001002000380040E3
:1029C000000C014070B5044602F0D6FC032811D07B
:1029D000204602F0D1FC084D05EB4010406800286D
:1029E00008D0204602F0C8FC05EB40104068BDE866
:1029F0007040004770BD0000841F002070B5044681
:102A000002F0BAFC032811D0204602F0B5FC084DB4
:102A100005EB40100069002808D0204602F0ACFC0D
:102A200005EB40100069BDE87040004770BD000034
:102A3000841F00202DE9F84F984616468A46044622
:102A4000FFF716FB814694F8510001281ED1BAF118
:102A5000000F73D0002E71D094F85000012815D0CB
:102A6000012784F85070032084F851000025656523
:102A7000C4F830A0A686E686A563A587E5876564C9
:102A80002564A068B0F5004F03D00CE00220BDE83B
:102A9000F88F2068016821F040010160206801681A
:102AA00041F48041016020680168490603D401684F
:102AB00041F040010160E068B0F5006F606803D04C
:102AC00048B3012E27D047E008B1012E1FD1206B5B
:102AD00021680088C86006E020688168890709D5F8
:102AE000216B0988C160206B801C2063E08E401E32
:102AF000E0860CE0FFF7BCFAA0EB0901414503D3E7
:102B0000B8F1FF3F03D035E0B8F1000F32D0E08ECE
:102B10000028E1D123E0206B21680078087306E0EB
:102B20002068816889070AD5216B09780173206BB9
:102B3000401C2063E08E401EE0860DE02BE0FFF796
:102B400097FAA0EB0901414503D3B8F1FF3F03D049
:102B500010E0B8F1000F0DD0E08E0028E0D14A4619
:102B60004146204602F0EEFB08B120206065A068D7
:102B700030B109E084F8517084F85050032086E7A2
:102B80002068C1688068009084F8517004F8505F34
:102B900060680028F3D0012079E72DE9FF4F81B06C
:102BA0001D46934604464FF001090E9EFFF760FA5A
:102BB000074694F851006168012806D0B1F5827F7C
:102BC0003CD1A168C9BB042838D10298002871D033
:102BD000BBF1000FFBD0002DF9D094F85000012874
:102BE0002CD04FF0010A84F850A094F8510004282A
:102BF00002D0052084F851004FF00008C4F854803A
:102C0000C4F838B0E587A58702992163E586A586D3
:102C1000C4F84080C4F8448020680168490603D4A1
:102C2000016841F040010160E068B0F5006F606844
:102C300008D0F0B3012D49D081E0FFE7022005B0B4
:102C4000BDE8F08F08B1012D39D1206B21680088D3
:102C5000C860206B801C2063E08E401EE0862EE062
:102C60002068816889070FD5E18E69B1B9F1010F3C
:102C70000AD1216B0988C160206B801C2063E08E23
:102C8000401EE0864FF0000920688168C9070CD01B
:102C9000E18F51B1C068A16B0880A06B801CA0635C
:102CA000E08F401EE0874FF00109FFF7E1F9C01BFC
:102CB00001E00BE067E0B04201D3701C50D1E08E20
:102CC0000028CDD1E08F0028CAD13EE0206B2168DA
:102CD00000780873206B401C2063E08E401EE08665
:102CE0002DE02068816889070FD5E18E69B1B9F1BF
:102CF000010F0AD1216B09780173206B401C2063FE
:102D0000E08E401EE0864FF0000920688168C90708
:102D10000CD0E18F51B1C068A16B0870A06B401C52
:102D2000A063E08F401EE0874FF00109FFF7A0F994
:102D3000C01BB04202D3701C01D011E086B1E08EFE
:102D40000028CED1E08F0028CBD13A46314620462C
:102D500002F0F8FA50B12020606584F8508012E04B
:102D600084F851A084F85080032068E7A06818B95F
:102D70002068C1688068009084F851A084F8508071
:102D8000606D0028F1D0012059E7000070B50446BD
:102D900090F851006568012806D0B5F5827F3AD1D8
:102DA000A568A5BB042836D191B38AB383B394F840
:102DB000500001282FD0012084F8500094F85100D1
:102DC000042802D0052084F85100002565652163A0
:102DD000A386E386A263A387E3872564656494F8EA
:102DE0005100042819D0E16C2748C8622748E16CDB
:102DF0008862E16C26480863E06C4563E38F2168D4
:102E0000A26B0C31E06CFEF76FFF00BB0AE002E042
:102E1000FFE7012070BD022070BDE16C1D48C86253
:102E20001D48E4E72068416841F001014160A06C61
:102E3000C562A06C8562A06C0563A06C4563E38EDF
:102E40002268216B0C32A06CFEF74EFF30B1606D32
:102E500040F01000606584F85050DAE7206801689F
:102E6000490603D4016841F04001016084F85050E4
:102E70002068416841F0200141602068416841F0CC
:102E800002014160002070BDB75100088F52000858
:102E900081510008A3510008C151000870B50446D3
:102EA00090F8510001281CD1C9B1C2B194F850006A
:102EB000012816D0012084F85000032084F8510026
:102EC000002565652163A286E286A56365642564A5
:102ED000A587E587A068B0F5004F04D00DE001207C
:102EE00070BD022070BD2068016821F040010160C2
:102EF0002068016841F480410160A16C1748C862F4
:102F0000A16C17488862A16C16480863A06C4563E1
:102F1000E38E2268216B0C32A06CFEF7E5FE30B127
:102F2000606D40F01000606584F85050D7E720686D
:102F30000168490603D4016841F04001016084F84A
:102F400050502068416841F020014160206841688C
:102F500041F002014160002070BD0000AD51000849
:102F60002B5200088151000810B502F005FA032821
:102F700008D0054901EB40100068002802D0BDE8E8
:102F80001040004710BD0000841F002070B50446AB
:102F900002F0F2F9032811D0204602F0EDF9084DB5
:102FA00005EB4010C068002808D0204602F0E4F984
:102FB00005EB4010C068BDE87040004770BD0000E0
:102FC000841F002070B5044602F0D6F9032811D002
:102FD000204602F0D1F9084D05EB4010806800282A
:102FE00008D0204602F0C8F905EB40108068BDE823
:102FF0007040004770BD0000841F002070B504467B
:1030000002F0BAF9032811D0204602F0B5F9084DB4
:1030100005EB40104069002808D0204602F0ACF9CA
:1030200005EB40104069BDE87040004770BD0000EE
:10303000841F002010B5401EB0F1807F01D3012015
:1030400010BD4FF0E02460610F21601704F0B4FD63
:103050000020A06107202061002010BD10B590F86D
:103060003C20012A22D0012280F83C20CA688C68CA
:1030700022F4407222434C6822F4806222430C689E
:1030800022F4006222430C6922F4805222434C69EC
:1030900022F400522243C969002322F480420A43E9
:1030A00001684A6480F83C30002010BD022010BD49
:1030B00070B590F83C20012A26D0012480F83C40CD
:1030C000022280F83D2003685A689D6822F070064D
:1030D0000A6832435A600D4B02689A4208D0B2F136
:1030E000804F05D00A4B9A4202D00A4B9A4204D133
:1030F000496825F080031943916080F83D40002124
:1031000080F83C10084670BD022070BD002C0140C4
:10311000000400400008004010B5040003D094F8FB
:103120003D0010B107E0012010BD002084F83C00F4
:10313000204600F01FF8022084F83D00211D206881
:1031400003F026FF012084F8460084F83E0084F84E
:103150003F0084F8400084F8410084F8420084F87D
:10316000430084F8440084F8450084F83D000020C2
:1031700010BD000038B5054600681349884221D1CA
:103180001248816941F4006181618069114C00F449
:10319000006000900E4820601020606000208021B8
:1031A000C4E90201890021618900C4E90510E061D8
:1031B0002046FEF76BFD08B1FEF7E6FA2C63AC6320
:1031C0006C63656238BD0000002C014000100240B5
:1031D00044000240F402002070B5044690F83C0020
:1031E0000025012817D0012684F83C60022084F8CD
:1031F0003D002068826822F0770222F47F428260DC
:103200000868502838D00DDC20284FD005DC90B35A
:10321000102811D14AE0022070BD302846D0402845
:103220000AD13BE060282FD070280DD0B0F5805F28
:1032300003D0B0F5005F12D0012584F83D60002076
:1032400084F83C00284670BDCB68D1E90121206894
:1032500003F05CFF2068816841F0770109E0CB68EA
:10326000D1E90121206803F051FF2068816841F411
:1032700080418160E1E719E0CA684968206803F08D
:10328000F9FF5021206806E0CA684968206804F008
:1032900002F86021206803F043FFCEE7CA6849685E
:1032A000206803F0E7FF40212068F4E72268014628
:1032B0001046F0E77047000000B585B0002100918E
:1032C00001910291039100680B49884212D10B4889
:1032D000816941F0040181618069694600F0040060
:1032E00004904FF400600090022001900390044885
:1032F000FEF7C4FD05B000BD002C014000100240E7
:103300000008014070B5044690F83C0000260D46C8
:1033100001280FD0012084F83C006AB1042A1DD096
:10332000082A2FD00C2A3FD00126002084F83C0028
:10333000304670BD022070BD206803F0F9FE2068A1
:10334000816941F0080181612068816921F00401EF
:103350008161206881692A69114311E0206803F0C6
:103360000FFF2068816941F40061816120688169F3
:1033700021F480618161206881692A6941EA022122
:103380008161D2E7206803F027FF2068C16941F01E
:103390000801C1612068C16921F00401C161206890
:1033A000C1692A69114311E0206803F041FF2068D8
:1033B000C16941F40061C1612068C16921F4806183
:1033C000C1612068C1692A6941EA0221C161ACE793
:1033D00010B5040003D094F83D0010B107E00120BF
:1033E00010BD002084F83C00204600F01EF80220AA
:1033F00084F83D00211D206803F0CAFD012084F8F7
:10340000460084F83E0084F83F0084F8400084F8C9
:10341000410084F8420084F8430084F8440084F8B2
:10342000450084F83D00002010BD7047704770478C
:103430002DE9F04117460D0004464FF000060CD070
:10344000042D11D0082D16D094F84100022819D06F
:1034500094F84100012818D07CE094F83E0002283E
:1034600010D094F83E00F5E794F83F00022809D008
:1034700094F83F00EEE794F84000022802D094F858
:103480004000E7E70220BDE8F081002F62D0002B6A
:1034900060D04649464ADFF81CC102204DB1042DD8
:1034A00018D0082D27D084F841000C2D44D00126D7
:1034B00079E084F83E00606A8162606A3946C262DF
:1034C000606AC0F830C02268606A3432FEF70CFCD3
:1034D00088BB21E084F83F00A06A8162A06A394677
:1034E000C262A06AC0F830C02268A06A3832FEF713
:1034F000FBFB00BB15E084F84000E06A8162E06AF3
:103500003946C262E06AC0F830C02268E06A3C32E4
:10351000FEF7EAFB78B909E02068C16841F4007160
:103520001EE02068C16841F4806119E02068C1682C
:1035300041F4006114E00DE0206B8162206B39469C
:10354000C262206BC0F830C02268206B4032FEF7A8
:10355000CBFB08B1012096E72068C16841F4805197
:10356000C16001222946206803F04EFD12492068FF
:10357000884203D1426C42F400424264206888428F
:1035800008D0B0F1804F05D00C49884202D00C49D8
:10359000884204D1816801F00701062903D001683F
:1035A00041F00101016030466DE700002370000822
:1035B00081700008B9700008002C01400004004030
:1035C0000008004030B504460D460068002203F0B4
:1035D0001BFD174B41F2111120688A10984209D146
:1035E000036A0B4206D1036A134203D1436C23F4EE
:1035F000004343642068036A0B4206D1016A11420A
:1036000003D1016821F00101016001203DB1042DC9
:1036100008D0082D09D084F84100002030BD84F87E
:103620003E00FAE784F83F00F7E784F84000F4E74B
:10363000002C0140704710B504460068406994F8BA
:103640004110C0F3C010212911D180B1206814307D
:1036500050E8001F21F0800140E80012002AF5D157
:10366000A06B08B1FEF7F9F9204603F067FF206868
:10367000406994F84210C0F38010222911D180B122
:103680002068143050E8001F21F0400140E800128B
:10369000002AF5D1E06B08B1FEF7DFF9204603F010
:1036A00026FF002010BD000010B503F055FF0328D1
:1036B0000AD000EBC001054800EB8100006900283A
:1036C00002D0BDE81040004710BD0000C41F00201C
:1036D000F8B5016804460868CA684B6910F00F0F16
:1036E0004FF0000559D003F0010602F490773743FC
:1036F00065D0C10705D0D10503D5616C41F001014A
:103700006164410705D5D90703D0616C41F002011E
:103710006164810705D5D90703D0616C41F00401CC
:103720006164010707D502F02001314303D0616CC9
:1037300041F008016164616C00293AD0800604D52B
:10374000900602D5204603F019FF20684069616C9D
:10375000C0F38010090700D460B3204603F0C7FE11
:1037600020684069400621D52068143050E8001FC9
:1037700021F0400140E80012002AF5D1E06BA8B129
:103780006D494163E06BFEF78BF9002811D0E06BC7
:10379000416B01B0BDE8F040084783060FD59306A2
:1037A0000DD52046BDE8F84003F0E8BE2046FFF7FF
:1037B0007BFFF8BD2046FFF777FF6564F8BD266BF9
:1037C0002023012E7CD1C6067AD5D60678D5086886
:1037D0004868009048694FF00206400640D5E16B0A
:1037E000086840680004000CE8D0A28D8242E5D948
:1037F000E085886920282DD020680C3050E8001F13
:1038000021F4807140E80012002AF5D120681430BC
:1038100050E8001F21F0010140E80012002AF5D114
:103820002068143050E8001F21F0400140E80012E9
:10383000002AF5D184F84230256320680C3050E826
:10384000001F21F0100140E80012002AF5D1E06BC2
:10385000FEF703F96663A08DE18D401A81B22AE07C
:10386000A08DE18D401A81B2E08D0028A6D00029FC
:10387000A4D022680C3252E8000F20F4907042E885
:103880000007002FF5D12068143050E8002F22F0F7
:10389000010240E80027002FF5D184F8423025636B
:1038A00020680C3050E8002F22F0100240E800237E
:1038B000002BF5D166632046FFF7BCFEF8BDFFE79D
:1038C00005062BD5150629D594F841002128F5D1F8
:1038D000A068B0F5805F01D12069B0B1206A411CB9
:1038E0002162216800784860E08C401E0004000CD2
:1038F000E084E3D12068C16821F08001C1602068C4
:10390000C16841F04001C160D8E7206A0088C0F377
:1039100008004860206A801C2062E5E74006CDD59B
:103920005006CBD5CA68204622F04002CA6084F80F
:10393000413000F0A9F9C1E7A573000870B5040093
:1039400004D094F84100002510B106E0012070BDBC
:1039500084F84050204600F023F8242084F84100E9
:103960002068C16821F40051C160204603F068FE60
:103970002068016921F4904101612068416921F0CA
:103980002A0141612068C16841F40051C160656449
:10399000202084F8410084F842006563002070BD57
:1039A000F0B585B000240094019402940394064677
:1039B000414F0368414802210322414DBB4226D1B9
:1039C000836943F480438361836903F480430493F0
:1039D000836943F0040383618069039200F004006B
:1039E00004900802CDE9000169462846FEF746FA30
:1039F0002815CDE90004694628460294FEF73EFAF0
:103A0000002205212520FEF7A5FB252050E02D4FA3
:103A1000BB424FD1C36943F40033C361C36903F4AC
:103A200000330493836943F0040383618069039244
:103A300000F0040004900420CDE900016946284606
:103A4000FEF71CFA0820CDE90004694628460294D6
:103A5000FEF714FA1D4D1C488027C5E90004C5E98E
:103A600002472C616C61AC612846EC61FEF70EF9EF
:103A700008B1FDF789FEF5636E62144D12484435B6
:103A8000143001C5102091C5104845F81049443044
:103A90006C61AC61EC61FEF7F9F808B1FDF774FEFA
:103AA000B5630022052126206E62FEF753FB262017
:103AB000FEF742FB05B0F0BD0038014000100240A7
:103AC00000080140004400406C000240C80500208E
:103AD00090F84230202B01D00220704721B11AB15A
:103AE0000023036303F008BE0120704710B503F004
:103AF00033FD03280AD000EBC001054800EB81002C
:103B0000C068002802D0BDE81040004710BD00008A
:103B1000C41F002010B503F01FFD03280AD000EBDE
:103B2000C001054800EB81008068002802D0BDE894
:103B30001040004710BD0000C41F00202DE9F843CD
:103B4000044690F84100984616460D46202802D0BB
:103B50000220BDE8F88385B17EB100206064212099
:103B600084F84100FEF784FAA6848146E684A068C2
:103B70002027B0F5805F02D003E00120E9E720694B
:103B800010B12E4600250EE000260CE080212046D4
:103B900003F0FAFDA8B9C6B116F8010B2168486018
:103BA000E08C401EE084E08C4B464FF00002CDF8E4
:103BB00000800028EAD14FF04001204603F0E4FDE8
:103BC00040B184F841700320C3E735F8020BC0F31D
:103BD0000800E3E784F841700020BAE770B50446B6
:103BE00090F84100202801D0022070BD49B342B3B3
:103BF0002162A284E28400206064212384F84130A1
:103C0000A56B114BAB62A56B104BEB62A56B104B18
:103C10002B63A36B5863256813462A1DA06BFEF720
:103C200063F821686FF0400008602068143050E8A5
:103C3000001F41F0800140E80012002AF5D1002069
:103C400070BD012070BD0000A3740008E574000879
:103C5000B573000890F84130202B01D00220704746
:103C600079B172B101628284C28400214164212150
:103C700080F841100068C16841F08001C1600020F7
:103C8000704701207047000010B503F065FC032861
:103C90000AD000EBC001054800EB81004068002815
:103CA00002D0BDE81040004710BD0000C41F002036
:103CB00010B503F051FC032809D000EBC001044803
:103CC00050F82100002802D0BDE81040004710BD88
:103CD000C41F0020FEE72DE9F041070AC6B200210B
:103CE000F0238722084600F0FBFA4FF48770044661
:103CF00004F0DAFC050014D0002029182F54801C91
:103D00004E70A042F9D300262146284600F060FB01
:103D1000761CF02EF8D3284604F01EFC0020BDE8E7
:103D2000F0816FF00100FAE72DE9FF5F1F465FEABF
:103D3000000B04D0F81D4FEAD00800262CE06FF0ED
:103D4000010004B0BDE8F09F06FB08BA00251FE0A3
:103D50001AF805905FF0000404EBC50080B2B84289
:103D600014D2109901291CD00121A14011EA090F98
:103D700008D0019A02991044314489B280B20F9A56
:103D800000F064F9641CE4B2082CE5D36D1CADB2FC
:103D90004545DDD3761CB6B20E988642D4D30020BA
:103DA000CFE78021E140E1E72DE9FF4F8BB08A4664
:103DB000DDE91817203A06464FF0FF335F2A08D294
:103DC000D0B20C296AD0102907D0182932D0202966
:103DD00064D018460FB0BDE8F08F31494FF0080BA2
:103DE00001EB0010029010200025009002980024A2
:103DF0000AEB050910F80580301983B21FFA89F122
:103E0000012F12D028FA04F010F0010F03D0184649
:103E10000E9A00F01BF9641CE4B25C45ECD36D1CF7
:103E20000098EDB28542E1D338E0C4F1070228FAE8
:103E300002F0E9E71B4900EB400001EB00100290A3
:103E40001820009002204FF00C0B002507900799D6
:103E500000240AEB050905FB01F83019DDF808C05C
:103E600083B20CEBD4001FFA89F118F80000012F7F
:103E700004F0070201D1C2F10702D04010F0010F97
:103E800003D018460E9A00F0E1F8641CE4B25C45D9
:103E9000E3D36D1C0098EDB28542D8D3002099E79A
:103EA000A8C3000898C900082DE9FF4F8BB08A46C7
:103EB000DDE91937203A06464FF0FF315F2A08D274
:103EC000D0B20C2B6CD0102B07D0182B34D0202B59
:103ED00066D008460FB0BDE8F08F32494FF0080BAE
:103EE00001EB0010029010200025009002980024A1
:103EF0000AEB050910F80580301983B21FFA89F121
:103F0000012F06D028FA04F010F0010F06D00E9A07
:103F100005E0C4F1070228FA02F0F5E7189A1846FE
:103F200000F094F8641CE4B25C45E5D36D1C009885
:103F3000EDB28542DAD333E01B4900EB400001EBE0
:103F4000001B0C20019018200090022000250990F1
:103F5000099800240AEB050905FB00F8301983B223
:103F60000BEBD4001FFA89F118F80000012F04F0C0
:103F7000070201D1C2F10702D04010F0010F01D0B9
:103F80000E9A00E0189A184600F060F8641C019838
:103F9000E4B28442E2D36D1C0098EDB28542D7D3DF
:103FA000002097E7A8C3000898C900082DE9F05F32
:103FB000141AA3EB01054FF0FF3201D4012300E0F6
:103FC00013469B46002D00DB01229246002C00DAAE
:103FD0006442002D00DA6D4254EA050208D0AC427A
:103FE0001ADD04EBD472561080468946002710E093
:103FF0000A9A00F02BF826E01FFA89F11FFA88F0E0
:104000000A9A00F023F8D844761B01D5D1442644FF
:104010007F1CA742F0DD16E005EBD57256108146F5
:10402000884600270DE000BF1FFA88F11FFA89F0CB
:104030000A9A00F00BF8D044361B01D5D9442E441F
:104040007F1CAF42F0DD0020BDE8F09F38B503468D
:1040500014481446007828B1012813D0022815D03E
:10406000032818D0184601231A4600F039F9200A0F
:104070008DF800008DF801400221684600F0A2F999
:10408000002038BD0846C3F1EF0109E0C1F1860008
:1040900080B21946E7E7C3F1860080B2C1F1EF01B3
:1040A00089B2E0E7980000202DE9FF4F83B08146F8
:1040B000DDE910AB0546144688465046BAF10C0FB0
:1040C0001CD0102808D0182809D0202816D04FF06E
:1040D000FF3007B0BDE8F08F092711260EE00D274D
:1040E00019260BE00A2A0ED0CDE900AB414628463E
:1040F000069BFFF759FEE81985B2641C2278002A56
:10410000F0D10020E5E708EB06004D461FFA80F8E5
:10411000F3E72DE9FF4F83B08146DDE911AB05469A
:10412000144688465046BAF10C0F1DD0102808D00E
:10413000182809D0202817D04FF0FF3007B0BDE86D
:10414000F08F092711260FE00D2719260CE00A2A07
:104150000FD0109B41468DE8080C2846069BFFF7C0
:10416000A3FEE81985B2641C2278002AEFD1002052
:10417000E4E708EB06004D461FFA80F8F3E700007D
:1041800070B504464A488AB04A4E04704FF48045E0
:10419000002229463046FDF766FF3220FDF7DCFDA0
:1041A000012229463046FDF75EFF3220FDF7D4FD9F
:1041B000362000F0C7F834B1012C06D0022C73D0A1
:1041C000032C05D172E0082000E0602000F0DAF84E
:1041D0003A2000F0B7F8052000F0D4F8B22000F043
:1041E000B1F835A1D1E90001CDE90801052108A800
:1041F00000F0E8F8B72000F0A5F8352000F0C2F88C
:10420000BB2000F09FF8192000F0BCF8C02000F09F
:1042100099F82C2000F0B6F8C22000F093F80120A5
:1042200000F0B0F8C32000F08DF8122000F0AAF8DA
:10423000C42000F087F8202000F0A4F8C62000F089
:1042400081F80F2000F09EF8D02000F07BF8A42029
:1042500000F098F8A12000F095F8E02000F072F846
:1042600017A00FC88DE80F000E21684600F0AAF8CD
:10427000E12000F067F816A104AC0FC984E80F0034
:104280000E2104A800F09EF8212000F05BF8112018
:1042900000F058F87820FDF75FFD292000F052F873
:1042A0000AB0002070BDFFE7A0208FE7C8208DE78F
:1042B00098000020000C01400C0C0033330000007B
:1042C000D0040D11132B3F544C180D0B1F2300006D
:1042D000D0040C11132C3F44512F1F1F202300002A
:1042E0002DE9FC4100F1340401F12807A518FE185E
:1042F0002A206D1E761E00F025F8200A8DF8000099
:104300008DF80140280A8DF802008DF80350042131
:10431000684600F057F82B2000F014F8380A8DF8A2
:1043200004008DF80570300A8DF806008DF80760DE
:10433000042101A800F046F82C2000F003F800202A
:10434000BDE8FC8131B500224FF480710B48FDF7C8
:104350008AFE0B4D4FF48054002221462846FDF77B
:1043600082FE01231A4669461846FCF72DFF0122FA
:1043700021462846FDF777FE002038BD00080140A1
:10438000000C014031B5012211020C48FDF76BFE13
:104390000B4D4FF48054002221462846FDF763FE62
:1043A00001231A4669461846FCF70EFF01222146F2
:1043B0002846FDF758FE002038BD000000080140E7
:1043C000000C014010B500F003F8002010BD000003
:1043D0002DE9F0410C460546012211020E48FDF779
:1043E00042FE0E4F4FF48056002231463846FDF70C
:1043F0003AFE0123224629461846FCF7E5FE012035
:10440000FCF7C8FE0128FAD1012231463846FDF7F3
:104410002AFE0020BDE8F08100080140000C0140A8
:1044200010B50848FDF7B6FA4FF0FF34012805D162
:1044300004481030FDF7AEFA012801D0204610BD27
:10444000002010BDD4F2000870B505004FF0FF3415
:1044500017D0B1B1FCF752FFA8B13AA003F082FB2C
:10446000202105F10800FBF705FFFFF7D9FFFCF756
:1044700041FF08302860427801463E4802F0CCF8FF
:1044800028B1204670BDFCF74BFF3BA0E6E7464E47
:104490000020B16B88472868364C90F8581011B14D
:1044A00001291DD108E061687F2081F8270061683B
:1044B00081F82E00616811E090F85A006168001DD3
:1044C00081F827002868616890F85A00001D81F87B
:1044D0002E002868616890F85A00001D81F82200BB
:1044E0006068716C1D30884760680078022802D0CF
:1044F000012804D018E01F4802F098FC14E0286856
:1045000090F8581011B101290ED102E02748007827
:1045100003E0B0F85A00001D80B228B1C2B205F124
:104520002801144802F09CFC0120FFF729FE00F04E
:1045300029FB40F2DC50FDF70FFC284600F056F94D
:10454000002070BD5B4D5231365D20436F6E666951
:1045500067206C6F616465642066726F6D20466CC5
:10456000617368207375636365737366756C6C79CA
:104570000D0A0000702C00205B4D5231365D204644
:104580006C61736820636F6E66696720696E76611F
:104590006C69642C207573696E672064656661754B
:1045A0006C74730D0A000000F0DC000805000020A8
:1045B0002DE9F047DFF8C091044699F80000DFF8D4
:1045C000BC81002500285BD0424600206C4912784F
:1045D000464601E0401CC0B2904208D20B5C202B42
:1045E000F8D0092BF6D00D2BF4D00A2BF2D0904244
:1045F00007D2085CA0F16101192908D941381928AE
:1046000005D922B15E49204600F0C8F833E05D4F7D
:104610009AB1402A11D25A493846FBF712FE307837
:1046200000E0401E00283D5408DD391811F8011C37
:104630000D29F6D00A29F4D000E03D705248816B74
:1046400000208847042003F033FA4E4E4FF4807A5E
:10465000403635704B49524640314A48FDF732F9F1
:104660000746307820B1474948A0403103F07AFA34
:104670003570012FEED0042003F01AFA89F80050AB
:10468000FCF7CEFDFCF7E2F8414E3146FBF7BFFFE9
:10469000A060FCF7C5FDD4E90423801A61EB030197
:1046A000FCF7D4F83146FBF7B2FFA061FCF7B8FD88
:1046B000384EC4E904017068007802282DD1616A7F
:1046C000A068FBF79EFF3449884226DD2068B0F8D9
:1046D0005C10090A84F8281090F85C1084F82910FE
:1046E000FF2184F82A1084F82B5084F82C1084F8C9
:1046F0002D5090F8581029B1B0F85A00001D81B221
:10470000062008E098F80010091DF9E72218401C5F
:1047100082F8285080B28842F8D3206890F8580078
:1047200010B1012821D106E070680078012809D075
:1047300002281AD106E070680078012802D0022809
:1047400013D103E0134802F029FA0EE0114802F0F9
:1047500025FAE169A068FBF754FFB0F17E5F04DB46
:10476000204600F06BFAA068E061FDF781FC03F0E1
:10477000A5F90020BDE8F087040000200500002016
:10478000370400207F2D0020F0DC00082573000096
:1047900000247449702C0020CDCCCC3D70B515465A
:1047A000040003D011B10DB17B2D02D94FF0FF30C1
:1047B00070BD206830F85C2F120A84F82820007839
:1047C00084F829002A4604F12A00FBF73AFD4FF647
:1047D000FF72A91C04F12800FCF77AFD020A611996
:1047E00001F82A2F4870002070BD00002DE9F04F1D
:1047F00091B004005CD02068002859D00020FFF759
:104800006AFA00251826CDE9006505214DF6A703B3
:10481000A8A20846FFF748FCDFF8A4A24FF4FC6703
:104820004FF6205B9AF80000012846D03B46A5A22F
:10483000CDE900650521C820FFF736FC48F210409D
:104840001E230090872219460020FFF7AFFB102699
:10485000CDE9006540F2FF7843469BA22821052060
:10486000FFF722FC20684FF6FF794B4690F858007E
:1048700030B3012826D096A24AF65553CDE90065FB
:1048800028214120FFF710FCCDE90065434692A2A4
:1048900041210520FFF708FCDAF804008CA2407FD4
:1048A000A8B1012815D0032815D0042814D10CE094
:1048B0004FF0FF3011B0BDE8F08F5B4688A2B7E73C
:1048C00088A2DBE78AA23B46D8E78BA204E08BA252
:1048D00002E08CA200E08DA2CDE9006541214B46AB
:1048E0000846FFF7E1FBCDE90065434689A25A215E
:1048F0000520FFF7D9FBDAF80410884A0023D1E934
:104900001201FBF75DFCCDE9000185A20F2107A88C
:1049100003F038F9CDE900654B4607AA5A21322049
:10492000FFF7C2FB9AF800002321012870D0CDE9DF
:10493000006543467CA27820FFF7B6FB4FF0370AAC
:104940007CA2142102A8D4F8A83003F01BF9CDE909
:1049500000653B4602AA51467820FFF7A5FB4FF0C1
:104960004B0A76A2142102A8D4F8AC3003F00AF95D
:10497000CDE900653B4602AA51467820FFF794FB3B
:104980004FF05F0A6FA2142102A8D4F8B03003F0F0
:10499000F9F8CDE900653B4602AA51467820FFF7B9
:1049A00083FBCDE90065434668A273210520FFF72C
:1049B0007BFB206867A21421B0F85E3002A803F0E8
:1049C000E1F8CDE900654F464B4602AA732141202C
:1049D000FFF76AFB20685FA21421B0F8603002A8DC
:1049E00003F0D0F8CDE900653B4602AA73217D2093
:1049F000FFF75AFB206857A21421B0F8623002A8D2
:104A000003F0C0F873213B4602AAB9204BE0FFE750
:104A1000CDE900654746434650A273210520FFF7C4
:104A200043FB20684BA20A21B0F85C3002A803F0D7
:104A3000A9F8CDE900654B4602AA73214120FFF792
:104A400033FBCDE900653B4646A228217820FFF7DD
:104A50002BFBDAF8040045A20A2190F950300BA88C
:104A600003F090F8CDE900655B460BAA2821B4203D
:104A7000FFF71AFB206890F85800012817D1CDE9FC
:104A800000653B463BA241217820FFF70DFB2068E3
:104A90003BA20A21B0F85A300EA803F073F8412166
:104AA0005B460EAABE20CDE90065FFF7FDFA0020A7
:104AB00000E700004D523136205374617475730065
:104AC000702C0020525800004D6F64653A000000C1
:104AD0004E4F4E4500000000526164696F3A00007D
:104AE000545800005641524941424C4500000000D4
:104AF0004649584544000000424C45004746534B48
:104B0000000000004C4F524100000000464C524350
:104B100000000000467265713A00000040420F003C
:104B2000256C6C754D487A007278636F756E743AB7
:104B3000000000006368313A256C75006368323A02
:104B4000256C75006368333A256C7500727869646A
:104B50003A00000030782530345800005458494459
:104B60003A000000506F7765723A00002564644295
:104B70006D000000446174614C656E3A00000000F5
:104B800025644200FEB50020FFF7A5F800241020A0
:104B9000CDE9000440F2FF7319A277216E20FFF7E0
:104BA00083FA01264DF6A70520208DE8610000223A
:104BB000302311461648FFF7B7F86420FDF7CCF80C
:104BC0001C208DE861000346042230211148FFF7C4
:104BD000ABF86420FDF7C0F81826CDE900642B4639
:104BE0000DA230210020FFF75FFACDE900642B46CB
:104BF0000DA248210020FFF757FA0020FEBD00005B
:104C0000496E697469616C697A696E672E2E2E002F
:104C100068DB000828DC00084D5231362D2D57691D
:104C200072656C65737300007472616E736D697385
:104C300073696F6E20746F6F6C0000002DE9F04196
:104C400088B0050004D020480078032805D039E05A
:104C50004FF0FF3008B0BDE8F081372755F8A83F86
:104C60001AA2142103A802F08DFF00241026CDE91A
:104C700000464FF4FC68434603AA39467820029464
:104C8000FFF747FA4B2713A2142103A86B6802F021
:104C900079FFCDE90046434603AA394678200294BD
:104CA000FFF737FA5F270DA2142103A8AB6802F0C3
:104CB00069FFCDE90046434603AA394678200294AD
:104CC000FFF727FA0020C5E7702C00206368313A0F
:104CD000256C75006368323A256C75006368333A59
:104CE000256C750000B5FCF77DFE012801D8062073
:104CF00000BD032801D8072000BD052801D80820E1
:104D000000BD072801D8092000BD092801D80A20C4
:104D100000BD0F2801D8172000BD282000BD0000CD
:104D20001D4808B5416941F0010141614069002217
:104D300000F00100009005210C20FDF70BFA0C207B
:104D4000FDF7FAF9002205210D20FDF703FA0D20E9
:104D5000FDF7F2F9002205210E20FDF7FBF90E20E8
:104D6000FDF7EAF9002205210F20FDF7F3F90F20E6
:104D7000FDF7E2F9002205211020FDF7EBF91020E4
:104D8000FDF7DAF9002205211120FDF7E3F9BDE86E
:104D900008401120FDF7D0B90010024010B5074AB5
:104DA0000021074804F010F90649074A0860BDE8E9
:104DB00010400021054804F007B9000050C3000866
:104DC000096F000800000020F4F20008BD7200081E
:104DD0002DE9F04186B000263E48009601960296E5
:104DE0000396816941F020018161816901F0200110
:104DF0000491816941F004018161816901F004013C
:104E00000491816941F0080181618069324F00F0AD
:104E100008004FF488740490002221463846FDF7BC
:104E200022F9DFF8B880002245F219214046FDF74B
:104E30001AF901258DE8700002246946384603946A
:104E4000FDF71CF8CDE902540095694640460195EE
:104E5000FDF714F84FF4A44003948DE8610069460F
:104E60004046FDF70BF8E00200901D48CDE9010631
:104E700069463846FDF702F818200090CDE9015444
:104E8000694640460394FCF7F9FFE020009015487E
:104E9000CDE9010469464046FCF7F0FFE001CDE9A9
:104EA0000006694602944046FCF7E8FF002205210F
:104EB0001720FDF74FF91720FDF73EF900220521D5
:104EC0002820FDF747F92820FDF736F906B0BDE8A0
:104ED000F08100000010024000080140000C014079
:104EE0000000211000001110104810B50E4901609B
:104EF0004FF48271416000218160C1604FF4007203
:104F00000161C0E905121022C0E9072141628162F6
:104F10000A21C162FDF750FC002803D0BDE8104013
:104F2000FCF732BC10BD0000003001403001002011
:104F3000104810B50E4901604FF4827141600021A4
:104F40008160C1604FF400720161C0E9051208225E
:104F5000C0E90721416281620A21C162FDF72CFC90
:104F6000002803D0BDE81040FCF70EBC10BD0000C7
:104F7000003800408801002010B596B000240F943E
:104F800010941194129413941C2108A81494FBF704
:104F900071F920216846FBF76DF927482549C0E9DA
:104FA00000145921C0E90241046144618461FEF7A3
:104FB000B3F808B1FCF7E8FB4FF480500F900FA94D
:104FC0001D48FEF709F908B1FCF7DEFB1A48FEF7A9
:104FD000FFF908B1FCF7D8FB139413A916481494F1
:104FE000FEF766F808B1FCF7CFFB6020CDE90804B6
:104FF0000A940C940D940C2208A90F480E94FEF705
:1050000081F908B1FCF7C0FB00944FF40050CDE9E2
:105010000440029401940394694607480794FEF7FC
:105020001DF808B1FCF7B0FB0348FEF745F916B0D0
:1050300010BD0000002C0140AC0200200C4810B54F
:105040000A4901600B494160002181600C22C16066
:10505000C0E904128161C161FEF770FC002803D031
:10506000BDE81040FCF790BB10BD000000380140C7
:1050700038050020A086010010B5104C0E480C2108
:1050800020604FF4E13060600020A060E060C4E97F
:105090000401A061E0612046FEF750FC08B1FCF776
:1050A00073FBFF2206490548FEF712FD2068C16820
:1050B00041F01001C16010BD004400408005002097
:1050C00038030020FEE7FEE7034910B50220087010
:1050D00001F050F910BD0000B8000020034910B5E0
:1050E0000420087001F046F910BD0000B80000204F
:1050F000034910B50320087001F03CF910BD000011
:10510000B800002010B504A002F02CFD06490520CF
:10511000087001F02FF910BD5B54585D2054585FA2
:10512000444F4E450D0A0000B800002010B504A001
:1051300002F018FD07490620087001F01BF910BDA8
:105140005B54585D2054585F54494D454F55542188
:105150000D0A0000B80000200148FDF7BDBA0000AC
:10516000300100200148FDF7B7BA00008801002097
:1051700010B5406A0021C187C186FDF78DFA10BDC8
:1051800010B5406A01684A6822F003024A60416D26
:1051900041F010014165012180F85110FDF77CFAC2
:1051A00010BD10B5406AFDF729FC10BD10B5406A6E
:1051B000FDF7ECFE10BD10B5406AFDF71FFF10BDF6
:1051C00070B50546446AFCF753FF0246286800683C
:1051D000800626D42068416821F020014160A06843
:1051E00018B96068B0F5827F16D02068416821F058
:1051F000010141606421204600F076F808B12020CA
:1052000060650020E087012084F85100606D40B1A6
:105210002046FDF741FA70BD2068416821F0030186
:10522000E7E72046FDF7CEFB70BD38B50546446A7A
:10523000FCF71EFF024628680068800623D4206819
:10524000416821F0200141602068416821F002019D
:1052500041606421204600F075F818B1606D40F09F
:1052600020006065A068002118B92068C2688068C5
:105270000090E186012084F85100606D18B120464D
:10528000FDF70AFA38BD2046FDF76EFE38BD70B551
:105290000546446AFCF7ECFE024628680068800672
:1052A0001ED42068416821F020014160642120461D
:1052B00000F048F818B1606D40F02000606520688B
:1052C000416821F0030141600020E086E087012071
:1052D00084F85100606D18B12046FDF7DDF970BD0E
:1052E0002046FDF76FFE70BDF8B5044640684FF4E8
:1052F0008273984217D1A0684FF48065B0F5004FD3
:1053000001D0A8420FD12068066826F0400606604A
:105310006068984207D1A068A84204D100920B4669
:105320000022012103E000920B460022802120464A
:1053300000F034F8002804D0606D40F02000606573
:105340000320F8BDF8B515460E460B4600920446FC
:105350000122022100F022F840B9334600228021C8
:105360002046009500F01AF8002804D0606D40F047
:10537000200060650320F8BD00680649884201D11D
:10538000002070470449884201D101207047032062
:105390007047000000300140003800402DE9F8431C
:1053A0001E46914688460446089DFCF761FE401B58
:1053B000351AFCF75DFE074625480068C0F3CB3080
:1053C000684338E0701C37D0FCF752FEC01BA8427F
:1053D00003D215B1009860B32CE02068416821F039
:1053E000E00141606068B0F5827F0BD1A068B0F544
:1053F000004F02D0B0F5806F04D12068016821F021
:1054000040010160A06AB0F5005F09D12068016821
:1054100021F4005101602068016841F400510160ED
:10542000012084F85100002084F850000320BDE8DA
:10543000F8830025401E00902068816838EA01004A
:1054400004D000214945BDD10020F0E70121F9E752
:105450001400002010B5002306E000BF30F8024B16
:1054600021F813405B1C9BB29342F7D310BD0000A0
:105470002DE9F05FA0F1006415468A468346B4F535
:10548000803F5FD2FCF7C4FCA70AC4F34806C6F508
:105490000074A54200D82C46DFF8AC904FF00060B5
:1054A00000EB872080464FF400722749FFF7D2FFB8
:1054B00000204FF6FF7106E0331839F813208A42B6
:1054C00003D1401C80B2A042F6D3A0422ED2404667
:1054D000FCF7C2F94CF25030FCF794F91B48016913
:1054E00021F0020101610020494606E03AF810204F
:1054F0008319401C21F8132080B2A042F6D3124930
:1055000040464FF4007200BF00F022F8A54215D0CB
:10551000281B0AEB440A0BEB440B002685B24FF420
:1055200000747F1CA542B9D82C46B7E74CF2503026
:10553000FCF768F9224651465846E5E7BDE8F05FBA
:10554000FCF71CBCBDE8F09F30200020002002408A
:105550002DE9F04116460F46054600240AE000BF3B
:1055600037F81420002329460120FCF711FC641CA5
:10557000A4B2AD1CB442F3D3BDE8F081C0F3401136
:105580004901C0F3001241EA0211C0F3C00241EA2E
:10559000C201C0F3800241EA8201C0F3400241EA45
:1055A000420108B500F0010001438DF8001001220E
:1055B0006946892000F016FB08BD08B5010A8DF880
:1055C00000108DF8010002226946972000F00AFBC6
:1055D00008BD10B54FF4AA7000F078FA044640F206
:1055E000531000F073FA44EA002010BD70B5204A51
:1055F000002001465278032A39DA002A37D0012ADE
:1056000035D140F6541000F061FA044640F65510CA
:1056100000F05CFA054640F6561000F057FA2104F7
:1056200041EA05210143C1F3130400F035F8FBF70B
:105630001BF902460B4600200E49FBF798F80022A2
:105640000D4BFBF722F805460E462046B4F5002F19
:1056500001D3A4F58010FBF707F9084A084BFBF7C4
:1056600014F82A463346BDE87040FBF780B870BD99
:10567000E00000200000994000408F40CDCCCCCC11
:10568000CCCCF83F08B502226946152000F0E8F9B5
:10569000BDF8000040BA08BD0949002089780A29F0
:1056A0000BD0182907D0262903D0342900D105486A
:1056B0007047054870470548704705487047000027
:1056C000E000002075190300EA320600D4650C00E2
:1056D000A8CB18000148007870470000E0000020C7
:1056E0001CB50446052269461D2000F0B9F9804822
:1056F00040782070032865D00FDCC0B1012815D197
:105700009DF80000404200EBD070401060709DF8A2
:105710000100802819D280081DE004287DD00F28C0
:1057200004D100202060A0800F2020701CBD9DF8B7
:105730000000404200EBD070401060709DF8010006
:10574000404200EBD070401005E0A0F58070C1171A
:1057500000EB91708010A0709DF802008109E07844
:1057600061F30000E0709DF80210490961F3410007
:10577000E0709DF80210090961F38200E0709DF865
:105780000210C90861F3C300E0709DF80210890897
:1057900061F30410E0709DF80210490861F34510B0
:1057A000E0709DF8021061F38610E0709DF8030030
:1057B0004109207961F3000020719DF8031061F325
:1057C00041008DE09DF80000404200EBD070401099
:1057D00060709DF80100404200EBD0704010A07056
:1057E0009DF802008109E07861F30000E0709DF807
:1057F0000210490961F34100E0709DF802100909A7
:1058000061F38200E0709DF80210C90861F3C300E3
:10581000E0709DF80210890800E025E061F30410B3
:10582000E0709DF80210490861F34510E0709DF8A2
:10583000021061F38610E0709DF803008109207961
:1058400061F3010020719DF80310490961F38200A2
:1058500020719DF80310090961F3C30020719DF8C0
:10586000031061F304103BE09DF80000404200EBA0
:10587000D070401060709DF80100404200EBD07085
:105880004010A0709DF802008109E07861F30000EB
:10589000E0709DF80210490961F34100E0709DF845
:1058A0000210090961F38200E0709DF80210C90836
:1058B00061F3C300E0709DF80210890861F30410E1
:1058C000E0709DF80210490861F34510E0709DF802
:1058D000021061F38610E0709DF8030000F00100F3
:1058E00020719DF8040000F0070060711CBD0000ED
:1058F000E00000200148407870470000E0000020F0
:10590000F8B50C46064615466946204600F01EF8D6
:105910002278AA4201D90120F8BD31469DF8000045
:1059200000F068F80020F8BD08B500208DF80000F0
:10593000012269461F2000F093F89DF800004042C4
:1059400000EBD07040F3470008BD0000F8B50D46ED
:10595000044602226946172000F082F80C4E707847
:1059600001280AD140F6031000F0B0F8C00904D0B5
:1059700040F6011000F0AAF805E0707804289DF8C0
:10598000000000D1801C20709DF801002870F8BD37
:10599000E000002008B500208DF8000001226946D3
:1059A000C02000F05DF89DF8000008BD70B5074DFF
:1059B0004FF480712846FCF72EF8044680212846D3
:1059C000FCF729F844EA4000C0B270BD000C014069
:1059D00010B5044600F0BAF82046BDE8104000F0CB
:1059E00001B800000022036880210148FCF716B8C6
:1059F000000C01402DE9F0410E46014615481446C1
:105A0000D51C1B2202704170002181700B4603E0FF
:105A1000C2185B1CD1709BB2A342F9D300F0B0F85E
:105A20000D4F002210213846FCF714F82A460B4986
:105A3000084801F045FA09492246C91C3046FAF7E0
:105A400000FC012210213846FCF704F8BDE8F041C3
:105A500000F096B870240020000801407028002053
:105A60002DE9F0410E460146901C85B214481446BB
:105A70000170002141700B4603E0C2185B1C91705D
:105A80009BB2A342F9D300F07BF80E4F0022102105
:105A90003846FBF7DFFF2A460B49094801F010FAA8
:105AA00009492246891C3046FAF7CBFB0122102116
:105AB0003846FBF7CFFFBDE8F04100F061B80000C9
:105AC00070240020000801407028002008B5012241
:105AD000694600F003F89DF8000008BD2DE9F0418B
:105AE0000E46111D164B8DB219211970010A5970FD
:105AF000987000211446D970084603E01A18401C1B
:105B0000117180B2A042F9D300F03AF80D4F002293
:105B100010213846FBF79EFF2A460B49084801F042
:105B2000CFF909492246091D3046FAF78AFB0122BE
:105B300010213846FBF78EFFBDE8F04100F020B899
:105B400070240020000801407028002010B51420A7
:105B5000FCF702F9094C002201212046FBF77AFFED
:105B60003220FCF7F9F8012211462046FBF772FFBC
:105B7000BDE810401420FCF7EFB80000000C014015
:105B800070B5054D4FF4807421462846FCF766FA3F
:105B90000128F9D070BD0000000C014070B50F481D
:105BA0001A23941C00F8013B002300F8013BFAF78C
:105BB00048FBFFF7E5FF0A4D002210212846FBF7BE
:105BC00049FF2146054801F06BF9012210212846C2
:105BD000FBF740FFBDE87040FFF7D2BF7024002004
:105BE000000801402DE9F0410546501C1446884646
:105BF00086B2FFF7C5FF0F4F002210213846FBF792
:105C000029FF0D482246414600F8015BFAF719FBCF
:105C10003146094801F044F9012210213846FBF7CA
:105C200019FF842D03D0BDE8F041FFF7A9BFBDE8FF
:105C3000F0810000000801407024002013B501220B
:105C400001A900F001F81CBD70B50346D01C84B258
:105C50000F48182500F8015B1D0A00F8015B00F8E9
:105C6000013BFAF7EEFAFFF78BFF0A4D00221021F5
:105C70002846FBF7EFFE2146054801F011F9012205
:105C800010212846FBF7E6FEBDE87040FFF778BF1D
:105C900070240020000801400249C86001F108009A
:105CA000FFF796BEE00000200348C17811B1012142
:105CB0000171704700F002B8E000002070B5514C4F
:105CC0002078002872D0E07830B1207900286DD09B
:105CD00072B60020207162B66678FFF7D3FC0546E5
:105CE0004FF6FF70FFF769FC2EB1012E40D0032E56
:105CF00001D0042E5AD1207804286FD0052855D120
:105D0000A80714D5680605D5E06880B1816971B12E
:105D1000022006E02807E06805D540B1816931B16D
:105D20000120884703E010B1406800B18047680750
:105D300004D5E06810B1806800B18047280705D518
:105D4000E06818B1816909B1012044E0680458D5C0
:105D5000E068002855D0406905E0680451D5E06846
:105D600000284ED0006900284BD0BDE870400047A5
:105D70002078042832D005280DD0062841D1E80427
:105D8000E4D5A804E06833D500283AD0C1690029D9
:105D900037D0012032E0A8070DD56806E06806D5A7
:105DA00048B1816939B10220884704E029E010B187
:105DB000406800B18047E80604D5E06810B1C068CB
:105DC00000B18047A806C1D5E0680028BED081692F
:105DD0000029BBD000208847B8E7FFE7E807BCD020
:105DE000E0680028B9D000680028B6D08047B4E742
:105DF000002806D0C169002903D00020BDE870400A
:105E0000084770BDE000002010B5144600F080F98E
:105E10002046BDE8104000F067BA01B5012269468E
:105E20009E20FFF7DFFE08BD08B52138010A8DF876
:105E300000108DF80100022269469820FFF7D2FE7B
:105E400008BD10B50446010E40F6CF10FFF7F6FE70
:105E5000C4F307414FF41D60FFF7F0FEC4F30721C0
:105E600040F6D110FFF7EAFEE1B2BDE8104040F67F
:105E7000D210FFF7E3BE00000148FFF7E2BF0000C9
:105E8000D6BE898E08B502228DF800008DF801106B
:105E900069468F20FFF7A6FE08BD000010B500225E
:105EA0001146C520FFF79EFE01490620087010BD6F
:105EB000E000002001B5012269468820FFF792FE2C
:105EC00001490620087008BDE000002008B5010A5D
:105ED0008DF800108DF801000548407808B10328BE
:105EE00005D10222694640F6C610FFF7ADFE08BD97
:105EF000E000002008B5010A8DF800108DF80100BF
:105F00000548407808B1032805D10222694640F6C9
:105F1000C810FFF799FE08BDE00000201CB5040A78
:105F20008DF800408DF80100080A8DF80200100A73
:105F30008DF804008DF80520180A8DF806008DF8FC
:105F400003108DF80730082269468D20FFF74AFEBE
:105F50001CBD000010B500221146C120FFF742FE13
:105F600001490320087010BDE00000200149002015
:105F7000C8707047E000002001B5012269469B20EF
:105F8000FFF730FE08BD000038B5234D0446007809
:105F90006978884201D000F0ADF8207803281DD040
:105FA00003DC38B1012822D10CE0042825D00F28C9
:105FB0001DD12AE060788DF80000A0788DF80100EE
:105FC000E07812E020798DF8000060798DF801000A
:105FD000A0798DF802006079A87008E0E0798DF86A
:105FE0000000207A8DF80100607A8DF8020003220B
:105FF00069468B20FFF7F6FD38BDA07A8DF80000CA
:10600000E07A8DF80100207BEFE700208DF800009A
:106010008DF80100E9E70000E00000201CB53449DC
:10602000044600784978884201D000F063F821786E
:106030000020032935D003DC39B101292BD118E028
:10604000042942D00F2926D14CE060788DF8000059
:10605000A0788DF80100E0788DF8020020798DF8A5
:10606000030060798DF80400A0798DF80500E079CF
:106070000FE0217A8DF80010617A8DF80110A17A75
:106080008DF80210E17A8DF80310217B8DF8041051
:106090002BE08DF80600072269468C20FFF7A2FD51
:1060A0001CBD607B8DF80000A07B8DF80100E07BBB
:1060B0008DF80200207C8DF80300607C8DF80400D0
:1060C000A07C8DF80500E07CE3E7217D8DF80010D1
:1060D000617D8DF80110A17D8DF80210E17D8DF8B4
:1060E000031000E000908DF804008DF80500D0E763
:1060F000E000002001B505499DF80000012248702C
:1061000069468A20FFF76EFD08BD0000E000002010
:106110000A4601460020FFF741BD00000149012069
:10612000C8707047E000002070B5074D002400BF24
:1061300005EB8400817835F82400FFF77FFD641CAF
:1061400024B2002CF4D070BDEADC000801B50122B5
:1061500069469620FFF746FD08BD000008B5FAF72E
:1061600094FB0022094BFAF702FBFAF79BFB010CA8
:106170008DF80010010A8DF801108DF8020003223D
:1061800069468620FFF72EFD08BD0000A8CB6840B9
:1061900008B58DF80000000C010A8DF801108DF88B
:1061A00002004FF6FF70FFF708FA032269468220CB
:1061B000FFF718FD01490520087008BDE000002028
:1061C0001CB58DF80000080A8DF801008DF802104A
:1061D000100A8DF803008DF80420052269469420EA
:1061E000FFF700FD0149052008701CBDE0000020FC
:1061F00000221146D520FFF7F5BC0000C107090FAA
:10620000C0F3400241EA8201C0F3800208B541EACE
:106210004201C0F3C00001438DF800100449002082
:106220000122087069468420FFF7DCFC08BD0000ED
:10623000E000002001B5012269468020FFF7D2FC72
:106240009DF80010034811B10221017008BD012121
:10625000FBE70000E00000200346194810B5427833
:1062600032B140F6CF10032A13D0042A22D11EE007
:106270000522012B04D0022B05D0032B1AD105E0F7
:1062800040F6CE1018E040F6D31015E040F6D810D6
:1062900012E00422012B0FD0022B02D0032B09D1D4
:1062A00002E040F6D41007E040F6D91004E00422E2
:1062B000012B01D0012010BDFFF7C6FC002010BD4E
:1062C000E000002070B5044640F6CD152846FFF7E3
:1062D000FDFB00F0F00104F00F0001432846BDE88B
:1062E0007040FFF7ABBC000008B58DF80000000C53
:1062F000010A8DF801108DF802004FF6FF70FFF7CC
:106300005CF9032269468320FFF76CFC01490420F5
:10631000087008BDE000002000221146D220FFF7DF
:1063200061BC00221146D120FFF75CBC08B51230D9
:106330008DF800008DF80110022269468E20FFF7CB
:1063400051FC08BD0649497819B1032901D0042937
:1063500004D1014640F6C510FFF770BC704700003D
:10636000E000002010B5FBF755FBBDE8104000F041
:10637000B9BD0000F8B54C4C494E4A4F801E04F19F
:10638000280506283DD2DFE800F003414C576F8610
:1063900046A001F0E7FB4E4F00257F223D70336E93
:1063A00039464C48984739784A487F2901D24554A4
:1063B00001E080F87E500088002546BAD4F800201D
:1063C0004FF6FF7C5E23204603EB4501515AC9B1CD
:1063D000614517D0B14215D100EB850454F8A81FD0
:1063E000491C216081684162022001F061FB01F0DB
:1063F000BBFA206800903B783246691C36A001F059
:10640000B1FB4BE06D1C032DDEDB47E040A001F04B
:10641000A9FB032001F04CFB2E48903800F006FD4C
:106420003CE045A001F09EFB032001F041FB4D48FC
:10643000F16D0068884731E04BA001F093FB01202B
:1064400001F036FB01F090FA206890F8581049B13D
:10645000B0F85A00001D84B221464EA001F082FB24
:10646000E2B210E03C78F7E750A001F07BFB03209C
:1064700001F01EFB206890F8581051B1B0F85A0096
:10648000001D80B2C2B213482946903800F0E8FCE3
:1064900004E03878F6E751A001F064FB0020F8BD75
:1064A000F0DC000805000020602F00200D0A5B5280
:1064B000585D203C3C3C205061636B657420526504
:1064C000636569766564203E3E3E0D0A000000006B
:1064D00008010020002D00205B636825645D2048D2
:1064E00065616465723A20307825303458207C200C
:1064F00053697A653A202564206279746573207C3B
:1065000020436F756E743A2025640D0A0000000068
:106510000D0A5B52585D202E2E2E2054696D656F3A
:106520007574202852657374617274696E672052A5
:1065300058290D0A000000000D0A5B52585D202109
:106540002121204552524F52202D20526563657003
:1065500074696F6E204661696C6564202121210D8C
:106560000A000000E4DF00080D0A5B54585D203C7F
:106570003C3C205061636B65742053656E742053FE
:1065800075636365737366756C6C79203E3E3E0D72
:106590000A0000005B54585D204C656E6774683AD1
:1065A0002025642062797465730D0A000D0A5B541E
:1065B000585D202121212054494D454F5554202D0F
:1065C000205472616E736D697373696F6E204661DA
:1065D000696C6564202121210D0A00000D0A5B43CE
:1065E00041445D204368616E6E656C20416374694F
:1065F000766974792044657465637465640D0A0076
:1066000020B1044909780172002070474FF0FF3033
:1066100070470000B80000202DE9FC411646040038
:106620004FF0FF372BD061604E70FFF79BFE4FF4A9
:10663000FA70FBF791FB794D79482968884779A072
:1066400001F090FA78A001F08DFA87A001F08AFAA3
:1066500075A001F087FA8FA195A001F083FA286B4D
:10666000804701469AA001F07DFA6FA001F07AFA06
:1066700046B1012E0BD0022E36D0032E39D038462B
:10668000BDE8FC819BA001F06DFA042003E0A5A009
:1066900001F068FA0120616881F835006168487787
:1066A000A96B002088476068E96B90F8350088473F
:1066B0006068296C353088476068696C1D30884790
:1066C0006068A96C806C88470021EA6C0846904796
:1066D00060682A6D90F8511090F9500090476168F9
:1066E000487802280AD017E098A001F03BFA002071
:1066F000D1E7A0A001F036FA0320CCE70120AA6D73
:10670000891C904761680220AA6DC91D9047616885
:106710000320AA6D0C3190476168487803280DD199
:106720000120AA6D1131904761680220AA6D1531D0
:10673000904761680320AA6D19319047E86E804741
:1067400038A001F00FFA9AA001F00CFAA8A001F00D
:1067500009FA97A001F006FA6068D0E912562846B7
:106760003146FAF773F8AD49F9F751FFFAF7B3F884
:10677000CDE900012A463346A9A001F0F3F960688B
:1067800090F95010B1A001F0EDF97F21B7A001F010
:10679000E9F961684878012802D003281BD031E06C
:1067A00091F83910B9A001F0DDF9606890F83A105D
:1067B000BDA001F0D7F9606890F83B10C1A001F0CE
:1067C000D1F9606890F82510C5A001F0CBF9606898
:1067D00090F8271013E091F83C10C8A001F0C2F91E
:1067E000606890F83D10CCA001F0BCF9606890F8AA
:1067F0002A10BBA001F0B6F9606890F82E10CDA069
:1068000001F0B0F9D2A001F0ADF969A001F0AAF948
:10681000D7A001F0A7F9002032E70000F0DC000863
:10682000C00000200D0A00003D3D3D3D3D3D3D3D89
:106830003D3D3D3D3D3D3D3D3D3D3D3D3D3D3D3D88
:106840003D3D3D3D3D3D3D3D3D3D3D3D3D3D3D3D78
:106850003D3D3D3D3D3D3D3D3D3D3D3D3D3D3D3D68
:106860003D3D3D3D0D0A000020202020202020201D
:1068700020202020202053583132383120526164AA
:10688000696F20496E697469616C697A6174696FB6
:106890006E0D0A004669726D7761726520566572E9
:1068A00073696F6E3A203137303931394100000059
:1068B00020204170706C69636174696F6E20566549
:1068C0007273696F6E203A2025730D0A0000000074
:1068D00020204669726D7761726520566572736912
:1068E0006F6E202020203A203078253034580D0A51
:1068F000000000000D0A5B2A5D20526164696F2070
:106900004D6F64653A20424C452028426C75657491
:106910006F6F7468204C6F7720456E6572677929B8
:106920000D0A00000D0A5B2A5D20526164696F2028
:106930004D6F64653A204C4F524120284C6F6E6772
:106940002052616E6765290D0A0000000D0A5B2A5E
:106950005D20526164696F204D6F64653A2047463F
:10696000534B2028476175737369616E2046534B02
:10697000290D0A000D0A5B2A5D20526164696F20AF
:106980004D6F64653A20464C52432028466173742B
:10699000204C6F6E672052616E676520436F6D6D8E
:1069A000756E69636174696F6E290D0A00000000DD
:1069B0002D2D2D2D2D2D2D2D2D2D2D2D2D2D2D2D07
:1069C0002D2D2D2D2D2D2D2D2D2D2D2D2D2D2D2DF7
:1069D0002D2D2D2D2D2D2D2D2D2D2D2D2D2D2D2DE7
:1069E0002D2D2D2D2D2D2D2D2D2D2D2D0D0A000074
:1069F0002020202020202020202020202020202097
:106A00002020436F6E66696775726174696F6E20CE
:106A100053756D6D6172790D0A0000000024744990
:106A200020205246204672657175656E637920207C
:106A300020203A20256C6C7520487A2028252E319C
:106A400066204D487A290D0A000000002020545885
:106A500020506F77657220202020202020203A20AF
:106A600025642064426D0D0A00000000202042755C
:106A7000666665722053697A6520202020203A20BE
:106A800025642062797465730D0A000020204C6F24
:106A900052612053462020202020202020203A2010
:106AA00025640D0A0000000020204C6F5261204236
:106AB000572020202020202020203A2025640D0A65
:106AC0000000000020204C6F526120435220202003
:106AD0002020202020203A2025640D0A00000000FC
:106AE0002020507265616D626C65204C656E2020BF
:106AF00020203A2025640D0A000000002020464C8A
:106B0000524320426974526174652F4257203A20E3
:106B100025640D0A000000002020464C524320430B
:106B2000522020202020202020203A2025640D0AF9
:106B30000000000020205061796C6F6164204C657A
:106B40006E20202020203A2025640D0A000000003D
:106B500020204D6F64652020202020202020202030
:106B600020203A20494E544552525550540D0A00A7
:106B70000D0A5B2A5D2053583132383120496E6945
:106B80007469616C697A6174696F6E20436F6D70AE
:106B90006C657465210D0A0D0A00000010B50446ED
:106BA000FFF78CF82046FFF72BFD002010BD0000FA
:106BB00070B50E4604002ED06068184D80F8526003
:106BC000A96B00208847032E1AD2616891F8520001
:106BD00000EB40021248825C81F83F20616891F826
:106BE000522002EB42020244527881F84020616850
:106BF00091F8522002EB42021044807881F8410063
:106C00006068E96B90F8350088476068296C35301A
:106C10008847002070BD4FF0FF3070BDF0DC0008E9
:106C2000A8DC000870B50E4604002ED06068184D30
:106C300080F85560A96B00208847042E1AD261683D
:106C400091F8550000EB40021248825C81F83C202C
:106C5000616891F8552002EB42020244527881F8B3
:106C60003D20616891F8552002EB42021044807883
:106C700081F83E006068E96B90F8350088476068ED
:106C8000296C35308847002070BD4FF0FF3070BD53
:106C9000F0DC0008DBDC000870B50E4604002ED0E6
:106CA0006068184D80F85460A96B00208847042E56
:106CB0001AD2616891F8540000EB40021248825CDD
:106CC00081F83620616891F8542002EB42020244B8
:106CD000527881F83720616891F8542002EB420223
:106CE0001044807881F838006068E96B90F83500CE
:106CF00088476068296C35308847002070BD4FF0A8
:106D0000FF3070BDF0DC0008CCDC000870B504007A
:106D10002CD06068174D80F85310A96B002088476D
:106D2000616891F8530000EB40021348825C81F8DF
:106D30003920616891F8532002EB420202445278F4
:106D400081F83A20616891F8532002EB4202104426
:106D5000807881F83B006068E96B90F835008847DF
:106D60006068296C35308847002070BD4FF0FF30D7
:106D700070BD0000F0DC0008B4DC00082DE9F04133
:106D80000E4604004FF0FF3713D0194D0020A96BB9
:106D900088476068E96B90F83500884760684670FE
:106DA00060684EB10121012E07D0022E08D0032EBB
:106DB00019D03846BDE8F081042180F8351001E093
:106DC000002211E0606841776068E96B90F8350057
:106DD00088476068296C353088476068696C1D3069
:106DE00088470020E6E7032280F83520EAE7000024
:106DF000F0DC000870B50D46040012D00A4E0020E9
:106E0000B16B88476068F16B90F83500884761681E
:106E10000020C1E912506068B16C806C8847002086
:106E200070BD4FF0FF3070BDF0DC000870B503217D
:106E3000017040680221074C017007480023656D0E
:106E400041881A460846A8470448E16D40688847CB
:106E5000002070BDF0DC0008B800002098DC0008BD
:106E60002DE9F0410E46012101704068094C15469C
:106E7000017009480023676D81881A460846B847A3
:106E80000648636E29468268304698470020BDE870
:106E9000F0810000F0DC0008B800002098DC000859
:106EA000064B10B501221A7013460A46014600200F
:106EB000FAF78AF9BDE8104004F03EBDF00000206A
:106EC00038B5074C01232370009313460A46014648
:106ED0000020FAF78EF9BDE8384004F02DBD00001F
:106EE000F000002010B5064A02210020FAF75EF9F2
:106EF0000021BDE81040034A0846FAF757B90000E0
:106F000069B400085DB4000810B502F05AF8BDE895
:106F1000104002F09EB810B5FBF7B0F805F05AF833
:106F2000012803D0BDE8104004F062BD10BD10B5CB
:106F300090B028216846F9F79DF914210AA8F9F7BD
:106F400099F901210804CDE90010420002920224BF
:106F50000491CDE907404FF4E01009906846FBF733
:106F60000BFA08B172B6FEE70F20CDE90A04002043
:106F70004FF48061CDE90C010E9002210AA8FBF7C5
:106F80001BF9002801D072B6FEE710B010BD7047A3
:106F9000F0B50268194B1A4C1A4D4FF080479842D1
:106FA00005D0B84203D0A04201D0A84203D122F0BC
:106FB00070064A683243984205D0B84203D0A042D6
:106FC00001D0A84203D122F44074CA6822434C691C
:106FD00022F08002224302608A68C2620A688262EA
:106FE000984201D109690163012141610169C90721
:106FF00003D0016921F001010161F0BD002C0140C5
:10700000000400400008004010B501F01F030121FA
:10701000046A99408C430462016A9A4011430162F8
:1070200010BD10B5446A0121626A824205D1217700
:107030008069F8B984F83E101CE0A26A824206D149
:10704000022222778069A8B984F83F1012E0E26A30
:10705000824206D104222277806958B984F8401010
:1070600008E0226B824205D108222277806908B9A4
:1070700084F841102046FCF7D9F90020207710BD94
:1070800010B5446A616A814201D101200DE0A16A14
:10709000814201D1022008E0E16A814201D104204D
:1070A00003E0216B814201D1082020772046FCF7C4
:1070B000BEF90020207710BD10B5446A0121626A34
:1070C000824203D1217784F83E1019E0A26A8242FD
:1070D00004D10220207784F83F1011E0E26A824256
:1070E00004D10420207784F8401009E0226B82420A
:1070F00004D10820207784F8411001E084F83D1085
:107100002046FCF7D7F80020207710BD10B5846822
:1071100042EA032224F47F440A432243826010BDE2
:10712000826822F070020A4342F0070181607047D2
:1071300030B5036A026A22F0010202624268846981
:1071400024F073050C682C4323F002058B682B4355
:107150000A4DA8420BD123F00805CB6822F44072F7
:107160002B434D6923F0040315438A692A43426087
:10717000846149684163036230BD0000002C014016
:1071800030B5026A036A23F010030362436884691E
:107190000D6824F4E64444EA05248D6822F02002B8
:1071A00042EA05120B4DA8420ED1CD6822F08002B2
:1071B00042EA05124D6923F4406343EA85038D6971
:1071C00022F0400243EA8503436084614968816399
:1071D000026230BD002C014030B5036A026A22F41D
:1071E000807202624268C46923F4007324F073055C
:1071F0000C682C438D6843EA05230C4DA8420ED140
:10720000CD6823F4006343EA05234D6922F440521C
:1072100042EA05128D6923F4806342EA0512426056
:10722000C4614968C163036230BD0000002C0140A5
:1072300030B5046A026A22F4805202624268C3696D
:107240000D6823F4E64343EA05238D6824F40054D3
:1072500044EA0534064DA84204D14D6922F4804227
:1072600042EA85124260C36149680164046230BD2C
:10727000002C014010B5036A046A24F00104046282
:10728000846924F0F00444EA021423F00A020A4359
:107290008461026210BD10B5036A046A24F0100410
:1072A0000462846923F0A00324F4704444EA0232A7
:1072B00043EA01118261016210BD000010B501F0C6
:1072C00005FE0A4A00210A4801F07EFE094C002210
:1072D0000A212060022001F048FE606001F028FED3
:1072E00001F06FFEBDE8104001F0B3BE18F30008D6
:1072F000F9720008302F002001F0D2FD002001F0CB
:10730000BBFD01F0C6FD24480068C16841F01001D2
:10731000C160F9F7EFFF00F108012048FDF794F88C
:10732000012000F0F1FA192000F04CFB4FF47A70C4
:1073300000F0B8FBF9F7DEFF007A012800D0022048
:1073400000F0B6FB00F010FB01F0A3FD134C054666
:1073500001261248FDF72CF9012001F08DFD01F006
:1073600098FD401B0E2810D3206890F8581079B172
:10737000B0F85A00001D82B20849002328310120CC
:10738000F9F78EFFA0680E35206284F82960E0E7E7
:1073900003480278121DEFE780050020602F0020CF
:1073A0000500002010B5406A0021C185C184FCF7AA
:1073B0007BF910BD70B5446A2068406994F84110AB
:1073C000C0F3C0100025212904D118B1E58420465E
:1073D00000F0B4F82068406994F84210C0F38010BF
:1073E000222904D118B1E585204600F080F8606CB0
:1073F00040F0100060642046FCF756F970BD10B5EF
:107400000146406A096809684FF0000289062ED4D7
:10741000C28501680C3151E8003F23F4807341E8D4
:107420000034002CF5D10168143151E8003F23F0FD
:10743000010341E80034002CF5D10168143151E812
:10744000003F23F0400341E80034002CF5D1202117
:1074500080F84210016B012909D101680C3151E813
:10746000003F23F0100341E80034002CF5D14263C3
:10747000016B012902D0FCF739FB10BD818DFCF7AF
:10748000D9F810BD10B5406A01214163016B012993
:1074900002D0FCF73FFB10BD818D4908FCF7CAF80C
:1074A00010BD10B50146406A09680968890616D4FE
:1074B0000021C1840168143151E8002F22F08002BC
:1074C00041E80023002BF5D101680C3151E8002F71
:1074D00042F0400241E80023002BF5D110BDFCF73B
:1074E000D3FB10BD10B5406AFCF7E2FB10BD01688C
:1074F0000C3151E8002F22F4907241E80023002B58
:10750000F5D10168143151E8002F22F0010241E861
:107510000023002BF5D1016B012909D101680C3141
:1075200051E8002F22F0100241E80023002BF5D192
:10753000202180F8421000210163704701680C315E
:1075400051E8002F22F0C00241E80023002BF5D1C2
:10755000202180F84110704700680649884201D117
:10756000002070470449884201D101207047032060
:1075700070470000004400400038014008B590F812
:107580004210222901D0022008BD82684FF48053A6
:107590009A4201D1016921B1816A9A421BD04AB154
:1075A0000AE00268816A5268C2F308020A80816AAE
:1075B000891C08E0026972B10268526802F07F0219
:1075C0000A70816A491C8162C18D491E0904090C37
:1075D000C18503D01BE002685268F1E70168CA6800
:1075E00022F02002CA600168CA6822F48072CA6070
:1075F00001684A6922F001024A61202180F84210A4
:1076000000214163026B012A03D0FCF76FFA0020CE
:1076100008BD016301680C3151E8002F22F010020F
:1076200041E80023002BF5D101680A68D20602D593
:107630000A6849680091818DFBF7FCFFE7E70000CD
:1076400070B5044600680169E26821F440511143B5
:1076500001612169A0680843616908432168CA681B
:1076600041F20C639A430243CA6020684169A269EF
:1076700021F44071114341611E492068884202D1C2
:10768000FAF740FE01E0FAF72DFE00EBC00101EB36
:107690000012606864218000B2FBF0F3B3FBF1F3E9
:1076A0006FF018067343B2FBF0F5B2FBF0F605EB92
:1076B0008305322303EB0515B5FBF1F5B6FBF1F6B7
:1076C00005F0F00505EB0615B2FBF0F6B2FBF0F0A5
:1076D000B0FBF1F06FF01802504306EB800003EBB3
:1076E0000010B0FBF1F0216800F00F002844886022
:1076F00070BD00000038014038B5816204468285C3
:10770000002013466064222284F84220E56B1B4A65
:10771000AA62E56B1A4AEA62E56B1A4A2A63E26BCF
:1077200050630A462168E06B091DFAF7DDFA20680C
:10773000016840680090206948B120680C3050E82A
:10774000001F41F4807140E80012002AF5D1206842
:10775000143050E8001F41F0010140E80012002AF7
:10776000F5D12068143050E8001F41F0400140E896
:107770000012002AF5D1002038BD0000FF73000878
:1077800085740008B57300082DE9F843984617463C
:107790000D460446089E24E0701C22D0FAF768FCCF
:1077A000A0EB0800B0421AD8CEB12068C1684907E2
:1077B00017D5802D15D0402D13D00168C943090776
:1077C0000FD401680025406800902046FFF78FFE27
:1077D0000820606484F840500120BDE8F88303204D
:1077E000FBE72068006835EA000004D00020B842BA
:1077F000D2D00020F1E70120F9E700000148FBF7B3
:1078000067BF00003805002010B50448FBF760FF93
:10781000BDE81040014800F04DB800008005002090
:1078200070B5050033D01A49286888422FD1284600
:10783000FBF701FF174800684068174CC0F1FF00D4
:10784000C1B2481E6170FE2816D214A000F08AF959
:107850004FF40073627815492846FCF76FF914A0BD
:1078600000F080F9207838B91049627801F1FF0002
:10787000F8F7E7FC01202070FF210C48F8F7FAFC2C
:107880002846BDE87040FF220849FCF721B970BDC9
:1078900000440040C8050020040000205B55415210
:1078A00054322052583A25645D20000038030020ED
:1078B0000D0A000082B000280DD0084A01689142EC
:1078C00009D10A68D243D20605D40A6849680091F2
:1078D00002B0FFF7A5BF02B07047000000440040AF
:1078E000FEE7000070B5074D0024686810B100F095
:1078F00033FE6C606C802C70BDE870400020F9F79E
:107900002DBC00009C00002070B5050002D0B5F52C
:10791000806F01D9012070BD114C207808B1FFF7AC
:10792000E1FF65806D1C05EB4500C500A80000F077
:10793000BBFE0022606008B1002104E06280E9E73C
:1079400040F82120491CA942FAD3012020700548A3
:107950000068416C41F400414164002070BD0000AA
:107960009C000020AC02002010B5FAF781FB014911
:10797000886010BDA8000020114830B401780029AB
:107980001BD04168002918D0428802EB420001EB6D
:10799000401300204FEA000443F82040401CC0B2CE
:1079A0001828F9D3521C02EB42004FF6FF7202EA8C
:1079B000C00230BC0020F9F7BFBB30BC70470000EC
:1079C0009C000020642800D9642001490873704796
:1079D000A800002070B5204C2578002D3BD065888C
:1079E000A84238D26468002C35D000EB400004EB8C
:1079F000401500245FF00100C4F1070600FA06F606
:107A0000164201D0392600E01C2645F82460641C8B
:107A1000E4B2082CF0D30822C2F10F0400FA04F4F7
:107A20000C4201D0392400E01C2445F82240521CAD
:107A3000D2B2102AF0D31021C1F1170200FA02F2DB
:107A40001A4201D0392200E01C2245F82120491CAD
:107A5000C9B21829F0D370BD9C00002010B40C46A8
:107A60000F490B78002B18D04968002915D00C4914
:107A70000C310B7B03FB00F164205C43B4FBF0F49E
:107A8000B1FBF0F15343B3FBF0F0E4B22246C3B2D2
:107A900010BCC9B20020FFF79DBF10BC70470000AA
:107AA0009C00002001498860704700009C00002075
:107AB0000149087070470000A8000020284A10B54E
:107AC000117800294BD05168002948D002F10C01EF
:107AD0004B68C31A322B42D30B78012B01D0022BF7
:107AE00006D18B689268C31A934201D903220A70A7
:107AF0004FF4FA72B0FBF2F202F001030A784C780C
:107B0000A24201D04A7008E0012A03D0022A01D023
:107B1000042A24D18C789C4221D08B704860052A9D
:107B200013D2DFE802F0120303080B006BB100224E
:107B3000FF21104606E00022114602E02BB1002290
:107B4000B421FF20FFF78AFF05E000231A461946FB
:107B50001846FFF73FFFBDE81040FFF70DBF10BD0F
:107B60009C0000200FB4054B10B503A9044A0298ED
:107B700000F008F910BC5DF814FB00004185000816
:107B8000200100200FB47CB50C0009AD01D0611EAE
:107B900000E00021CDE90001064B6A46294608981D
:107BA00000F0F0F8002C02D0009A002111707CBC8B
:107BB0005DF814FB8B8400080907090E002804DB1C
:107BC00000F1E02080F80014704700F00F0000F191
:107BD000E02080F8141D7047004870472C010020F9
:107BE00002E008C8121F08C1002AFAD17047704786
:107BF000002001E001C1121F002AFBD170470000E4
:107C00002DE9FF5F82B00021DDE90430020DDDF8CF
:107C100040B0034318D044F61050A2F2FF32424362
:107C20001514119801281FD0A5EB0B00401C5FEA2A
:107C3000000A4FF000064E4FDFF83891B04650462C
:107C400015D5CAF1000413E0119801244AA30128B4
:107C500001D16FEA0B010298119AC0E90031C0E925
:107C6000024206B0BDE8F09FCBF10000DFE704461A
:107C70000021404A491842EB0450CDE9001012E0BF
:107C8000E00707D032463B4640464946F8F7FDFC40
:107C90008046894632463B4610461946F8F7F5FCC1
:107CA00006460F466410002CEAD1DDE90401DDE947
:107CB0000023BAF1000F06DAF8F7E7FC42464B461C
:107CC000F8F7E3FC05E0F8F752FD42464B46F8F7BB
:107CD0004EFD04460E460022284BF9F72DF803D836
:107CE0004FF0FF30014607E00022254B2046314689
:107CF000F8F763FFF9F708F8102409E0002C0ADB15
:107D00000A220023F8F75CFA039B30321A55641EEE
:107D100050EA0102F2D1641C039AC4F11103144425
:107D2000119A012A03D0012208430DD10AE0084329
:107D300004D000204FF0110B119072E7A3EB0B055C
:107D40006D1E0DE05B4504DD4FF0000205F10105FD
:107D500004E003DA4FF00002A5F10105002AECD09F
:107D600002981199C0E90231C0E9004579E70000A5
:107D7000000014400000F03F300000000000F0431D
:107D80000000E03F2DE9FF4F95B09A468846064631
:107D90000025EEE1252877D100242746F94A012164
:107DA000039400E0044316F8013F203B01FA03F07E
:107DB0001042F7D130782A2811D06FF02F03307895
:107DC000A0F13002092A16D8039A44F0020402EB0B
:107DD000820203EB42021044761C0390EFE758F84E
:107DE000042B0392002A03DA504244F40054039017
:107DF00044F00204761C30782E2816D116F8010FB4
:107E000044F004042A280DD06FF02F023078A0F13E
:107E10003003092B09D807EB870302EB4303C7188C
:107E2000761CF3E758F8047B761C30786C280FD06A
:107E300006DC4C2817D068280DD06A2814D104E03D
:107E4000742810D07A280FD10DE044F400140AE011
:107E500044F4801401E044F440147278824202D168
:107E600004F58014761C761C307866280BD013DC61
:107E7000582877D009DC002875D04528F6D0462848
:107E8000F4D047281AD193E118E0632835D064284C
:107E900079D0652812D18BE1702873D008DC67286F
:107EA000F1D069286FD06E280DD06F2806D1ACE0D4
:107EB00073282CD0752874D0782853D0524617993F
:107EC00090476D1C54E1C4F30250022809D00328E6
:107ED0000DD0D8F8001004280DD00D6008F104086A
:107EE00046E1D8F80010EA17C1E90052F6E7D8F8E1
:107EF00000100D80F2E70D70F0E718F8041B8DF804
:107F0000001000208DF80100EB46012003E058F836
:107F100004BB4FF0FF3061074FF0000102D40DE0C9
:107F200009F101018946B9420FDA8145F8DB1BF8F6
:107F300009100029F4D108E009F1010189468142C4
:107F4000FADB1BF809100029F6D103985346A0EB81
:107F5000090721463846179A00F080FA284400EBBA
:107F6000090507E044E008E10DE01BF8010B52466B
:107F700017999047B9F10109F7D25346214638467F
:107F8000179AF2E039E00A21C4F302524FF0000BD5
:107F90000091022A06D058F8040BC117032A09D011
:107FA0000AE023E008F1070020F00702F2E80201EE
:107FB000904605E000B2C117042A01D140B2C117B2
:107FC000002906DA0A460021404261EB02012D2217
:107FD00002E0220504D52B228DF80420012203E0C3
:107FE000E20701D02022F7E7914657E00A2100E09E
:107FF00010214FF0000B00910BE010214FF0000B0F
:1080000044F004040827009103E008204FF0000B1F
:108010000090C4F30252022A05D058F8040B002144
:10802000032A08D008E008F1070020F00702F2E870
:108030000201904603E080B2042A00D1C0B24FF0A2
:10804000000922072AD53278702A07D0DDF800C04F
:108050008CF0100C5CEA0B0C05D00EE040228DF881
:108060000420012208E050EA010306D030238DF8F5
:1080700004308DF8052002229146009B83F008030E
:1080800053EA0B030AD150EA010201D1620705D578
:1080900030228DF804204FF001097F1E3278582AD3
:1080A00004D039A20C920CAA02920BE03BA2F9E791
:1080B0005B46009AF8F784F80C9B9B5C029A521E70
:1080C0000292137050EA0102F2D1029804A9081A30
:1080D00000F1200B600702D524F4803400E0012772
:1080E0005F4502DDA7EB0B0000E0002000EB0B0179
:1080F000009003984944401A0390E00306D4534685
:108100002146179A039800F0A9F90544002706E0D4
:1081100001A85246C05D179990476D1C7F1C4F45C2
:10812000F6DBE0030CD553462146179A039800F07E
:1081300095F9054404E030205246179990476D1C8C
:108140000099481E00900029F5DC08E00298029989
:1081500052460078491C0291179990476D1CBBF15B
:108160000001ABF1010BF1DC5BE100F065F90544C6
:10817000761C307800287FF40DAE19B02846BDE893
:10818000F08F0000092801003031323334353637A2
:108190003839616263646566000000003031323353
:1081A00034353637383941424344454600000000F3
:1081B000600700D4062708F1070020F00700F0E868
:1081C0000223804603F0004C5FEA0C0001D097A028
:1081D00009E0200501D596A005E0E00701D095A0B3
:1081E00001E0AFF24C001390307823F00043652893
:1081F0000CD006DC452809D046281DD047287FD161
:108200003BE0662818D067287AD136E00021112F8C
:1082100001DB112000E0781CCDE9000104A90CA8C5
:10822000FFF7EEFCDDE90D010C9A4FF0000B07F1B2
:108230000109109200914EE04FF000400097CDE907
:10824000011004A90CA8FFF7DBFCDDE90D020C9B73
:108250000F994FF0000B91461093009211B9791CC1
:1082600000EB0109B7EB090003D4C0F1FF3B07F1B4
:108270000109A9EB0700019042E0012F00DA012774
:108280000021112F01DD112000E03846CDE9000169
:1082900004A90CA8FFF7B4FCDDE90D010C9A0091CC
:1082A0004FF0000BB946109221070FD4009A4A45AF
:1082B00003DA914601E0A9F10109B9F1010F05DDE9
:1082C000109AA9F10101515C3029F4D0B84202DAC8
:1082D00010F1040F03DA0121CDE9011010E00028AC
:1082E00003DC8344A9EB000102E0411C494500DDA9
:1082F0008946A0EB0B00401C01904FF0004002901B
:10830000200705D40198484502DB4FF0FF3001906B
:1083100000208DF84B0002980DF14B07B0F1004F93
:1083200025D002200C902B200D90029800280CDA0A
:10833000404202902D200D9007E00A210298F8F7A4
:10834000DDFA3031029007F8011D0C99481E0C909F
:108350000029F2DC02980028EFD1791E0D980870F0
:10836000307800F0200040F0450007F8020D11A819
:10837000C01BC01D02901398007800B1012000EBD3
:108380000901019801EBE071029801440398401A39
:10839000401E0390E00306D453462146179A0398E3
:1083A00000F05CF805441398007818B1524617990C
:1083B00090476D1CE00323D553462146179A039836
:1083C00000F04CF805441BE0BBF1000F07DB009800
:1083D000584504DD1098179910F80B0001E0179923
:1083E00030205246904701980BF1010B401E05F1D9
:1083F0000105019004D12E205246179990476D1C1B
:10840000B9F10001A9F10109DEDC05E017F8010B63
:108410005246179990476D1C0299481E02900029F8
:10842000F4DC53462146179A03989EE62D0000007F
:108430002B000000200000002DE9F041044600253B
:108440001E461746880404D405E039462020B0476C
:108450006D1C641EF9D52846BDE8F0812DE9F04178
:10846000044600251E469046C80301D5302700E08B
:108470002027880404D505E041463846B0476D1CE6
:10848000641EF9D52846BDE8F0814A68002A06D066
:108490000A68531C0B6010704868401E48607047A3
:1084A00070B5144600280FD0002C0DD0002B0BD037
:1084B0005A1E914200DB591E0D460A4601462046CF
:1084C000F7F7E3FE0020605570BD00002DE9F04194
:1084D000040006D0184E306884420AD10020BDE85E
:1084E000F081502080F31188BFF34F8FBFF36F8F5F
:1084F000FEE703F01BF86569776BB66B03F036F89F
:10850000BD4201D0B54201D10220E8E70B488542C7
:1085100008D1A06A0028F7D194F858000128F3D0B8
:108520000320DCE705481438854202D00DB1012054
:10853000D5E70420D3E7000018000020600B0020DE
:1085400013B50020F8F79EFE4FF0FF330122694675
:10855000FBF7F4FA00981CBD10B5002821D0114B90
:108560000022001F196803E0814203D80A464968C7
:108570000029F9D152B11368841A9C4204D10068D1
:1085800018441060104602E0506000E0186039B1F5
:1085900002680B1A934203D10B681A4402604968BF
:1085A000416010BD2401002018B1012803D003A0B0
:1085B000704704A0704706A070470000554E4B4E10
:1085C0004F574E005641524941424C450000000071
:1085D000464958454400000038B1012807D0022818
:1085E00007D0032807D00548704705A0704705A0AD
:1085F000704706A0704707A070470000BC850008C0
:10860000424C45004C4F5241000000004746534B3E
:1086100000000000464C52430000000086281FD096
:108620000EDC4C281CD006DC042819D0282817D0D2
:10863000452813D114E0692812D070280ED10FE01C
:10864000C7280DD006DC8D280AD0AA2808D0B1286A
:1086500004D105E0CE2803D0EF2801D000207047D8
:108660000120704728B1102803D0202801D0002015
:10867000704701207047F9F709FDFEF758FCFCF739
:10868000A7FBFCF74DFBFCF72FFCFCF751FCFCF7BC
:1086900073FCFCF7D3FCFCF7EFFC00F005FCFCF7E7
:1086A0007DFB00F029FCFEE7F0B50B30154D20F006
:1086B00007010024144A0FE003688B420BD38B425E
:1086C00005D95E1A43184768C3E9006700E04368AC
:1086D000136002C004E0021D10680028ECD120469F
:1086E000002802D1286808B10020F0BD064A0748DA
:1086F0001060074A121A22F00702C0E90024012084
:108700002860D7E728010020240100201C30002029
:10871000183200202DE9F047A4B0002615468946FE
:10872000824619961A9619AA012128461B96F9F72E
:10873000A5F807461AAA02212846F9F79FF8044629
:108740001BAA03212846F9F799F80546202109A814
:10875000F7F790FD202111A8F7F78CFD20211CA828
:10876000F7F788FD2FB1202309AA38461999FFF79A
:1087700097FE2CB1202311AA20461A99FFF790FEEC
:108780002DB120231CAA28461B99FFF789FEDDA1E5
:1087900009A8F7F79CFD002848D0DCA109A8F7F745
:1087A00096FDDC4C002856D0DBA109A8F7F78FFD19
:1087B00000285ED0D9A109A8F7F789FD002861D06B
:1087C000D8A109A8F7F783FD0127D84C002864D069
:1087D000D7A109A8F7F77BFD0DF14408002871D057
:1087E000D6A109A8F7F773FDD54D00286BD0D5A108
:1087F00009A8F7F76CFD002870D0D3A109A8F7F7F6
:1088000066FD00286BD0D2A109A8F7F760FD00280B
:10881000F8D0D1A109A8F7F75AFD0028F2D0D0A1CD
:1088200009A8F7F754FD002879D0E4E0CE48F7F71F
:1088300038FDCE4C6168884200D86660CB4BCA4A8E
:108840001B1D4946504600F01EFC002800D1666002
:1088500024B0BDE8F087F8F74DFD0168491C0160C0
:10886000F8F748FD014638222046FCF701FEC0A279
:108870007BE0F8F73FFD014638222046FCF7EAFD91
:10888000C3A272E0F8F74CFDF8F734FD00F10801DF
:10889000A648FBF7D9FDC7A267E09AA111A8F7F790
:1088A00016FD88B19DF8440010B3CBA111A8F7F7CD
:1088B0000EFD58B1CBA111A8F7F709FD80B111AB9E
:1088C000CAA2E9E01CE047E0CE4A4EE0206880F80A
:1088D00058609648FCF7B2F9CBA246E05FE06CE046
:1088E000206880F858709148FCF7A8F9CEA23CE0C7
:1088F000206890F85800FFF757FE0346D1A2CBE05E
:108900009DF8440010B3002202A940460296F7F7F2
:10891000EDFD02990346414504D111AB00E067E04B
:10892000CEA2B9E0581E7B2801D3D3A2B4E02068C0
:10893000A0F85A307D48FCF781F92068D94AB0F890
:108940005A30181DCDE90003494690E02068D64A08
:10895000B0F85A30181DF5E768680770206890F87D
:10896000581039B1012908D0D0A249465046FFF726
:1089700009F9C2E0D648007803E0B0F85A00801C3C
:1089800080B26A49C2B228316D48FEF769FA674879
:10899000FBF72CFF6548FCF751F9CEA2E5E76968C3
:1089A000022008706648FEF741FA6048FBF71EFF98
:1089B0005E48FCF743F9CEA2D7E79DF828309DF832
:1089C00044105E20313B0029216800EB430006D0B3
:1089D00008444B46524611A902F0EEFC8DE0085ABD
:1089E0000090CCA2494650465B1CFFF7CBF884E0D0
:1089F0009DF8440068B1CEA109A8F7F768FC98B1CA
:108A0000CDA109A8F7F763FC00284AD009ABCCA296
:108A100042E02068B0F86220B0F86010CDE90012A2
:108A2000B0F85E30D6A221E09DF8440060B100228B
:108A300002A911A80296F7F721FD029903464145C4
:108A40000AD111ABDEA227E0686818B190F9503066
:108A5000E2A221E0E7A288E703F1120020280AD36E
:108A60000D216FF01100EEA2CDE9000149465046FC
:108A7000FFF788F841E069685CB259B181F850406D
:108A8000F34A69682046126D91F8511090472748C3
:108A9000FCF7D4F82346EFA249465046FFF772F898
:108AA0002BE068684078FFF797FD0646206890F84D
:108AB0005800FFF779FD69680A78012A1FD0EBA3F7
:108AC00091F950202168B1F86240CDE90542CDE925
:108AD0000763B1F86020B1F85E30B1F85C40B1F8DE
:108AE0005A100294CDE903320D1DCDE9001503465D
:108AF000DF4A49465046FFF745F80020A8E6DDA3C7
:108B0000DEE7000068656C70000000007361766548
:108B10000000000000F80008676574007265736566
:108B2000740000006D6F646500000000602F00207D
:108B300066697865646C656E0000000074780000FA
:108B4000702C002072780000727869643100000097
:108B50007278696432000000727869643300000042
:108B60007278696400000000D1F10008080100205B
:108B7000436F6E66696775726174696F6E207361A9
:108B800076656420746F20466C617368210D0A005D
:108B9000436F6E66696775726174696F6E206C6F82
:108BA000616465642066726F6D20466C6173680D48
:108BB0000A000000436F6E66696775726174696FC1
:108BC0006E20726573657420746F206465666175CC
:108BD0006C7473210D0A00005641524941424C45C4
:108BE000000000004649584544000000496E766187
:108BF0006C696420666F726D61743A2025730D0A8A
:108C00000000000028FA00084461746120666F7259
:108C10006D61742073657420746F3A205641524917
:108C200041424C450D0A00004461746120666F7238
:108C30006D61742073657420746F3A2046495845FD
:108C4000440D0A0043757272656E7420666F726D12
:108C500061743A2025730D0A00000000496E7661A8
:108C60006C6964206C656E6774682076616C7565EC
:108C70003A2025730D0A00004C656E677468206FFA
:108C80007574206F662072616E67653A20256C7579
:108C9000202876616C69643A20312E2E31323329D6
:108CA0000D0A00002CF60008C8F5000843616E6E3E
:108CB0006F74207472616E736D69743A20696E7698
:108CC000616C696420666F726D61740D0A0000004A
:108CD000050000205472616E736D697474696E676B
:108CE000207061636B65742E2E2E0D0A000000004B
:108CF0005374617274696E6720636F6E74696E7508
:108D00006F757320726563656976652E2E2E0D0A68
:108D10000000000043757272656E74205258494419
:108D200025643A203078253034580D0A00000000C0
:108D3000706F77657200000073686F770000000045
:108D4000496E76616C696420636F6D6D616E643A23
:108D50002025730D0A55736520276D723136206802
:108D6000656C702720666F7220617661696C616244
:108D70006C6520636F6D6D616E64730D0A00000099
:108D80005258204944733A0D0A2020525849443120
:108D90003A203078253034580D0A20205258494462
:108DA000323A203078253034580D0A202052584964
:108DB00044333A203078253034580D0A0000000042
:108DC000496E76616C696420706F77657220766198
:108DD0006C75653A2025730D0A00000043757272A8
:108DE000656E7420706F7765723A20256420644246
:108DF0006D0D0A0043757272656E7420706F776531
:108E0000723A2028726164696F206E6F7420696EF7
:108E1000697469616C697A6564290D0A0000000053
:108E2000506F776572206F7574206F662072616E67
:108E300067653A20256C642064426D202876616C59
:108E400069643A2025642E2E2564290D0A0000004D
:108E5000F0DC0008506F7765722073657420746FC2
:108E60002025642064426D0D0A0000005258000065
:108E70008CF600085458000010B5EFF3058111B1CD
:108E80006FF0050403E0002408B102F027FC20463F
:108E900010BDEFF3058008B103F0B0B803F0A8B837
:108EA0004FF47A7070470000EFF3058010B16FF057
:108EB000050070470448016811B14FF0FF3070475A
:108EC00001210160002070476800002010B5EFF319
:108ED000058010B16FF0050010BD03F07BF820B1E4
:108EE000022804D04FF0FF3010BD012010BD02F069
:108EF000E9FC002010BD000010B5EFF3058010B1B3
:108F00006FF0050010BD08480168012902D04FF03C
:108F1000FF3010BD054A002182F8141D02210160B6
:108F200002F08CFC002010BD680000200BE000E087
:108F300070B5EFF3058010B16FF0050413E003F096
:108F400049F84FF0FF3510B102280BD108E0012499
:108F500003F038F9012806D003F03CF810B102E024
:108F6000002400E02C46204670BDF8B514464FF0B2
:108F70000005EFF3058212BB08B301B3A4B1D4E935
:108F8000023263B1502A1AD32269C2B1676900FB69
:108F900001F6B74213D3009502F061FD07E072B904
:108FA000226962B9626952B9002202F037FD0500F8
:108FB00005D00CB1216800E0002102F059FB2846E1
:108FC000F8BD03F001B800002DE9FF414FEA0103AD
:108FD0004FF00005EFF30581039549BB40B38027AF
:108FE000182100244AB3166806B1344696691EB1AA
:108FF0003146761E382E02D21679F60703D00020AD
:1090000004B0BDE8F081566906B1B708D2F808C0CF
:10901000BCF1000F0DD0D5685C2D18D312693AB1A0
:1090200036B18DE806103A46214602F0A2FF0390C1
:109030000DE0D6685EB912694AB903AACDE90012FB
:10904000BAB2214602F068FF012800D003950398C8
:10905000D6E770B50546EFF3058010B16FF0050453
:109060000FE04DB12846FFF731FA042807D000245D
:10907000284602F059FB04E06FF0030401E06FF0B2
:109080000204204670BD2DE9F04781461D460C467E
:1090900090461046F7F705F9296806460027B142C1
:1090A00001D32F601AE0012C01D9641E00E00024D6
:1090B0002046741A844200D30446002CF1D0414467
:1090C00022464846F7F7BDF809F80470286820449E
:1090D0002860B04202D20120BDE8F0870020FBE703
:1090E0002DE9F041134C0F460546E6682068001D47
:1090F00002F0C0F9681C07D137B12168BDE8F04122
:109100000D48091D02F006BA20683544B542456095
:10911000216805D2A06BBDE8F041091D02F0E2B95B
:10912000606B091D02F0DEF9A06A854200D2A562DB
:10913000BDE8F08118000020600B00202DE9F0410F
:10914000054602F0F3F92D4CA068401CA060206891
:109150002B4F10B1606930B32BE02560A068012867
:1091600027D1002606EB860007EB800002F0ACF961
:10917000761C382EF6D3234802F0A6F92148143085
:1091800002F0A2F91F48283002F09EF91D483C3039
:1091900002F09AF91B48503002F096F919486063C2
:1091A0001430A06305E02068E96AC06A884200D8EC
:1091B0002560606A401C60626864E86A21698842D0
:1091C00000D9206100EB800007EB8000291D02F030
:1091D000A1F902F0CBF9606900280CD02068E96A97
:1091E000C06A884207D208494FF080500860BFF338
:1091F0004F8FBFF36F8FBDE8F08100001800002093
:10920000B0060020100B002004ED00E038B502F09D
:109210008DF9104C2068C8B90F4802F055F90E4876
:10922000143002F051F90C48E060143020610A4B10
:109230000020F03B009003F1500210210A2002F0C0
:109240000EFC206010B105A102F012FABDE8384012
:1092500002F08CB954000020640C0020546D72514F
:109260000000000030B4026C0B46002A0BD0C1682D
:109270001144C1608468A14201D30168C16030BC5F
:109280001846F6F7DEBF30BC70472DE9F041856B1C
:10929000174604460026026C82B1C7B1E068F6F7B3
:1092A000D0FFE168206C091AE1602268914202D285
:1092B000A168081AE060022F16D017E02068A8B94C
:1092C000A06802F007FF06460020A0600EE060687C
:1092D000F6F7B7FF216C606808446060A1688842B7
:1092E00004D32068606001E005B16D1E6D1CA563AC
:1092F0003046BDE8F08110B5044690F8590058B1E9
:1093000001280CD002280FD0502080F31188BFF321
:109310004F8FBFF36F8FFEE7206B02F03BF92046C3
:10932000BDE8104002F036B910BD000010484FF4FF
:109330004061420706D0C01D0D4920F00700411AC8
:10934000C1F540610B4A00230144C2E9000308391A
:10935000183A21F0070111604B600B600B1AC0E94D
:10936000001393604FF0004053605061704700005D
:10937000441300208400002010B5094CA26812B9E3
:1093800004F10C02A260126853680A461946F6F707
:109390007CFFA0684068A060002800D0012010BDBC
:1093A000F4000020144E154CA6F29C474FF0805854
:1093B000DFF84C9012E000BF02F0B8F8F068C56822
:1093C000281D02F057F8A068401EA0606068401E8B
:1093D000606002F0CBF82846FFF78DFF6068002838
:1093E000EAD138680128F9D9C9F80080BFF34F8F56
:1093F000BFF36F8FF2E700004C0B00201800002035
:1094000004ED00E070B51D46049C51B1C4F8002085
:10941000C4E90F010121204602F054FB84F84C50AE
:1094200070BD2460F4E700002DE9F05F8846DDE9B7
:109430000B941546834691009A460A9EA522206BFE
:10944000F6F711FF6FF00301206B01EB8501084473
:1094500020F00707780707D0502080F31188BFF36A
:109460004F8FBFF36F8FFEE70025B8F1000F0FD0CD
:109470005FF00000221818F8001082F8341018F875
:10948000001011B1401C1028F4D384F8435001E0BF
:1094900084F83450382E00D33726E662C4E91365C9
:1094A000201D02F01CF804F1180002F018F82461E5
:1094B000C6F138006462A061656584F85850524670
:1094C0005946384600F05AFA2060B9F1000F01D031
:1094D000C9F80040BDE8F09F30B5114900E01146E1
:1094E0000A688242FBD34B685C18844203D140680F
:1094F00018444860084643681C18944209D1084C37
:10950000183C2468A24209D052681A4442600A6892
:1095100012680260814200D0086030BD0460F9E743
:109520008400002070B5002441600B4D0061914221
:1095300006D8D11A8269914206D2011D286907E036
:109540009A4203D2994201D3012403E0011DE86845
:1095500001F0C8FF204670BD5400002010B504463D
:1095600001F0E4FFA06B28B15FF0000401F0FEFF02
:10957000204610BD0124F9E730B589B03C4D6EE0BE
:109580000498002806DADDE90601059A9047049858
:10959000002864DB069C606910B1201D01F06AFFA1
:1095A00003A800F0D7F8024604980A2857D2DFE84B
:1095B00000F00505052D334A05052D3394F82800E4
:1095C00040F0010084F828000599A069059B01443A
:1095D0002046FFF7A7FF68B3216A2046884794F822
:1095E000280040073BD5002000900598A169002382
:1095F00042181946204602F077FED8B9502080F371
:109600001188BFF34F8FBFF36F8FFEE714F8280F59
:1096100020F00100207022E094F8280040F00100C2
:1096200084F828000598A06128B1811813462046C7
:10963000FFF778FF13E0502080F31188BFF34F8FBE
:10964000BFF36F8FFEE794F82800810703D420460C
:1096500001F0A0FF03E020F0010084F828000022C0
:1096600004A9286802F082FB002889D109B030BD26
:10967000540000202DE9FC410F46054602F022F976
:1096800001A800F067F80446019818B102F09AFDAD
:10969000BDE8FC81254EAFB130690068D0B300272A
:1096A000291B3A46306801F0F7FF02F08BFD0028D5
:1096B000EED11F494FF080500860BFF34F8FBFF3CA
:1096C0006F8FE5E7A542EBD802F07CFDF0682746F6
:1096D000C068C468201D01F0CDFE94F82800410741
:1096E00019D5A0692B4641193A462046FFF71AFFC3
:1096F000A8B100200346014600902A46204602F009
:10970000F3FD60B9502080F31188BFF34F8FBFF392
:109710006F8FFEE707E020F0010084F82800216A3F
:1097200020468847B4E70127BAE70000540000202C
:1097300004ED00E00648416B096829B1416BC96836
:10974000C9684968816270474FF0FF31FAE700004D
:109750001800002070B5054602F04AFC064E04468B
:10976000B068844203D200F009F8012000E0002034
:1097700028602046B46070BD54000020F8B5194D33
:1097800020E0C068C4680668201D01F073FE216AED
:109790002046884794F82800400713D5A069304434
:1097A000B04206D924616060211DE86801F09AFE8C
:1097B00008E000200346014600903246204602F0B1
:1097C00093FD38B1E86801680029DAD12969C5E953
:1097D0000310F8BD502080F31188BFF34F8FBFF303
:1097E0006F8FFEE75400002008484068401C4FF08F
:1097F000500080F3118804D0BFF34F8FBFF36F8FF9
:10980000FEE7BFF34F8FBFF36F8FFEE78C000020A2
:10981000074CE068016841B1C0680021D0F8000041
:10982000FFF728FFFFF7A8FEF3E701210020F7E785
:10983000540000202DE9F041044601F077FE94F930
:10984000455004F1240609E0606A48B1304602F050
:1098500081FC08B101F0B8FF6D1E6DB2002DF3DC84
:109860004FF0FF3684F8456001F080FE01F05EFEA7
:1098700094F9445004F1100709E0206948B13846D2
:1098800002F068FC08B101F09FFF6D1E6DB2002D63
:10989000F3DC84F84460BDE8F04101F067BE0000ED
:1098A0002DE9F0410546002702F00CF8324E3068F1
:1098B00008B9FFF73BFD706905424ED1C5B30835C5
:1098C00068070ED005F00700C0F1080005446807DE
:1098D00007D0502080F31188BFF34F8FBFF36F8FF5
:1098E000FEE72DB37068854237D82348183001460B
:1098F0000C6801E020460C466168A94202D221684A
:109900000029F7D131688C4227D0076821680160AF
:1099100060680837411B10290FD96019420708D029
:10992000502080F31188BFF34F8FBFF36F8FFEE796
:1099300013E041606560FFF7CFFD61687068401A11
:109940007060B268904200D2B0607069014300203C
:10995000C4E90001F068401CF06002F033FC7807B5
:1099600007D0502080F31188BFF34F8FBFF36F8F64
:10997000FEE73846BDE8F0816C00002010B5031FFB
:109980004FF080741C601B1F21F001011960191F2A
:10999000024B0B60143940380A6010BDE99700088B
:1099A0002DE9F047B2B000271546894682462E972A
:1099B0002F9730972EAA012128463197F7F75EFF9F
:1099C00080462FAA02212846F7F758FF064630AAFC
:1099D00003212846F7F752FF044631AA04212846FE
:1099E000F7F74CFF054620211EA8F6F743FC20217F
:1099F0000EA8F6F73FFC202116A8F6F73BFC202125
:109A000026A8F6F737FCB8F1000004D020231EAAE0
:109A10002E99FEF745FD2EB120230EAA30462F9930
:109A2000FEF73EFD2CB1202316AA20463099FEF702
:109A300037FD2DB1202326AA28463199FEF730FDA7
:109A4000D8A11EA8F6F743FCD84E28B1D8A11EA86D
:109A5000F6F73DFCA0B118E0D848F6F722FCB16853
:109A6000884200D8B760D14BD44A083349465046A3
:109A7000FFF709FB002800D1B76032B0BDE8F087DE
:109A8000C8A10EA8F6F723FC28B1CDA11EA8F6F7B1
:109A90001EFC90B116E0CC48F6F703FCF168884252
:109AA00000D8F760C14BC84A0C3349465046FFF70F
:109AB000EAFA0028E1D1F760DFE7BAA10EA8F6F7CD
:109AC00006FC38B19DF898000024A8B10022114688
:109AD00026A817E0BD48F6F7E4FB3169884200D8B4
:109AE0003761B24BB94A103349465046FFF7CBFABB
:109AF0000028C2D13761C0E79DF8580028B1002284
:109B0000114616A8F6F7F2FC0446B1A11EA8F6F716
:109B1000DEFBB14D002831D0A5A11EA8F6F7D7FB7A
:109B2000DFF8B88200285AD0A5A11EA8F6F7CFFB0F
:109B300000286ED0AAA11EA8F6F7C9FB002801F0E4
:109B4000FB81AAA11EA8F6F7C2FB002801F07082D3
:109B5000A8A11EA8F6F7BBFB002801F07F82A8A1F0
:109B60001EA8F6F7B4FB002801F0C882A6A11EA823
:109B7000F6F7ADFB0028F7D0A6A293E09DF83800D9
:109B8000B0B1AAA10EA8F6F7A2FBC0B1A8A10EA879
:109B9000F6F79DFBA8B1A8A10EA8F6F798FB90B127
:109BA000A7A10EA8F6F793FB78B10EABA6A271E0C1
:109BB00068684078FEF710FD0346AAA26AE000211B
:109BC00004E0012102E0022100E003218248FDF7C8
:109BD000D5F808B1AAA265E00EABB0A25AE09DF894
:109BE0003800002868680AD090F83500002879D03D
:109BF000012870D003286FD004286ED139E090F886
:109C0000351099B1012920D0032928D0042903D087
:109C100000E000E3A7A245E090F8412090F8401052
:109C2000CDE9001290F83F30ABA208E090F8382060
:109C300090F83710CDE9001290F83630B4A24946BA
:109C40005046FDF79FFF01F06DBA90F83B2090F869
:109C50003A10CDE9001290F83930BBA2EFE790F846
:109C60003E2090F83D10CDE9001290F83C30C1A2A2
:109C7000E5E7CDA10EA8F6F72AFB80B1CCA10EA88E
:109C8000F6F725FBB8B1CDA10EA8F6F720FBD0B1B1
:109C90000EABCCA249465046FDF774FFD3E7EF2C3C
:109CA00005D9D2A249465046FDF76CFFCBE768685C
:109CB00080F83F40A8E20F2C01D9D7A2F2E76868EC
:109CC00080F84040A0E24CB1102C07D0202C05D0E9
:109CD000DCA2E7E706E032E057E2ABE2686880F832
:109CE000414091E2B0A10EA8F6F7F1FA60B1B0A13F
:109CF0000EA8F6F7ECFA78B1B0A10EA8F6F7E7FADD
:109D000090B10EABDCA2C5E7EF2C01D9E4A2C9E704
:109D1000686880F8364077E20F2C01D9EBA2C1E7E2
:109D2000686880F837406FE22CB1102C03D0202CEB
:109D300001D0F1A2B6E7686880F8384064E2FBA180
:109D40000EA8F6F7C4FA50B1F9A10EA8F6F7BFFABB
:109D5000D8B1F8A10EA8F6F7BAFA00B327E2502C52
:109D60000FD0602C0DD0702C0BD0802C09D0902CF3
:109D700007D0A02C05D0B02C03D0C02C01D0EEA26F
:109D800090E7686880F839403EE2342C08D0262CF1
:109D900006D0182C04D00A2C02D0EEA282E7EBE108
:109DA000E6E1000068656C7000000000080100201A
:109DB0006D6F64756C6174696F6E0000E8DF000898
:109DC0007061636B65740000A7E4000859EA00083D
:109DD0006D6F646500000000702C0020F0DC00084E
:109DE000626175647261746500000000706F776570
:109DF0007200000072616D7074696D650000000092
:109E0000726666726571000072666672657175656C
:109E10006E637900556E6B6E6F776E207261646948
:109E20006F20636F6D6D616E640D0A00424C4500DA
:109E30004C4F5241000000004746534B00000000C9
:109E4000464C524300000000556E6B6E6F776E20DB
:109E5000726164696F206D6F64653A2025730D0A25
:109E60000000000043757272656E7420726164694F
:109E70006F206D6F64653A2025730D0A00000000A5
:109E80004661696C656420746F207365742072612B
:109E900064696F206D6F64650D0A0000526164692A
:109EA0006F206D6F64652073657420746F20257357
:109EB0000D0A0000556E6B6E6F776E206D6F6475C6
:109EC0006C6174696F6E207061636B657420747966
:109ED00070650D0A000000004D6F64756C61746957
:109EE0006F6E28424C45293A2062725F62773D309E
:109EF000782558206D6F64696E6465783D257520FE
:109F000073686170696E673D307825580D0A0000EE
:109F10004D6F64756C6174696F6E284746534B29A9
:109F20003A2062725F62773D30782558206D6F6409
:109F3000696E6465783D25752073686170696E6728
:109F40003D307825580D0A004D6F64756C61746959
:109F50006F6E284C6F5261293A2073663D30782528
:109F6000582062773D307825582063723D3078253F
:109F7000580D0A004D6F64756C6174696F6E2846E8
:109F80004C5243293A2062725F62773D30782558FF
:109F90002063723D307825582073686170696E6760
:109FA0003D307825580D0A0062725F62770000002C
:109FB0006D6F64696E64657800000000736861709D
:109FC000696E6700556E6B6E6F776E206D6F64758E
:109FD0006C6174696F6E206669656C6420666F726F
:109FE00020424C453A2025730D0A0000496E7661E7
:109FF0006C69642062725F62772076616C7565209F
:10A00000666F7220424C4520286D61783A20307886
:10A010004546290D0A000000496E76616C6964208E
:10A020006D6F64696E6465782076616C7565206615
:10A030006F7220424C4520286D61783A20313529D5
:10A040000D0A0000496E76616C6964207368617066
:10A05000696E672076616C756520666F7220424C70
:10A06000452028307830302F307831302F3078321A
:10A0700030290D0A00000000556E6B6E6F776E2060
:10A080006D6F64756C6174696F6E206669656C6470
:10A0900020666F72204746534B3A2025730D0A0005
:10A0A000496E76616C69642062725F6277207661C6
:10A0B0006C756520666F72204746534B20286D6192
:10A0C000783A2030784546290D0A0000496E7661BD
:10A0D0006C6964206D6F64696E6465782076616C6C
:10A0E000756520666F72204746534B20286D617856
:10A0F0003A203135290D0A00496E76616C69642079
:10A1000073686170696E672076616C756520666F33
:10A1100072204746534B2028307830302F3078312A
:10A12000302F30783230290D0A00000073660000AD
:10A130006277000063720000496E76616C6964208A
:10A1400073662076616C756520666F72204C4F5285
:10A15000410D0A00496E76616C6964206277207651
:10A16000616C756520666F72204C4F52410D0A007C
:10A17000686880F83A4047E0601E072801D3F5A2DE
:10A1800090E5686880F83B403EE0AFF2E4110EA82D
:10A19000F6F79DF868B1AFF264010EA8F6F797F8EC
:10A1A000E8B1AFF2E8110EA8F6F791F810B3F0A2FB
:10A1B00078E5042C0FD0282C0DD0452C0BD0692C21
:10A1C00009D0862C07D0AA2C05D0C72C03D0EB2CA5
:10A1D00001D0EEA266E5686880F83C4014E02CB13E
:10A1E000022C03D0042C01D0F0A25BE5686880F853
:10A1F0003D4009E02CB1102C03D0202C01D0F2A25C
:10A2000050E5686880F83E406868D8F840103530FE
:10A210008847F6A246E59DF83800002868680BD00C
:10A22000407FF84E002870D001286FD003286ED0F0
:10A23000042851D0F4A235E5417F99B1012924D0F9
:10A24000032930D0042901D0F7A22BE590F8321071
:10A2500090F8343090F833208DE80E0090F83130CB
:10A26000F74AE6E390F8211002AD90F8244090F808
:10A27000233090F8222085E81E0090F82020C17F2E
:10A28000CDE90012837FEF4A21E090F8261090F884
:10A29000294090F8283090F827208DE81E0090F88B
:10A2A0002530E94A17E190F82D1002AD90F83040C2
:10A2B00090F82F3090F82E2085E81E0090F82C2082
:10A2C00090F82B10CDE9001290F82A30DF4A494669
:10A2D0005046FDF757FCB6E4DDA10EA8F5F7F7FFF1
:10A2E00080B1DFA10EA8F5F7F2FFB8B1DFA10EA88B
:10A2F000F5F7EDFFD0B1E1A10EA8F5F7E8FFE8B161
:10A30000E1A2CFE4042C05D902E020E0FCE246E320
:10A31000E4A2C7E4686880F83140D5E2012C01D995
:10A32000E9A2BFE4686880F83240F6E7072C01D95B
:10A33000EDA2B7E4686880F83340EEE71CB1082C62
:10A3400001D0F1A2AEE4686880F83440E5E7F7A1F7
:10A350000EA8F5F7BCFFB8B3F7A10EA8F5F7B7FF45
:10A3600098B3F9A10EA8F5F7B2FF78B3FAA10EA839
:10A37000F5F7ADFF58B3FBA10EA8F5F7A8FF38B36A
:10A38000FBA10EA8F5F7A3FFB0B3FCA10EA8F5F74B
:10A390009EFF002878D0FCA10EA8F5F798FF0028B2
:10A3A00073D0FBA10EA8F5F792FF00286ED0FAA19A
:10A3B0000EA8F5F78CFF002869D0B0A10EA8F5F71C
:10A3C00086FF00287BD004E005E019E026E03AE0B3
:10A3D0005EE0F2A266E484B1102C0ED0202C0CD0EA
:10A3E000302C0AD0402C08D0502C06D0602C04D041
:10A3F000702C02D0F04A55E472E06868847763E21A
:10A400004CB1022C07D0042C05D0062C03D0082C0C
:10A4100001D0EAA246E46868C47755E27CB1102C0A
:10A420000DD0202C0BD0302C09D0402C07D0502C34
:10A4300005D0602C03D0702C01D0EF4A32E468685C
:10A4400080F8204040E230680AAD417B047CC37B49
:10A45000827B85E81E00417A06AD047BC37A827A4E
:10A4600085E81E00417902AD047AC379827985E8D6
:10A470001E000279C178CDE900128378DF4A49468F
:10A480005046FDF77FFB09E44CE015E21DE225E2B2
:10A490009DF85800B0B10022114616A8F6F726F82C
:10A4A00031680346000E88703168180CC870316836
:10A4B000180A0871306843713068877100E01AE249
:10A4C000CFA220E43068C1788479437902798DE89D
:10A4D0001E008378D3A249465046FDF753FBFAE6A7
:10A4E0009DF85800A0B10022114616A8F5F7FEFF0E
:10A4F00031680346000EC8713168180CD4A2087286
:10A500003168180A4872306883723068C772D8E7B9
:10A510003068017AC47A837A427A8DE81E00C37962
:10A52000D4A2D8E79DF8580098B10022114616A889
:10A53000F5F7DCFF31680346000E08733168180C2C
:10A5400048733168180A88733068C37330680774B9
:10A55000A6E1A7E1496E76616C696420637220769A
:10A56000616C756520666F72204C4F52410D0A0078
:10A57000556E6B6E6F776E206D6F64756C6174696C
:10A580006F6E206669656C640D0A0000496E766125
:10A590006C69642062725F62772076616C756520F9
:10A5A000666F7220464C52430D0A0000496E766178
:10A5B0006C69642063722076616C756520666F72C9
:10A5C00020464C52430D0A00496E76616C69642046
:10A5D00073686170696E672076616C756520666F5F
:10A5E0007220464C52430D0A000000004D6F647506
:10A5F0006C6174696F6E20757064617465640D0AB6
:10A6000000000000602F0020556E6B6E6F776E208B
:10A6100063757272656E74207061636B657420740B
:10A620007970650D0A000000556E6B6E6F776E20B5
:10A630007061636B657420747970650D0A000000A9
:10A64000FCF8000890F80008D8F7000824F8000883
:10A65000436F6E6E656374696F6E537461746500E9
:10A660004372634669656C6400000000426C65508B
:10A6700061636B6574547970650000005768697494
:10A68000656E696E67000000556E6B6E6F776E20A9
:10A69000424C45207061636B6574206669656C642B
:10A6A0000D0A0000496E76616C696420424C4520B9
:10A6B000436F6E6E656374696F6E53746174652069
:10A6C00028302D34290D0A00496E76616C696420AA
:10A6D000424C45204372634669656C642028302DE6
:10A6E00031290D0A00000000496E76616C69642012
:10A6F000424C455061636B65745479706520283015
:10A700002D37290D0A000000496E76616C696420BE
:10A71000424C452057686974656E696E6720283021
:10A720007830302F30783038290D0A00507265614A
:10A730006D626C650000000053796E63576F726440
:10A740004C656E677468000053796E63576F72646E
:10A750004D6174636800000053796E63576F7264D3
:10A760000000000053796E63576F7264310000007F
:10A7700053796E63576F72643200000053796E63D1
:10A78000576F7264330000004865616465720000B1
:10A790005061796C6F61640043726300556E6B6E3B
:10A7A0006F776E204746534B207061636B65742052
:10A7B0006669656C640D0A00F4F40008496E766100
:10A7C0006C6964204746534B2053796E63576F7210
:10A7D000644C656E6774682028307830302F30788C
:10A7E00030322F307830342F307830362F30783088
:10A7F00038290D0A0000000080F50008B4F90008AF
:10A800004746534B2073796E6320776F7264203113
:10A810002073657420746F2030782530386C580DA3
:10A820000A0000004746534B2053796E6320576F50
:10A83000726420313A202530325825303258253084
:10A84000325825303258253032580D0A00000000A9
:10A850004746534B2073796E6320776F72642032C2
:10A860002073657420746F2030782530386C580D53
:10A870000A0000004746534B2053796E6320576F00
:10A88000726420323A202530325825303258253033
:10A89000325825303258253032580D0A0000000059
:10A8A000CBA20EE63068417B047CC37B827B8DE8C3
:10A8B0001E00037BCFA20EE61CB1202C01D0D8A233
:10A8C0005EE4686880F821402FE3601EFF2801D312
:10A8D000DCA255E4686880F8224026E33CB1102CE5
:10A8E00005D0202C03D0302C01D0DEA248E46868CB
:10A8F00080F8234019E31CB1082C01D0E4A23FE406
:10A90000686880F8244010E3AFF2E0110EA8F5F774
:10A91000DEFCC0B1AFF290110EA8F5F7D8FCD0B1B3
:10A92000AFF294110EA8F5F7D2FCE8B1AFF298118E
:10A930000EA8F5F7CCFC00B3DFA10EA8F5F7C7FC15
:10A9400020B3E0A21CE4FF2C01D9E5A218E468685A
:10A9500080F82540E9E21CB1802C01D0E8A20FE488
:10A96000686880F82640E0E2601EFF2801D3EDA26F
:10A9700006E4686880F82740D7E21CB1202C01D09B
:10A98000F0A215E4686880F82840CEE21CB1402CA3
:10A9900001D0F4A20CE4686880F82940C5E2AFF267
:10A9A00074210EA8F5F793FCF0B3AFF274210EA852
:10A9B000F5F78DFCC8B3AFF270210EA8F5F787FC50
:10A9C000A0B3AFF26C210EA8F5F781FC78B3AFF21B
:10A9D0006C210EA8F5F77BFC50B3AFF26C210EA8EA
:10A9E000F5F775FC30B3AFF26C210EA8F5F76FFCEC
:10A9F000A8B3AFF26C210EA8F5F769FC80B3AFF2F3
:10AA000070210EA8F5F763FC00287DD0AFF2782105
:10AA10000EA8F5F75CFC002877D0AFF2A0310EA8A5
:10AA2000F5F755FC002806E008E01EE02CE040E0C9
:10AA30005AE07BE07FE069D0D3A206E48CB1102C11
:10AA40000FD0202C0DD0302C0BD0402C09D0502C06
:10AA500007D0602C05D0702C03D0D24A51E489E095
:10AA6000A7E0686880F82A405FE24CB1022C07D06A
:10AA7000042C05D0062C03D0082C01D0CAA240E437
:10AA8000686880F82B4050E27CB1102C0DD0202C4F
:10AA90000BD0302C09D0402C07D0502C05D0602C86
:10AAA00003D0702C01D0CF4A2BE4686880F82C408A
:10AAB0003BE2306807AD417E047FC37E827E85E83D
:10AAC0001E00417D03AD047EC37D827D85E81E00AE
:10AAD000817C037DC27C8DE80E00437CC24A4946DE
:10AAE0005046FDF74FF81DE39DF85800B0B1002225
:10AAF000114616A8F5F7FAFC3268010E5174326857
:10AB0000010C9174010A02E05CE0F9E105E23268AF
:10AB10000346D1743168B5A20875D2E43068817CEF
:10AB2000037DC27C8DE80E00437CB9A249465046A5
:10AB3000FDF728F8F6E29DF8580090B10022114682
:10AB400016A8F5F7D3FC31680346000E4875316846
:10AB5000180CB9A288753168180AC8753068037670
:10AB6000AFE43068817D037EC27D8DE80E00437DB9
:10AB7000BAA2DBE79DF8580090B10022114616A852
:10AB8000F5F7B4FC31680346000E48763168180CBE
:10AB9000BCA288763168180AC8763068037790E4DA
:10ABA0003068817E037FC27E8DE80E00437EBEA2A8
:10ABB000BCE71CB1202C01D0C5A20BE4686880F86A
:10ABC0002D40B2E1601EFF2800D393E194E1000024
:10ABD0004746534B2073796E6320776F726420333E
:10ABE0002073657420746F2030782530386C580DD0
:10ABF0000A0000004746534B2053796E6320576F7D
:10AC0000726420333A2025303258253032582530AE
:10AC1000325825303258253032580D0A00000000D5
:10AC2000496E76616C6964204746534B20486561E4
:10AC30006465722028307830302F30783230290D1A
:10AC40000A000000496E76616C6964204746534BE8
:10AC5000205061796C6F61642028312D323535299F
:10AC60000D0A0000496E76616C6964204746534BBB
:10AC7000204372632028307830302F307831302FE5
:10AC8000307832302F30783330290D0A0000000040
:10AC9000496E76616C6964204746534B205768695A
:10ACA00074656E696E672028307830302F307830C8
:10ACB00038290D0A00000000496E7665727449510A
:10ACC00000000000556E6B6E6F776E204C6F526106
:10ACD000207061636B6574206669656C640D0A00A1
:10ACE000496E76616C6964204C6F526120507265C8
:10ACF000616D626C652028302D323535290D0A00D2
:10AD0000496E76616C6964204C6F526120486561C0
:10AD10006465722028307830302F30783830290D33
:10AD20000A000000496E76616C6964204C6F5261C4
:10AD3000205061796C6F61642028312D32353529BE
:10AD40000D0A0000496E76616C6964204C6F526197
:10AD5000204372632028307830302F307832302909
:10AD60000D0A0000496E76616C6964204C6F526177
:10AD700020496E7665727449512028307830302F22
:10AD800030783430290D0A00556E6B6E6F776E2067
:10AD9000464C5243207061636B6574206669656C34
:10ADA000640D0A00B0F40008496E76616C69642095
:10ADB000464C52432053796E63576F72644C656EF4
:10ADC0006774682028307830302F307830322F3058
:10ADD0007830342F307830362F30783038290D0ADB
:10ADE0000000000038F500084CF90008464C5243BA
:10ADF0002073796E6320776F7264203120736574DD
:10AE000020746F2030782530386C580D0A0000000F
:10AE1000464C52432053796E6320576F7264203141
:10AE20003A202530325825303258253032582530D6
:10AE300032580D0A00000000464C52432073796ED0
:10AE40006320776F726420322073657420746F20E2
:10AE500030782530386C580D0A000000464C5243BB
:10AE60002053796E6320576F726420323A20253068
:10AE700032582530325825303258253032580D0A94
:10AE800000000000464C52432073796E6320776FB8
:10AE9000726420332073657420746F2030782530FD
:10AEA000386C580D0A000000464C52432053796E0E
:10AEB0006320576F726420333A2025303258253092
:10AEC000325825303258253032580D0A0000000023
:10AED000496E76616C696420464C52432048656136
:10AEE0006465722028307830302F30783230290D68
:10AEF0000A0000008CA2E3E4686880F82E4014E0A9
:10AF00003CB1102C05D0202C03D0302C01D08EA2C7
:10AF1000D6E4686880F82F4007E01CB1082C01D007
:10AF200094A2CDE4686880F830406868D8F844108E
:10AF30001D30884799A2C3E49F490EA8F5F7C7F9C9
:10AF400070B19DF83800002868681DD0417871B351
:10AF500001293BD0022946D0032952D097A2AFE461
:10AF60009C48F5F79EF97169884200D877619A4B41
:10AF7000984A49465046FEF786F800287EF47DAD93
:10AF8000776132B0BDE8F0874078FDF725FB69684E
:10AF9000034691F8550091F8542091F8534091F8E8
:10AFA0005210CDE90220CDE900148C4A83E4FFE77A
:10AFB000022C02D923468AA273E4E1B280F852102F
:10AFC0009348FBF7F5FD7C4B883327E0072C02D92B
:10AFD000234690A265E4E1B280F853108C48FBF759
:10AFE00095FE98A31AE0032C02D9234697A258E4B1
:10AFF000E1B280F854108648FBF74EFE6E4B943356
:10B000000CE0032C02D923469CA24AE4E1B280F86A
:10B0100055107F48FBF706FE674B9C3308B1A3A28F
:10B020003FE4ACA2494650460094FCF7ABFD79E002
:10B030009DF8380068B1686864B280F8504068686C
:10B04000D8F8502090F85110204690472346ACA2E3
:10B0500027E46868B1A290F9503022E49DF83800E6
:10B06000002158B10A2C36D027DC022C3AD0042C0F
:10B070002BD0062C2BD0082C25D12AE0686802237F
:10B0800090F8510010F01F0F15D14011082812D26E
:10B09000DFE800F0110406080A0C0E1004230AE091
:10B0A000062308E0082306E00A2304E00C2302E05C
:10B0B000102300E01423A0A22FE50C2C0DD0102C9F
:10B0C0000DD0142C0DD0A3A210E420210AE04021C1
:10B0D00008E0602106E0802104E0A02102E0C02118
:10B0E00000E0E021686880F851106868D8F85020C6
:10B0F00090F95000904723469BA20EE59DF838003A
:10B1000030B121464248FBF775FE23469DA204E577
:10B110006868A2A2D0E91210CDE900104946504655
:10B12000FCF730FD00202CE7496E76616C696420E5
:10B13000464C5243205061796C6F61642028312D58
:10B14000323535290D0A0000496E76616C6964203C
:10B15000464C5243204372632028307830302F30E1
:10B160007831302F307832302F30783330290D0A53
:10B1700000000000496E76616C696420464C5243C1
:10B180002057686974656E696E67202830783030A2
:10B190002F30783038290D0A000000005061636BB1
:10B1A000657420706172616D65746572732075706D
:10B1B00064617465640D0A00A49D0008556E6B6E91
:10B1C0006F776E20726164696F206D6F64650D0A20
:10B1D0000000000042F200081C01002010FB0008E3
:10B1E000496E76616C696420424C452062617564E9
:10B1F0007261746520696E6465783A20256C7520EB
:10B200002876616C69643A20302D32290D0A0000DD
:10B21000702C0020496E76616C6964204C6F52611D
:10B2200020626175647261746520696E6465783A44
:10B2300020256C75202876616C69643A20302D37A2
:10B24000290D0A004C6F526100000000496E7661C2
:10B250006C6964204746534B206261756472617467
:10B260006520696E6465783A20256C7520287661C2
:10B270006C69643A20302D33290D0A00496E7661DD
:10B280006C696420464C524320626175647261743B
:10B290006520696E6465783A20256C752028766192
:10B2A0006C69643A20302D33290D0A004661696CBF
:10B2B000656420746F2075706461746520626175C7
:10B2C000647261746520666F72202573206D6F64EF
:10B2D000650D0A0042617564726174652075706461
:10B2E0006174656420666F72202573206D6F6465DC
:10B2F000202D3E20696E64657820256C750D0A004E
:10B30000545820706F7765722073657420746F20B5
:10B3100025642064426D0D0A0000000043757272BE
:10B32000656E7420545820706F7765723A202564DA
:10B330002064426D0D0A000043757272656E7420C0
:10B3400072616D702074696D653A20256C75207589
:10B35000730D0A00496E76616C69642072616D70CC
:10B3600074696D650D0A000052616D702074696D1D
:10B37000652073657420746F20256C752075730DBE
:10B380000A000000524620667265712073657420C1
:10B39000746F20256C7520487A0D0A00437572720F
:10B3A000656E7420524620667265713A20256C6C79
:10B3B0007520487A0D0A00007CB51D460B461646DE
:10B3C000044601AA0EA11846F4F796FFBDF8043012
:10B3D0004FF6FE704BB1834207D8238009A229465D
:10B3E0003046FCF7CFFB00207CBD009001230BA270
:10B3F00029463046FCF7C6FB4FF0FF307CBD00000D
:10B4000025687800525849442073657420746F3A57
:10B41000203078253034580D0A0000005258494435
:10B4200020736574206661696C65643A20696E7684
:10B43000616C69642076616C75650D0A56616C6992
:10B44000642072616E67653A203078253034582D5B
:10B450003078253034580D0A0000000001490020E2
:10B4600008707047F0000020014900200870704704
:10B47000F0000020D0E9013201699A60D0E901238F
:10B480005A604A68824201D182684A6000220261A1
:10B490000868401E0860086870470000034B03609E
:10B4A00003F15C0008608020106070478C0C002065
:10B4B000044B036003F15C0008604FF4807010607F
:10B4C00070470000E80E002000F108014FF0FF3245
:10B4D000C0E90112C16001610021016070470021D3
:10B4E0000161704730B50B685A1C02D000F10802A8
:10B4F00002E0026904E02246546825689D42FAD9B8
:10B5000053684B6099608A60516008610168491C0A
:10B51000016030BD42684A6093688B6093685960EF
:10B52000916008610168491C01607047502080F3F8
:10B530001188BFF34F8FBFF36F8F0A494868401CD3
:10B54000486001280CD10848006810F0FF0F07D0B0
:10B55000502080F31188BFF34F8FBFF36F8FFEE74A
:10B56000704700008C00002004ED00E008494868A6
:10B5700028B1401E486001D180F3118870475020E7
:10B5800080F31188BFF34F8FBFF36F8FFEE700008A
:10B590008C00002070B500282AD0164DA0F10804B8
:10B5A00060686969084207D1502080F31188BFF3B1
:10B5B0004F8FBFF36F8FFEE722683AB1502080F3C0
:10B5C0001188BFF34F8FBFF36F8FFEE78843606032
:10B5D00000F078F960686968084468602046FDF703
:10B5E0007BFF2869401C2861BDE8704000F0EABD7F
:10B5F00070BD00006C0000204FF0E02000210161D0
:10B60000816105494FF47A720968B1FBF2F1491E74
:10B6100041610721016170471400002010B5F4F763
:10B62000B9FD114910280ED300F1E02090F8F00385
:10B630000A78904207D2502080F31188BFF34F8FD1
:10B64000BFF36F8FFEE709480068896800F4E06087
:10B65000884207D9502080F31188BFF34F8FBFF382
:10B660006F8FFEE710BD00008C0000200CED00E0A5
:10B6700010B5084B002200BF53F832401CB1521CD9
:10B68000082AF9D310BD43F8321003EBC201486019
:10B6900010BD00007006002070B515460E46044629
:10B6A000FFF744FF94F944100020491C01D184F8AD
:10B6B000440094F94510491C01D184F84500FFF776
:10B6C00055FFA06B28B92A46314604F1240000F04A
:10B6D00099F82046BDE87040FEF7ACB810B50200FE
:10B6E00014D00F48006B38B1502080F31188BFF39D
:10B6F0004F8FBFF36F8FFEE700F0E4F80021104694
:10B70000FDF7EEFC00F05EFD002807D105494FF083
:10B7100080500860BFF34F8FBFF36F8F10BD0000E4
:10B720001800002004ED00E070B50546FFF7FEFEAE
:10B730001E4C05B92568281DFFF79CFEA86A18B1A4
:10B7400005F11800FFF796FE606A401C60622068F1
:10B75000854207D1291D1648FFF7DCFE6068401CB2
:10B76000606007E0A068401EA0602846FDF7C3FDAA
:10B77000FDF7E0FFFFF7FAFE6069002814D02068AB
:10B78000854211D1206B38B1502080F31188BFF36E
:10B790004F8FBFF36F8FFEE706494FF08050086070
:10B7A000BFF34F8FBFF36F8F70BD000018000020F4
:10B7B0004C0B002004ED00E002490A6A0260C968EF
:10B7C000416070471800002001490120C86170479E
:10B7D0001800002010B50C4650B10949096818310D
:10B7E000FFF780FE2046BDE810400121FDF778BC40
:10B7F000502080F31188BFF34F8FBFF36F8FFEE7A8
:10B800001800002070B514460D4668B10A49096851
:10B810001831FFF77FFE0CB14FF0FF352146284667
:10B82000BDE87040FDF75CBC502080F31188BFF389
:10B830004F8FBFF36F8FFEE71800002030B587B041
:10B840000024039405AA04A903A80494FFF726FE84
:10B85000DDE903010094CDE90110002315A117488B
:10B86000059A00F086FB164D0028E8621FD000F014
:10B870000BFD012809D0401C19D1502080F31188FC
:10B88000BFF34F8FBFF36F8FFEE7502080F3118817
:10B89000BFF34F8FBFF36F8F4FF0FF30A8620120CF
:10B8A0006861EC6007B0BDE8304000F04DB807B00B
:10B8B00030BD000049444C4500000000A59300083D
:10B8C000180000200248016B491C0163704700000A
:10B8D00018000020164810B5016B11B10121C1619B
:10B8E00010BD0021C1610169124A01E0B9B1491ED0
:10B8F00001EB810352F82330002BF7D001EB8103D9
:10B9000002EB830202F1080453685B685360A342B0
:10B9100001D15B685360DA680260016110BD50209C
:10B9200080F31188BFF34F8FBFF36F8FFEE70000E6
:10B9300018000020B006002010B50020F5F72AFC02
:10B940000128FAD110BD00001CB5264908780190E5
:10B95000FF20087008788DF800009DF800009DF821
:10B96000002000F0F000904207D0502080F31188B2
:10B97000BFF34F8FBFF36F8FFEE79DF800001A4CA7
:10B9800000F0500020700720A06005E09DF8002026
:10B9900052008DF80020401E9DF800201206F5D4BC
:10B9A000A060032807D0502080F31188BFF34F8F89
:10B9B000BFF36F8FFEE74FF44070A06001980870EE
:10B9C0000A48016841F470010160016841F070416A
:10B9D0000160FFF711FE00206060F4F7A5FB002076
:10B9E0001CBD000000E400E08C00002020ED00E021
:10B9F00010B5502080F31188BFF34F8FBFF36F8FC6
:10BA000000F004FB18B104494FF08050086000209A
:10BA100080F3118810BD000004ED00E0F8B5174672
:10BA20000E46050013D005FB06F05030FDF738FF39
:10BA300004000AD0002084F8460004F150023B467E
:10BA4000314628460094FDF7DDFC2046F8BD502025
:10BA500080F31188BFF34F8FBFF36F8FFEE738B5C8
:10BA6000049D18B153B1CAB181B120E0502080F3D8
:10BA70001188BFF34F8FBFF36F8FFEE7502080F325
:10BA80001188BFF34F8FBFF36F8FFEE7502080F315
:10BA90001188BFF34F8FBFF36F8FFEE739B150208E
:10BAA00080F31188BFF34F8FBFF36F8FFEE75024F1
:10BAB0001C46012384F846302B460094FDF7A2FC77
:10BAC000204638BD70B50D46040025D0FFF72EFD89
:10BAD000D4E90F20216802FB0011A1600021A163BD
:10BAE000216861600A46D4E90F01401E00FB012174
:10BAF000E16021464FF0FF3001F8440F487004F137
:10BB000010008DB1FFF7E0FC04F12400FFF7DCFC2E
:10BB1000FFF72CFD012070BD502080F31188BFF38A
:10BB20004F8FBFF36F8FFEE721690029F0D000F03F
:10BB300011FB0028ECD004494FF080500860BFF39F
:10BB40004F8FBFF36F8FE3E704ED00E02DE9FF4770
:10BB500082B01D468A464FF00008040003D0BAF1B7
:10BB6000000F08D011E0502080F31188BFF34F8FF1
:10BB7000BFF36F8FFEE7206C38B1502080F311883F
:10BB8000BFF34F8FBFF36F8FFEE7022D0AD1E06B3B
:10BB9000012807D0502080F31188BFF34F8FBFF3E7
:10BBA0006F8FFEE700F016FA3F4F4FF000094FF09D
:10BBB000805648B9049838B1502080F31188BFF3FB
:10BBC0004F8FBFF36F8FFEE7FFF7B0FCA06BE16B09
:10BBD000884207D3022D05D00498D0B1B8F1000FE8
:10BBE0001AD01EE02A4651462046FDF74EFB616AF8
:10BBF00019B104F1240000F0ADFA20B13E60BFF3AA
:10BC00004F8FBFF36F8FFFF7B1FC012006B0BDE887
:10BC1000F087FFF7ABFC22E06846FFF7CDFD4FF061
:10BC20000108FFF7A3FCFFF74DFEFFF77FFC94F937
:10BC30004400401C01D184F8449094F94500401C14
:10BC400001D184F84590FFF791FC04A9684600F003
:10BC500029F930B12046FDF7EDFD00F0B3FA0020E0
:10BC6000D4E7FFF763FCA06BE16B884213D1FFF7C9
:10BC70007DFC04F110000499FFF7ACFD2046FDF7B0
:10BC8000D9FD00F09FFA00289ED13E60BFF34F8F90
:10BC9000BFF36F8F98E7FFF769FC2046FDF7CAFDF9
:10BCA00000F090FA90E7000004ED00E02DE9F04785
:10BCB0001F4690468946040003D0B9F1000F08D012
:10BCC00011E0502080F31188BFF34F8FBFF36F8FC7
:10BCD000FEE7206C38B1502080F31188BFF34F8FFE
:10BCE000BFF36F8FFEE7022F0AD1E06B012807D068
:10BCF000502080F31188BFF34F8FBFF36F8FFEE7A3
:10BD0000FFF78CFC5020EFF3118680F31188BFF30E
:10BD10004F8FBFF36F8FA06BE16B884206D3022F6A
:10BD200004D0002086F31188BDE8F08794F94550CF
:10BD3000A06B3A4649462046FDF7A7FA681C04D096
:10BD40006D1C84F845500120ECE7606A0028FAD0A9
:10BD500004F1240000F0FEF90028F4D0B8F1000F3F
:10BD6000F1D00121C8F80010EDE700002DE9F747F8
:10BD7000002683B08A46040003D0BAF1000F08D031
:10BD800011E0502080F31188BFF34F8FBFF36F8F06
:10BD9000FEE7206C38B1502080F31188BFF34F8F3D
:10BDA000BFF36F8FFEE700F015F9DFF8F4804FF076
:10BDB00000094FF0805748B9059838B1502080F3FA
:10BDC0001188BFF34F8FBFF36F8FFEE7FFF7AEFB16
:10BDD000A56BC5B151462046FDF744FA6D1EA5631B
:10BDE000206950B104F1100000F0B4F928B1C8F88E
:10BDF0000070BFF34F8FBFF36F8FFFF7B7FB0120CA
:10BE000006B0BDE8F087059808B11EB106E0FFF75F
:10BE1000ADFB27E06846FFF7CFFC0126FFF7A6FB46
:10BE2000FFF750FDFFF782FB94F94400401C01D15D
:10BE300084F8449094F94500401C01D184F8459061
:10BE4000FFF794FB05A9684600F02CF8002820466F
:10BE50000AD0FDF7EFFC00F0B5F92046FDF77EFBB8
:10BE60000028B3D00020CBE7FDF778FB90B104F1B8
:10BE700024000599FFF7AEFC2046FDF7DBFC00F03F
:10BE8000A1F90028A2D1C8F80070BFF34F8FBFF30B
:10BE90006F8F9BE72046FDF7CDFC00F093F995E707
:10BEA00004ED00E02DE9F0410C46050011D0C4B1CD
:10BEB000FFF73CFB174BDA686E682068911B471C44
:10BEC00017D02F681B6A9F4219D0964217D80124B9
:10BED00010E0502080F31188BFF34F8FBFF36F8FB6
:10BEE000FEE7502080F31188BFF34F8FBFF36F8FB1
:10BEF000FEE70024FFF73AFB2046BDE8F0818842C8
:10BF000005D9401A20602846FFF756FCF1E70020CB
:10BF10002060DCE7180000202DE9FF5F8346DDE9A3
:10BF20000E87994616468A469000FDF7B9FC050033
:10BF30001CD05C20FDF7B4FC040014D00020256365
:10BF400084F85900CDE90240CDE900874B463246DE
:10BF500051465846FDF768FA2046FDF7EFF80120F4
:10BF600004B0BDE8F09F2846FFF714FB4FF0FF3008
:10BF7000F6E7F0B585B0DDE90B640A9DA6B1DCB14A
:10BF80005C2700972663022684F85960002604AFD8
:10BF9000CDE90246CDE90057FDF746FA2046FDF708
:10BFA000CDF8049805B0F0BD502080F31188BFF3A0
:10BFB0004F8FBFF36F8FFEE7502080F31188BFF3E0
:10BFC0004F8FBFF36F8FFEE7014800687047000096
:10BFD000180000200548416919B1006B18B1002014
:10BFE00070470120704702207047000018000020B1
:10BFF0000148C068704700001800002010B5FFF726
:10C000000DFB0148C06810BD180000202DE9F0416B
:10C010002E4C0027206B28B1A069401CA061384637
:10C02000BDE8F081E668761CE66013D1606B0068BD
:10C0300038B1502080F31188BFF34F8FBFF36F8F5B
:10C04000FEE7606BA16B6163A063206A401C206205
:10C05000FDF770FBA06ADFF87880864209D3606B39
:10C060000068A0B1606BC068C5686868864211D27C
:10C07000A0622068C06A00EB800158F82100012806
:10C0800000D90127E0690028C9D00127C7E74FF090
:10C09000FF30EDE7281DFFF7EDF9A86A18B105F1AB
:10C0A0001800FFF7E7F9E86A2169884200D92061A2
:10C0B00000EB800108EB8100291DFFF72BFAE86AED
:10C0C0002168C96A8842CAD30127C8E7180000203E
:10C0D000B006002070B504004FF0000133D01B4DB6
:10C0E0002868844207D0502080F31188BFF34F8F17
:10C0F000BFF36F8FFEE7206D38B1401E2065E36C03
:10C10000E26A9A421FD040B11DE0502080F31188AE
:10C11000BFF34F8FBFF36F8FFEE7201DFFF7AAF924
:10C12000E06CE062C0F13800A061E06A29698842F1
:10C1300000D92861064900EB800001EB8000211D39
:10C14000FFF7E8F90121084670BD00001800002043
:10C15000B006002070B5C068C46854B104F118007E
:10C160000646FFF787F9144D286B50B13146134846
:10C1700015E0502080F31188BFF34F8FBFF36F8F0E
:10C18000FEE7201DFFF776F9E06A2969884200D9A9
:10C1900028610B4900EB800001EB8000211DFFF7B7
:10C1A000B9F9E06A2968C96A884202D90120E861C0
:10C1B00070BD002070BD000018000020380B00206A
:10C1C000B00600202DE9F0472C4D00242746286BAF
:10C1D00038B1FFF7ABF9286B401E2863286B40B1DC
:10C1E00046E0502080F31188BFF34F8FBFF36F8F6D
:10C1F000FEE7A968224E0120D1B3A6F591698046D9
:10C200003068E0B1F068C46804F11800FFF732F953
:10C21000201DFFF72FF9E06A2969884200D92861BB
:10C2200000EB800109EB8100211DFFF773F9E06A43
:10C230002968C96A8842E3D3C5F81C80E0E70CB1DD
:10C24000FDF778FAAC694CB14FEA0806FFF7DEFE5D
:10C2500000B1EE61641EF9D10020A861E86938B12F
:10C260000849012738070860BFF34F8FBFF36F8F6E
:10C27000FFF77CF93846BDE8F08700001800002081
:10C28000380B002004ED00E010B586B0FCF7BEFFCF
:10C29000114C2068B8B100200390049005AA04A9AD
:10C2A00003A8FFF705F9DDE9032102208DE8070067
:10C2B00000230AA10B48059AFFF75BFE606010B1EE
:10C2C00006B0012010BD502080F31188BFF34F8FBE
:10C2D000BFF36F8FFEE7000054000020546D722002
:10C2E00053766300119800082DE9FF411E4613465E
:10C2F00002000A9D4FF0000016D0144C2768002F52
:10C300000FD0CDE900130292062917DAFFF762FE7B
:10C3100002284FF000030FD0002269462068FFF783
:10C3200015FC04B0BDE8F081502080F31188BFF304
:10C330004F8FBFF36F8FFEE72A46EEE700233246AA
:10C3400069463846FFF7B2FCEBE7000054000020D6
:10C35000C4F300080000000000000000000000001E
:10C3600000000000000200001800000000000000B3
:10C3700000000000010202030405060708090A0B79
:10C380000C0D0E0F10100000000000000000010254
:10C39000030406070809000000000102030400006E
:10C3A000AC0200200C0000000000000000000000B3
:10C3B0000000000000000000000000080808080855
:10C3C000080800001818000000486C241200000043
:10C3D00000000000000000000000002424247F1260
:10C3E00012127F12121200000000081C2A2A0A0CE6
:10C3F0001828282A2A1C08080000002225151515CF
:10C400002A585454542200000000000C1212120A40
:10C4100076252911916E0000000606040300000035
:10C420000000000000000000004020101008080874
:10C43000080808101020400000020408081010101E
:10C4400010101008080402000000000008086B1C0F
:10C450001C6B080800000000000000000808080825
:10C460007F0808080800000000000000000000002D
:10C4700000000000060604030000000000000000A9
:10C48000FE000000000000000000000000000000AE
:10C490000000000006060000000080404020201040
:10C4A000100808040402020000000018244242425E
:10C4B0004242424224180000000000080E0808080A
:10C4C00008080808083E00000000003C42424220E4
:10C4D00020100804427E00000000003C4242201868
:10C4E00020404042221C000000000020302824246C
:10C4F00022227E20207800000000007E0202021A24
:10C5000026404042221C0000000000382402021A8B
:10C5100026424242241800000000007E2222101011
:10C5200008080808080800000000003C42424224B5
:10C5300018244242423C00000000001824424242BB
:10C5400064584040241C000000000000000018183F
:10C5500000000000181800000000000000000008A3
:10C56000000000000008080400000040201008043B
:10C5700002040810204000000000000000007F00BE
:10C5800000007F00000000000000000204081020EE
:10C5900040201008040200000000003C42424640D7
:10C5A00020101000181800000000001C225A5555D9
:10C5B00055552D42221C00000000000808181414D4
:10C5C000243C224242E700000000001F2222221EDB
:10C5D00022424242221F00000000007C4242010130
:10C5E00001010142221C00000000001F22424242C1
:10C5F00042424242221F00000000003F4212121E2F
:10C6000012120242423F00000000003F4212121E7E
:10C6100012120202020700000000003C2222010167
:10C6200001712122221C0000000000E74242424228
:10C630007E42424242E700000000003E080808082F
:10C6400008080808083E00000000007C10101010C8
:10C65000101010101010110F0000007722120A0E97
:10C660000A121222227700000000000702020202D2
:10C6700002020202427F00000000007736363636A2
:10C680002A2A2A2A2A6B0000000000E346464A4A6A
:10C6900052525262624700000000001C2241414198
:10C6A00041414141221C00000000003F4242424201
:10C6B0003E020202020700000000001C224141412C
:10C6C00041414D53321C60000000003F4242423E57
:10C6D0001212222242C700000000007C42420204E3
:10C6E00018204042423E00000000007F4908080830
:10C6F00008080808081C0000000000E74242424207
:10C7000042424242423C0000000000E742422224F2
:10C7100024141418080800000000006B4949494916
:10C720005555362222220000000000E7422424183A
:10C730001818242442E70000000000772222141475
:10C7400008080808081C00000000007E21201010C6
:10C7500008040442423F000000780808080808085E
:10C760000808080808087800000002020404080805
:10C770000810102020204040001E10101010101033
:10C780001010101010101E000038440000000000AF
:10C790000000000000000000000000000000000099
:10C7A00000000000000000FF00060800000000007C
:10C7B0000000000000000000000000000000003C3D
:10C7C0004278444242FC0000000000030202021AC8
:10C7D00026424242261A00000000000000000038F5
:10C7E00044020202443800000000006040404078EB
:10C7F0004442424264D80000000000000000003CB7
:10C80000427E0202423C0000000000F08808087EE0
:10C8100008080808083E0000000000000000007C36
:10C8200022221C023C42423C000000030202023A67
:10C830004642424242E700000000000C0C00000E9D
:10C8400008080808083E00000000003030000038EA
:10C85000202020202020221E00000003020202725D
:10C86000120A1612227700000000000E08080808BD
:10C8700008080808083E0000000000000000007FD3
:10C880009292929292B70000000000000000003BDC
:10C890004642424242E70000000000000000003C27
:10C8A00042424242423C0000000000000000001BE7
:10C8B00026424242221E02070000000000000078CB
:10C8C00044424242447840E000000000000000770B
:10C8D0004C040404041F0000000000000000007C61
:10C8E00042023C40423E0000000000000008083EBA
:10C8F000080808080830000000000000000000637D
:10C900004242424262DC000000000000000000E7FA
:10C91000422424140808000000000000000000EB7E
:10C920004949555522220000000000000000007611
:10C9300024181818246E000000000000000000E712
:10C940004224241418080807000000000000007E9C
:10C9500022100808447E000000C020202020201063
:10C96000202020202020C0001010101010101010C7
:10C9700010101010101010100006080808080810F9
:10C9800008080808080806000C32C2000000000071
:10C990000000000000000000000000000000000097
:10C9A0000000000000000000000000000000000087
:10C9B0000000000000000000000000000000000077
:10C9C0000000000000000000000000000000000067
:10C9D0006000600060006000600060006000400077
:10C9E0002000200020000000000000006000600027
:10C9F000600000000000000000000000600660060B
:10CA0000300398018800440000000000000000008E
:10CA10000000000000000000000000000000000016
:10CA20000000000000000000000000000000000006
:10CA30001002100210021002FE07FE070802080191
:10CA4000080108010801FE07FE07040104010401B2
:10CA50000401000000000000000000000000400091
:10CA60004000F00158034C03CC034C005800700008
:10CA7000E000C001C00140034C035C034C034801CB
:10CA8000F000400040000000000000000000000036
:10CA90000E010A01910091009100510051003A00ED
:10CAA000AE03A00250045004480448044804840221
:10CAB00084030000000000000000000000000000EF
:10CAC00038006C006C006C006C006C002C00980747
:10CAD0001C011A01330133016301E300C308C609D5
:10CAE0003C07000000000000000000000C001C00DB
:10CAF000100010000800040000000000000000000A
:10CB00000000000000000000000000000000000025
:10CB1000000000000000000000000000000400020F
:10CB20000001800080004000400020002000200024
:10CB300020002000200020004000400080008000F5
:10CB400000010002000400000000000002000400D8
:10CB500008001000100020002000400040004000AD
:10CB60004000400040004000200020001000100065
:10CB700008000400020000000000000000000000A7
:10CB8000000000004000C0004000460C4E0FD001E5
:10CB9000F0015E0F460C4000400040000000000025
:10CBA0000000000000000000000000000000000085
:10CBB0000000000000004000400040004000400035
:10CBC000FE0F400040004000400040000000000018
:10CBD0000000000000000000000000000000000055
:10CBE0000000000000000000000000000000000045
:10CBF0000000000000000000000000000C001C000D
:10CC000010001000080004000000000000000000F8
:10CC10000000000000000000000000000000000014
:10CC2000FE070000000000000000000000000000FF
:10CC300000000000000000000000000000000000F4
:10CC400000000000000000000000000000000000E4
:10CC50000000000000000000000000001C001C009C
:10CC60001C0000000000000000000000000400069E
:10CC7000000200030001000180008000400040002D
:10CC800060002000200010001000080008000C00C8
:10CC90000400060002000000000000000000000088
:10CCA0000000F00098010C030C03060606060606B9
:10CCB000060606060606060606060C030C03980181
:10CCC000F000000000000000000000000000000074
:10CCD000000040007C0060006000600060006000B8
:10CCE0006000600060006000600060006000600044
:10CCF000FC03000000000000000000000000000035
:10CD00000000F8008401020306030603000300018B
:10CD10008001C0006000200010000802040206022A
:10CD2000FE03000000000000000000000000000002
:10CD300000007800C6008601860180018001C000E5
:10CD40007000800100010003000306030603860152
:10CD5000F8000000000000000000000000000000DB
:10CD6000000080018001C001A001A00190018801A4
:10CD7000880184018201FE0F800180018001800111
:10CD8000E0070000000000000000000000000000BC
:10CD90000000FC0304000400040004000400F4008C
:10CDA0008C010403000300030603060382018401CF
:10CDB000F80000000000000000000000000000007B
:10CDC0000000E00118030C030C0004000600E6015B
:10CDD00016030E0606060606060604060C021803CF
:10CDE000F000000000000000000000000000000053
:10CDF0000000F8070C060402040100010001800095
:10CE00008000400040004000600060006000600062
:10CE100060000000000000000000000000000000B2
:10CE20000000F8010C030606060606060C021C03A9
:10CE3000F000C8010C0306060606060606060C03EB
:10CE4000F0010000000000000000000000000000F1
:10CE50000000F0000C010C0306020606060606069A
:10CE600006078C0678060006000300030C018C01FF
:10CE7000780000000000000000000000000000003A
:10CE8000000000000000000000000000E000E000E2
:10CE9000E00000000000000000000000E000E000F2
:10CEA000E0000000000000000000000000000000A2
:10CEB00000000000000000000000000060006000B2
:10CEC0000000000000000000000000000000600002
:10CED0006000400020002000000000000000000072
:10CEE0000004000200018000400020001000080043
:10CEF0000400080010002000400080000001000233
:10CF0000000400000000000000000000000000001D
:10CF1000000000000000000000000000FE0700000C
:10CF200000000000FE0700000000000000000000FC
:10CF300000000000000000000000000000000000F1
:10CF400004000800100020004000800000010002E2
:10CF500000040002000180004000200010000800D2
:10CF600004000000000000000000000000000000BD
:10CF70000000E0031806040C040C0C0C0C0C000759
:10CF8000800140004000400000000000E000E000A0
:10CF9000E0000000000000000000000000000000B1
:10CFA000E00018030C02CC0564056605A605B6046E
:10CFB000B604B604B604B602E4010C040C0218036D
:10CFC000F000000000000000000000000000000071
:10CFD0000000600060005000D000900090008800C9
:10CFE00088010801F8010403040304020202020696
:10CFF0000F0F000000000000000000000000000013
:10D000000000FE008C030C030C030C030C038C01CA
:10D01000FC000C030C020C060C060C060C060C03A0
:10D02000FE01000000000000000000000000000001
:10D030000000E00318030C060C04040406000600BC
:10D04000060006000600060006040C040C02180385
:10D05000F0000000000000000000000000000000E0
:10D0600000007F008C010C030C030C060C060C0660
:10D070000C060C060C060C060C060C030C038C01AB
:10D080007F00000000000000000000000000000021
:10D090000000FF030603060406040600860086005F
:10D0A000FE008600860086000600060406040602CE
:10D0B000FF0300000000000000000000000000006E
:10D0C0000000FF030603060406040600860086002F
:10D0D000FE008600860086000600060006000600A8
:10D0E0001F00000000000000000000000000000021
:10D0F0000000F00018010C020C02040206000600F9
:10D1000006000600C60F060306030C030C031803F3
:10D11000F00000000000000000000000000000001F
:10D1200000000F0F06060606060606060606060699
:10D13000FE07060606060606060606060606060696
:10D140000F0F0000000000000000000000000000C1
:10D150000000FC0360006000600060006000600090
:10D1600060006000600060006000600060006000BF
:10D17000FC030000000000000000000000000000B0
:10D180000000F807C000C000C000C000C000C00020
:10D19000C000C000C000C000C000C000C000C0008F
:10D1A000C000C60066003C00000000000000000057
:10D1B0000000CF038601C600460026001600360098
:10D1C0002E006E004600C60086008601060106039A
:10D1D0008F070000000000000000000000000000B9
:10D1E00000001F00060006000600060006000600FC
:10D1F00006000600060006000600060406040602F5
:10D20000FF0300000000000000000000000000001C
:10D2100000000707860386038E038E034E034E032A
:10D220004A035A035A033A03320332033203120306
:10D230008707000000000000000000000000000060
:10D2400000008E0F0C021C021C0234023402640225
:10D2500064024402C40284028403840304030403BA
:10D260001F0200000000000000000000000000009D
:10D270000000F00098010C030C02060606060606E4
:10D28000060606060606060606060C020C039801AC
:10D29000F00000000000000000000000000000009E
:10D2A0000000FF000603060606060606060606063A
:10D2B0008603FE00060006000600060006000600C3
:10D2C0001F0000000000000000000000000000003F
:10D2D0000000F00098010C030C0206060606060684
:10D2E000060606060606060676064C02CC039801DC
:10D2F000F0008007000300000000000000000000B4
:10D300000000FF01060306060606060606060603DB
:10D31000FE004600C60086008601060306030606D8
:10D320000F0E0000000000000000000000000000E0
:10D330000000F8020C030602060206000E003C0084
:10D34000F800E003800300070206020606060C034D
:10D35000F0010000000000000000000000000000DC
:10D360000000FE0762046108610860006000600060
:10D3700060006000600060006000600060006000AD
:10D38000F8010000000000000000000000000000A4
:10D3900000001E070C020C020C020C020C020C0214
:10D3A0000C020C020C020C020C020C020C02180102
:10D3B000F00000000000000000000000000000007D
:10D3C00000000F070602040104010C010C01880093
:10D3D0008800980098005000500070003000200035
:10D3E000200000000000000000000000000000001D
:10D3F0000000F70E6204420446044604640264021C
:10D40000E402E4029C029C019801980188018800D2
:10D410008800000000000000000000000000000084
:10D4200000009E070C01080118019000B000600088
:10D43000200060006000D000900088010801040313
:10D440008E07000000000000000000000000000047
:10D4500000000F0F060404020C0208011801B800B6
:10D46000B00070006000600060006000600060005C
:10D47000F8010000000000000000000000000000B3
:10D480000000FC070C02060302018001800040003E
:10D490004000200020001000180008040C040402C2
:10D4A000FE0300000000000000000000E003200078
:10D4B000200020002000200020002000200020006C
:10D4C000200020002000200020002000200020005C
:10D4D00020002000E0030000000000000000000029
:10D4E00004000400080008001000100010002000D4
:10D4F000200040004000C0008000800000010001CA
:10D500000002000200020004000000007C00400055
:10D51000400040004000400040004000400040000B
:10D5200040004000400040004000400040004000FB
:10D53000400040007C0000000000600090000801F6
:10D5400000000000000000000000000000000000DB
:10D5500000000000000000000000000000000000CB
:10D5600000000000000000000000000000000000BB
:10D5700000000000000000000000000000000000AB
:10D58000000000000000000000000000000000009B
:10D59000000000000000FF0F000000001800600005
:10D5A000000000000000000000000000000000007B
:10D5B000000000000000000000000000000000006B
:10D5C000000000000000000000000000000000005B
:10D5D000000000000000000000000000F0010C034B
:10D5E0000C030003E0031C030E03060306038E0B6B
:10D5F0007C0E0000000000000000000000000000A1
:10D6000008000E000C000C000C000C00CC013C03C8
:10D610001C060C060C060C060C060C060C021C0361
:10D62000E401000000000000000000000000000015
:10D63000000000000000000000000000F0008C016D
:10D640008C01860106000600060006020C020C0191
:10D65000F0000000000000000000000000000000DA
:10D660000002C003000300030003000378038C03DF
:10D670000C030603060306030603060304038C07D4
:10D680007801000000000000000000000000000021
:10D69000000000000000000000000000E00118038E
:10D6A00008020C060C06FC070C000C0018041802FB
:10D6B000E001000000000000000000000000000089
:10D6C0000000C0036006300630003000FE0130006C
:10D6D00030003000300030003000300030003000CA
:10D6E000FC0100000000000000000000000000003D
:10D6F000000000000000000000000000F007D80655
:10D700008C018C018C019801F8000C00FC00CC030A
:10D71000060306038E03F80000000000000000006E
:10D7200008000E000C000C000C000C00EC011C03A7
:10D730000C030C030C030C030C030C030C030C0371
:10D740009E07000000000000000000000000000034
:10D750000000600060000000000040007C006000ED
:10D7600060006000600060006000600060006000B9
:10D77000FC030000000000000000000000000000AA
:10D780000000C001C001000000000001F0018001A4
:10D790008001800180018001800180018001800181
:10D7A00080018001CC007C0000000000000000002F
:10D7B00008000E000C000C000C000C008C038C0008
:10D7C0008C004C006C005C008C008C010C010C0384
:10D7D0009E070000000000000000000000000000A4
:10D7E00040007C006000600060006000600060003D
:10D7F0006000600060006000600060006000600029
:10D80000FC03000000000000000000000000000019
:10D810000000000000000000000000003707EE06D6
:10D820006606660666066606660666066606660698
:10D83000FF0F0000000000000000000000000000DA
:10D84000000000000000000000000000EE011C03CA
:10D850000C030C030C030C030C030C030C030C0350
:10D860009E07000000000000000000000000000013
:10D87000000000000000000000000000F00098011F
:10D880000C03060606060606060606060C030C032F
:10D89000F000000000000000000000000000000098
:10D8A000000000000000000000000000EE011C036A
:10D8B0000C060C060C060C060C060C060C031C03CE
:10D8C000EC010C000C003E00000000000000000015
:10D8D00000000000000000000000000078028C033F
:10D8E0000C030603060306030603060304038C0366
:10D8F000780300030003C0070000000000000000E0
:10D900000000000000000000000000009F03580617
:10D910003806180018001800180018001800180021
:10D92000FF000000000000000000000000000000F8
:10D93000000000000000000000000000F0031C03D5
:10D940000C020C023800F000C003040304038C0333
:10D95000FC010000000000000000000000000000CA
:10D96000000000002000200030003000FE013000E8
:10D970003000300030003000300030003002300223
:10D98000E0010000000000000000000000000000B6
:10D990000000000000000000000008028E030C03DD
:10D9A0000C030C030C030C030C030C030C039C076B
:10D9B00078010000000000000000000000000000EE
:10D9C0000000000000000000000000001E070C0224
:10D9D0000801080118019000B000B000600060006C
:10D9E0002000000000000000000000000000000017
:10D9F000000000000000000000000000F70E6204BC
:10DA0000460464026402EC029C01980198019801AA
:10DA100008000000000000000000000000000000FE
:10DA2000000000000000000000000000BC0718011A
:10DA30001001B00060006000E000900008010803E1
:10DA40009E07000000000000000000000000000031
:10DA50000000000000000000000000009E07080118
:10DA60000801080190009000B000600060006000B4
:10DA70002000200024001C00000000000000000026
:10DA8000000000000000000000000000FC01840114
:10DA9000C4004400600020003000180208020C039B
:10DAA000FC010000000000000000000000038000F6
:10DAB00080008000800080008000800080004000A6
:10DAC00020004000800080008000800080008000F6
:10DAD0008000800000030000400040004000400043
:10DAE0004000400040004000400040004000400036
:10DAF0004000400040004000400040004000400026
:10DB00004000400040004000000000000C001000F9
:10DB10001000100010001000100010001000200075
:10DB20004000200010001000100010001000100035
:10DB3000100010000C00000000001C002204C204B1
:10DB40008003000000000000000000000000000052
:10DB500000000000000000000000000000000000C5
:10DB6000000000000000000001F80000FFC007FCFA
:10DB70000001FFE00FFF0007FFF01FFF800FFFF025
:10DB80003FFFC01FFFF83FFFE07FFFF83FFFF0FFC0
:10DB9000FFF83FFFFBFFFFF83FFFFFFFFFF83FFFEE
:10DBA000FFFFFFF83FFFFFFF9FF83FFFFFFF0FF86A
:10DBB0003FF3FFFC0FF83FF1FFF80FF83FF0FFE0F5
:10DBC0000FF83FF07F800FF83FF01E000FF83FF096
:10DBD00008000FF83FF000000FF83FF000000FF8CA
:10DBE0003FF0000E0FF83FF0001E0FF83FE0007E00
:10DBF0000FF83FE000FE0FF83FE001FE0FF83FE0B6
:10DC000003FE0FF83FE007FE0FF83FE007FE0FF8B6
:10DC10003FE003FE0FF83FE001FE0FF83FE000FE9B
:10DC20000FF83FE0007E0FF80000000007FFFF80C4
:10DC30000FFFFFE01FFFFFF01FFFFFF83FFFFFFC9C
:10DC400000001FFC00000FFC00000FF800001FF890
:10DC500000003FF01FFFFFE03FFFFFC03FFFFF80DE
:10DC60007FFFFF007FFFFE007FF1FE00FFE0FC0072
:10DC7000FFE07C00FFC07E00FFC03E00FFC03F0011
:10DC8000FF801F00FF800F80FF800F80FF0007C014
:10DC900000000000000000000200D0070200FFFFAB
:10DCA0000200D0070200FFFFCE01208D01204C01B1
:10DCB00020000000C03407A03404B00A0380180616
:10DCC000801801601801500A04500A01EF0120CEAB
:10DCD00001208D01204C0120000000EB0010AA0063
:10DCE000106900106904100000000000000000002E
:10DCF000995C00084D5B000895590008E55B000839
:10DD0000615A0008495C00083D5C0008DD5A0008C3
:10DD1000CD5A00089D5B0008F5590008AD59000870
:10DD2000D35500084D61000835620008F560000811
:10DD3000895F00081D6000085D610008855E0008BD
:10DD40002D6300081D5F00085962000891610008FA
:10DD500001590008095E00081D6100086D5F000898
:10DD600029610008D5560008FD610008555F0008CC
:10DD7000E9620008C16100089D5E00082363000895
:10DD800019630008F5580008B55E00084D590008F1
:10DD9000E15600082959000885560008BB550008BF
:10DDA0007D550008F1610008295E00081B5E00082F
:10DDB000795F000811610008C5620008F55E00087F
:10DDC000435E0008795E0008CD5E000845630008E8
:10DDD000ED5500080000891112239B322446AD57EF
:10DDE0003665BF74488CC19D5AAFD3BE6CCAE5DBA3
:10DDF0007EE9F7F88110080193331A22A5562C47C3
:10DE0000B7753E64C99C408DDBBF52AEEDDA64CB82
:10DE1000FFF976E802218B30100299132667AF765E
:10DE20003444BD554AADC3BC588ED19F6EEBE7FA62
:10DE30007CC8F5D983310A2091121803A7772E6682
:10DE4000B5543C45CBBD42ACD99E508FEFFB66EA42
:10DE5000FDD874C904428D5316619F702004A91522
:10DE60003227BB364CCEC5DF5EEDD7FC6888E19922
:10DE70007AABF3BA85520C4397711E60A114280542
:10DE8000B3373A26CDDE44CFDFFD56ECE998608902
:10DE9000FBBB72AA06638F7214409D512225AB34DE
:10DEA0003006B9174EEFC7FE5CCCD5DD6AA9E3B8E2
:10DEB000788AF19B87730E6295501C41A3352A2402
:10DEC000B1163807CFFF46EEDDDC54CDEBB962A8C2
:10DED000F99A708B088481951AA793B62CC2A5D3A2
:10DEE0003EE1B7F04008C919522BDB3A644EED5FB2
:10DEF000766DFF7C899400859BB712A6ADD224C3B2
:10DF0000BFF136E0C1184809D33B5A2AE55E6C4F91
:10DF1000F77D7E6C0AA583B4188691972EE3A7F24D
:10DF20003CC0B5D14229CB38500AD91B666FEF7E71
:10DF3000744CFD5D8BB502A499961087AFF326E271
:10DF4000BDD034C1C3394A28D11A580BE77F6E6E51
:10DF5000F55C7C4D0CC685D71EE597F42880A19111
:10DF60003AA3B3B2444ACD5B5669DF78600CE91D31
:10DF7000722FFB3E8DD604C79FF516E4A990208131
:10DF8000BBB332A2C55A4C4BD7795E68E11C680D11
:10DF9000F33F7A2E0EE787F61CC495D52AA1A3B0CD
:10DFA0003882B193466BCF7A5448DD59622DEB3CF1
:10DFB000700EF91F8FF706E69DD414C5ABB122A0F1
:10DFC000B9923083C77B4E6AD5585C49E33D6A2CD1
:10DFD000F11E780F00F40008D0F3000879930008D0
:10DFE00000000000020000103D3D3D3D3D3D3D3D37
:10DFF0003D3D3D3D3D3D3D3D3D3D3D3D3D3D3D3D51
:10E000003D3D3D3D3D3D3D3D3D3D3D3D3D3D3D3D40
:10E010003D3D3D3D3D3D3D3D3D3D3D3D3D3D3D3D30
:10E020003D3D3D3D3D3D3D3D3D3D3D3D3D3D3D3D20
:10E030003D3D3D3D0D0A726164696F203C73756220
:10E04000636D643E205B617267735D20202D2053F9
:10E05000583132383120726164696F20636F6E7499
:10E06000726F6C0D0A2D2D2D2D2D2D2D2D2D2D2D5D
:10E070002D2D2D2D2D2D2D2D2D2D2D2D2D2D2D2DD0
:10E080002D2D2D2D2D2D2D2D2D2D2D2D2D2D2D2DC0
:10E090002D2D2D2D2D2D2D2D2D2D2D2D2D2D2D2DB0
:10E0A0002D2D2D2D2D2D2D2D2D2D2D2D2D2D2D2DA0
:10E0B0002D0D0A4D6F646520436F6E66696775723A
:10E0C0006174696F6E3A0D0A20206D6F6465203CA3
:10E0D000424C457C4C4F52417C4746534B7C464C0E
:10E0E00052433E20202020202020202D2043686104
:10E0F0006E676520776F726B696E67206D6F646500
:10E100000D0A2020726666726571203C487A3E20B6
:10E1100020202020202020202020202020202020FF
:10E1200020202020202D2053657420524620667226
:10E13000657175656E63790D0A2D2D2D2D2D2D2D93
:10E140002D2D2D2D2D2D2D2D2D2D2D2D2D2D2D2DFF
:10E150002D2D2D2D2D2D2D2D2D2D2D2D2D2D2D2DEF
:10E160002D2D2D2D2D2D2D2D2D2D2D2D2D2D2D2DDF
:10E170002D2D2D2D2D2D2D2D2D2D2D2D2D2D2D2DCF
:10E180002D2D2D2D2D0D0A506172616D65746572F6
:10E1900020436F6E66696775726174696F6E3A0DC0
:10E1A0000A20206D6F64756C6174696F6E203C6627
:10E1B00069656C643E203C76616C75653E2020206C
:10E1C000202020202D20536574206D6F64756C61B4
:10E1D00074696F6E20706172616D65746572730D24
:10E1E0000A20207061636B6574203C6669656C640D
:10E1F0003E203C76616C75653E202020202020204A
:10E20000202020202D20536574207061636B65747D
:10E2100020706172616D65746572730D0A202062F1
:10E2200061756472617465205B696E6465785D20F8
:10E2300020202020202020202020202020202020DE
:10E240002D205365742062617564726174652028A5
:10E250006175746F2D646574656374206D6F64659A
:10E26000290D0A2020706F776572203C64426D3E54
:10E27000202020202020202020202020202020209E
:10E280002020202020202D205365742054582070F9
:10E290006F77657220282D31382E2E2B3133290DC2
:10E2A0000A202072616D7074696D65203C75733E43
:10E2B000202020202020202020202020202020205E
:10E2C000202020202D205365742072616D702074F1
:10E2D000696D652028327C347C367C387C31307C1A
:10E2E00031327C31367C3230290D0A2D2D2D2D2DE9
:10E2F0002D2D2D2D2D2D2D2D2D2D2D2D2D2D2D2D4E
:10E300002D2D2D2D2D2D2D2D2D2D2D2D2D2D2D2D3D
:10E310002D2D2D2D2D2D2D2D2D2D2D2D2D2D2D2D2D
:10E320002D2D2D2D2D2D2D2D2D2D2D2D2D2D2D2D1D
:10E330002D2D2D2D2D2D2D0D0A4F706572617469B7
:10E340006F6E20436F6D6D616E64733A0D0A20200D
:10E350007478207C2072782020202020202020200B
:10E3600020202020202020202020202020202020AD
:10E37000202D2054582F5258206F70657261746997
:10E380006F6E730D0A2D2D2D2D2D2D2D2D2D2D2D37
:10E390002D2D2D2D2D2D2D2D2D2D2D2D2D2D2D2DAD
:10E3A0002D2D2D2D2D2D2D2D2D2D2D2D2D2D2D2D9D
:10E3B0002D2D2D2D2D2D2D2D2D2D2D2D2D2D2D2D8D
:10E3C0002D2D2D2D2D2D2D2D2D2D2D2D2D2D2D2D7D
:10E3D0002D0D0A48656C7020436F6D6D616E64731E
:10E3E0003A0D0A20206D6F64756C6174696F6E2040
:10E3F00068656C70207C207061636B657420686553
:10E400006C70202020202D2053686F772064657465
:10E4100061696C65642068656C700D0A202062611A
:10E420007564726174652068656C702020202020FE
:10E430002020202020202020202020202020202DCF
:10E440002053686F7720626175647261746520641F
:10E45000657461696C730D0A3D3D3D3D3D3D3D3D3B
:10E460003D3D3D3D3D3D3D3D3D3D3D3D3D3D3D3DDC
:10E470003D3D3D3D3D3D3D3D3D3D3D3D3D3D3D3DCC
:10E480003D3D3D3D3D3D3D3D3D3D3D3D3D3D3D3DBC
:10E490003D3D3D3D3D3D3D3D3D3D3D3D3D3D3D3DAC
:10E4A0003D3D3D3D0D0A003D3D3D3D3D3D3D3D3D3C
:10E4B0003D3D3D3D3D3D3D3D3D3D3D3D3D3D3D3D8C
:10E4C0003D3D3D3D3D3D3D3D3D3D3D3D3D3D3D3D7C
:10E4D0003D3D3D3D3D3D3D3D3D3D3D3D3D3D3D3D6C
:10E4E0003D3D3D3D3D3D3D3D3D3D3D3D3D3D3D3D5C
:10E4F0003D3D3D3D3D3D3D3D3D3D3D3D3D3D3D3D4C
:10E500003D3D3D3D3D3D3D3D3D3D3D3D3D3D3D3D3B
:10E510003D3D3D0D0A6D6F64756C6174696F6E20D1
:10E520003C6669656C643E203C76616C75653E2096
:10E53000202D20536574206D6F64756C6174696F54
:10E540006E20706172616D65746572730D0A2020B2
:10E55000424C452F4746534B206669656C64733ABD
:10E560000D0A2020202062725F6277202020203A4E
:10E57000203078303428322E304D2F322E344D2931
:10E580007C7C3078323828312E364D2F322E344D67
:10E59000297C7C3078344328312E304D2F322E3474
:10E5A0004D297C7C3078343528312E304D2F312E5A
:10E5B000324D290D0A20202020202020202020203C
:10E5C000202020203078373028302E384D2F322E22
:10E5D000344D297C7C3078363928302E384D2F3117
:10E5E0002E324D297C7C3078384428302E354D2F02
:10E5F000312E324D297C7C3078383628302E354DFE
:10E600002F302E364D290D0A2020202020202020BA
:10E61000202020202020203078423128302E344DF8
:10E620002F312E324D297C7C3078414128302E34D8
:10E630004D2F302E364D297C7C3078434528302EA6
:10E6400032354D2F302E364D297C7C30784337289B
:10E65000302E32354D2F302E334D297C7C3078458D
:10E660004628302E3132354D2F302E334D290D0AAC
:10E67000202020206D6F64696E646578203A203018
:10E6800028302E3335297C7C3128302E3530297CBA
:10E690007C3228302E3735297C7C3328312E30309F
:10E6A000297C7C3428312E3235297C7C3528312E4A
:10E6B0003530297C7C3628312E3735297C7C37282B
:10E6C000322E3030290D0A2020202020202020202A
:10E6D0002020202020203828322E3235297C7C39F9
:10E6E00028322E3530297C7C313028322E3735299E
:10E6F0007C7C313128332E3030297C7C31322833F8
:10E700002E3235297C7C313328332E3530297C7CE0
:10E71000313428332E3735297C7C313528342E305E
:10E7200030290D0A2020202073686170696E6720EF
:10E73000203A2030783030284F4646297C7C30788B
:10E7400031302842545F315F30297C7C3078323060
:10E750002842545F305F35290D0A20204C4F52412A
:10E76000206669656C64733A0D0A20202020736668
:10E77000203A203078353028534635297C7C307853
:10E78000363028534636297C7C307837302853463B
:10E7900037297C7C3078383028534638297C7C30C7
:10E7A00078393028534639297C7C307841302853D9
:10E7B000463130297C7C307842302853463131292B
:10E7C0007C7C307843302853463132290D0A202092
:10E7D00020206277203A20307833342842575F3245
:10E7E00030304B297C7C307832362842575F3430C9
:10E7F000304B297C7C307831382842575F383030B4
:10E800004B297C7C307830412842575F313630309C
:10E810004B290D0A202020206372203A20307830C6
:10E820003128342F35297C7C3078303228342F360B
:10E83000297C7C3078303328342F37297C7C307821
:10E84000303428342F38297C7C30783035284C49B6
:10E850005F342F35297C7C30783036284C495F3442
:10E860002F36297C7C30783037284C495F342F375D
:10E87000290D0A2020464C5243206669656C64735A
:10E880003A0D0A2020202062725F6277202020202B
:10E890003A203078303428322E364D2F322E344DF7
:10E8A000297C7C3078323828322E30384D2F322E69
:10E8B000344D297C7C3078343528312E334D2F313E
:10E8C0002E324D297C7C3078363928312E30344D2B
:10E8D0002F312E324D290D0A2020202020202020EB
:10E8E000202020202020203078383628302E363541
:10E8F0004D2F302E364D297C7C3078414128302EEA
:10E9000035324D2F302E364D297C7C3078433728D8
:10E91000302E3332354D2F302E334D297C7C3078DC
:10E92000454228302E32364D2F302E334D290D0AD8
:10E93000202020206372202020202020203A203018
:10E940007830302843525F312F32297C7C30783048
:10E95000322843525F332F34297C7C30783034287E
:10E9600043525F312F30290D0A2020202073686127
:10E9700070696E6720203A2030783030284F464644
:10E98000297C7C307831302842545F315F30297CDB
:10E990007C307832302842545F305F35290D0A458B
:10E9A00078616D706C65733A20726164696F206D77
:10E9B0006F64756C6174696F6E2062725F6277203C
:10E9C000307834430D0A20202020202020202020D1
:10E9D000726164696F206D6F64756C6174696F6ECC
:10E9E00020736620307837300D0A3D3D3D3D3D3D7A
:10E9F0003D3D3D3D3D3D3D3D3D3D3D3D3D3D3D3D47
:10EA00003D3D3D3D3D3D3D3D3D3D3D3D3D3D3D3D36
:10EA10003D3D3D3D3D3D3D3D3D3D3D3D3D3D3D3D26
:10EA20003D3D3D3D3D3D3D3D3D3D3D3D3D3D3D3D16
:10EA30003D3D3D3D3D3D3D3D3D3D3D3D3D3D3D3D06
:10EA40003D3D3D3D3D3D3D3D3D3D3D3D3D3D3D3DF6
:10EA50003D3D3D3D3D3D0D0A003D3D3D3D3D3D3D86
:10EA60003D3D3D3D3D3D3D3D3D3D3D3D3D3D3D3DD6
:10EA70003D3D3D3D3D3D3D3D3D3D3D3D3D3D3D3DC6
:10EA80003D3D3D3D3D3D3D3D3D3D3D3D3D3D3D3DB6
:10EA90003D3D3D3D3D3D3D3D3D3D3D3D3D3D3D3DA6
:10EAA0003D3D3D3D3D3D3D3D3D3D3D3D3D3D3D3D96
:10EAB0003D3D3D3D3D3D3D3D3D0D0A7061636B6516
:10EAC00074203C6669656C643E203C76616C7565BB
:10EAD0003E20202D20536574207061636B65742087
:10EAE000706172616D6574657273202863757272EE
:10EAF000656E74205061636B657454797065206233
:10EB000061736564290D0A2020424C4520666965C1
:10EB10006C64733A0D0A20202020436F6E6E65638B
:10EB200074696F6E5374617465203A2030284D41CA
:10EB3000535445525F534C415645297C7C31284102
:10EB4000445645525449534552297C7C32285458E6
:10EB50005F54455354297C7C332852585F544553A5
:10EB600054297C7C3428525854585F5445535429B6
:10EB70000D0A202020204372634669656C642020C2
:10EB80002020202020203A2030284F4646297C7C17
:10EB900031284352435F3342290D0A20202020426E
:10EBA0006C655061636B6574547970652020203A00
:10EBB000203028505242535F39297C7C31285052F2
:10EBC00042535F3135297C7C32284559454C4F4EA4
:10EBD000475F315F30297C7C33284559454C4F4E87
:10EBE000475F305F31290D0A20202020202020207F
:10EBF00020202020202020202020202020203428F9
:10EC000045594553484F52545F315F30297C7C351C
:10EC10002845594553484F52545F305F31297C7C19
:10EC20003628414C4C5F31297C7C3728414C4C5F65
:10EC300030290D0A2020202057686974656E696E9E
:10EC400067202020202020203A2030783030284FA4
:10EC50004E297C7C30783038284F4646290D0A20D2
:10EC6000204746534B206669656C64733A0D0A2051
:10EC7000202020507265616D626C6520202020206C
:10EC80002020203A2030783030283462697473298B
:10EC90007C7C30783130283862697473297C7C3010
:10ECA00078323028313262697473297C7C30783351
:10ECB0003028313662697473290D0A202020202003
:10ECC0002020202020202020202020202020202044
:10ECD000203078343028323062697473297C7C307B
:10ECE00078353028323462697473297C7C30783608
:10ECF0003028323862697473297C7C307837302848
:10ED0000333262697473290D0A2020202053796EF2
:10ED100063576F72644C656E67746820203A2030C8
:10ED2000783030283162797465297C7C30783032D3
:10ED300028326279746573297C7C307830342833CA
:10ED40006279746573297C7C307830362834627936
:10ED5000746573297C7C3078303828356279746525
:10ED600073290D0A2020202053796E63576F726437
:10ED70004D617463682020203A2030783030284F6D
:10ED80004646297C7C307831302831297C7C3078AB
:10ED900032302832297C7C3078333028315F322978
:10EDA0007C7C307834302833297C7C3078353028AE
:10EDB000315F33297C7C3078363028325F33297CD0
:10EDC0007C3078373028315F325F33290D0A2020BC
:10EDD000202053796E63576F7264312F322F3320A6
:10EDE00020203A203C6865785F62797465733E2024
:10EDF0002D205365742073796E6320776F726420C1
:10EE0000312F322F3320286D6178203520627974BC
:10EE1000657320666F72204746534B290D0A2020E8
:10EE2000202053796E63576F7264202020202020A9
:10EE300020203A2053686F7720616C6C2073796EC4
:10EE40006320776F7264730D0A202020204865616B
:10EE5000646572202020202020202020203A2030AD
:10EE6000783030285641524941424C45297C7C300B
:10EE7000783230284649584544290D0A2020202060
:10EE80005061796C6F616420202020202020202098
:10EE90003A20312D32353520286279746573290D79
:10EEA0000A202020204372632020202020202020C0
:10EEB00020202020203A2030783030284F46462924
:10EEC0007C7C30783130283162797465297C7C30E3
:10EED00078323028326279746573297C7C307833DB
:10EEE0003028336279746573290D0A202020205759
:10EEF000686974656E696E67202020202020203AA2
:10EF00002030783030284F4E297C7C3078303828BB
:10EF10004F4646290D0A20204C4F52412066696514
:10EF20006C64733A0D0A20202020507265616D6276
:10EF30006C6520202020202020203A20302D3235E2
:10EF400035202873796D626F6C7320636F756E74F2
:10EF5000290D0A2020202048656164657220202048
:10EF6000202020202020203A2030783030285641A0
:10EF7000524941424C452F4558504C494349542928
:10EF80007C7C307838302846495845442F494D50CC
:10EF90004C49434954290D0A202020205061796CA6
:10EFA0006F61642020202020202020203A20312D55
:10EFB00032353520286279746573290D0A202020A6
:10EFC0002043726320202020202020202020202089
:10EFD000203A2030783230284F4E297C7C307830EF
:10EFE00030284F4646290D0A20202020496E76659C
:10EFF0007274495120202020202020203A2030788F
:10F000003430284E4F524D414C297C7C3078303082
:10F0100028494E564552544544290D0A2020464C55
:10F020005243206669656C64733A2053616D6520B4
:10F030006173204746534B2028507265616D626CA6
:10F04000652F53796E63576F72644C656E67746891
:10F050002F53796E63576F72644D617463682F53D9
:10F06000796E63576F7264312F322F332F48656189
:10F070006465722F5061796C6F61642F4372632FE6
:10F0800057686974656E696E67290D0A2020202013
:10F0900053796E63576F7264312F322F33202020E3
:10F0A0003A203C6865785F62797465733E202D2054
:10F0B0005365742073796E6320776F726420312FEB
:10F0C000322F3320286D6178203420627974657383
:10F0D00020666F7220464C5243290D0A4578616DB7
:10F0E000706C65733A20726164696F207061636B44
:10F0F0006574205061796C6F61642036340D0A208C
:10F10000202020202020202020726164696F207040
:10F1100061636B65742043726320307832300D0A6E
:10F1200020202020202020202020726164696F2070
:10F130007061636B65742053796E63576F726431CD
:10F1400020307831323334353637380D0A202020DC
:10F1500020202020202020726164696F207061636C
:10F160006B65742053796E63576F72640D0A3D3D71
:10F170003D3D3D3D3D3D3D3D3D3D3D3D3D3D3D3DBF
:10F180003D3D3D3D3D3D3D3D3D3D3D3D3D3D3D3DAF
:10F190003D3D3D3D3D3D3D3D3D3D3D3D3D3D3D3D9F
:10F1A0003D3D3D3D3D3D3D3D3D3D3D3D3D3D3D3D8F
:10F1B0003D3D3D3D3D3D3D3D3D3D3D3D3D3D3D3D7F
:10F1C0003D3D3D3D3D3D3D3D3D3D3D3D3D3D0D0AD2
:10F1D000003D3D3D3D3D3D3D3D3D3D3D3D3D3D3D9C
:10F1E0003D3D3D3D3D3D3D3D3D3D3D3D3D3D3D3D4F
:10F1F0003D3D3D3D3D3D3D3D3D3D3D3D3D3D3D3D3F
:10F200003D3D3D3D3D3D3D0D0A3D3D3D3D3D3D3D91
:10F210003D3D3D3D3D3D3D3D3D3D3D3D3D3D3D3D1E
:10F220003D3D3D3D3D3D3D3D3D3D3D3D3D3D3D3D0E
:10F230003D3D3D3D3D3D3D3D3D3D3D3D3D3D3D0D2E
:10F240000A003D3D3D3D3D3D3D3D3D3D3D3D3D3D5E
:10F250003D3D3D3D3D3D3D3D3D3D3D3D3D3D3D3DDE
:10F260003D3D3D3D3D3D3D3D3D3D3D3D3D3D3D3DCE
:10F270003D3D3D3D3D3D3D3D3D3D3D3D3D3D3D3DBE
:10F280003D3D3D3D3D3D3D0D0A3D3D3D3D3D3D3D11
:10F290003D3D3D3D3D3D3D3D3D3D3D3D3D3D3D3D9E
:10F2A0003D3D3D3D3D3D3D3D3D3D3D3D3D3D3D3D8E
:10F2B0003D3D3D3D3D3D3D3D3D3D3D3D3D3D3D3D7E
:10F2C0003D3D3D3D3D3D3D3D3D3D3D3D3D3D0D0AD1
:10F2D0000000000054FB000878FA000815870008B9
:10F2E000FF0000005CFB0008C4FA0008A1990008B8
:10F2F000FF00000064FB00080000000000000000A8
:10F3000000000000000000000004000030000000C9
:10F3100000000000000000005CFB0008000000008E
:10F3200000000000000000000000000000040000D9
:10F3300018000000000000000000000000404040F5
:10F3400040404040404041414141414040404040B8
:10F350004040404040404040404040404005020264
:10F360000202020202020202020202020220202023
:10F37000202020202020200202020202020290907F
:10F38000909090901010101010101010101010107D
:10F3900010101010101010100202020202028888D1
:10F3A00088888888080808080808080808080808DD
:10F3B00008080808080808080202020240000000C5
:10F3C0003DF3000864656661756C745461736B008D
:10F3D0000D0A68656C703A0D0A204C6973747320CD
:10F3E000616C6C20746865207265676973746572FE
:10F3F000656420636F6D6D616E64730D0A0D0A00A4
:10F4000068656C7000000000496E636F727265631E
:10F410007420636F6D6D616E6420706172616D65E3
:10F420007465722873292E2020456E74657220221F
:10F4300068656C702220746F207669657720612082
:10F440006C697374206F6620617661696C61626CAF
:10F450006520636F6D6D616E64732E0D0A0D0A0079
:10F46000436F6D6D616E64206E6F74207265636FA3
:10F47000676E697365642E2020456E74657220275F
:10F4800068656C702720746F20766965772061202D
:10F490006C697374206F6620617661696C61626C5F
:10F4A0006520636F6D6D616E64732E0D0A0D0A0029
:10F4B000496E76616C696420464C524320507265F7
:10F4C000616D626C652028307830302F30783130B3
:10F4D0002F307832302F307833302F307834302F4F
:10F4E000307835302F307836302F30783730290D5E
:10F4F0000A000000496E76616C6964204746534BF0
:10F5000020507265616D626C652028307830302F34
:10F51000307831302F307832302F307833302F3010
:10F520007834302F307835302F307836302F3078AF
:10F530003730290D0A000000496E76616C6964203D
:10F54000464C52432053796E63576F72644D617419
:10F5500063682028307830302F307831302F307881
:10F5600032302F307833302F307834302F307835B8
:10F57000302F307836302F30783730290D0A0000A0
:10F58000496E76616C6964204746534B2053796E0F
:10F5900063576F72644D617463682028307830302F
:10F5A0002F307831302F307832302F307833302F81
:10F5B000307834302F307835302F307836302F3067
:10F5C000783730290D0A000043757272656E742019
:10F5D0006669786564206C656E6774683A20257585
:10F5E0002062797465732028757365722064617474
:10F5F00061290D0A546F74616C207061636B6574CE
:10F600003A20257520627974657320284865616405
:10F6100065725B325D2B446174615B25755D2B43C4
:10F6200052435B325D290D0A00000000466978658F
:10F6300064206C656E6774682073657420746F2035
:10F64000257520627974657320287573657220644E
:10F65000617461290D0A546F74616C207061636B71
:10F6600065743A2025752062797465732028486591
:10F67000616465725B325D2B446174615B25755D0D
:10F680002B4352435B325D290D0A00003D3D3D3D59
:10F690003D3D3D3D204D52313620436F6E666967DA
:10F6A00075726174696F6E203D3D3D3D3D3D3D3D50
:10F6B0000D0A4461746120466F726D617420203AB6
:10F6C0002025730D0A557365722044617461204CC6
:10F6D000656E3A20257520627974657320287075EF
:10F6E00072652064617461290D0A546F74616C2025
:10F6F0005061636B6574203A2025752062797465CA
:10F700007320284865616465722B446174612B43E2
:10F710005243290D0A5458204944202020202020FB
:10F7200020203A203078253034580D0A525820498C
:10F730004420312020202020203A203078253034E9
:10F74000580D0A52582049442032202020202020E1
:10F750003A203078253034580D0A52582049442038
:10F76000332020202020203A203078253034580DB6
:10F770000A545820506F77657220202020203A20AC
:10F7800025642064426D0D0A526164696F204D6FDB
:10F7900064652020203A2025730D0A526164696F48
:10F7A00020526F6C652020203A2025730D0A3D3DC4
:10F7B0003D3D3D3D3D3D3D3D3D3D3D3D3D3D3D3D79
:10F7C0003D3D3D3D3D3D3D3D3D3D3D3D3D3D3D3D69
:10F7D0003D3D3D0D0A0000005061636B6574284C8F
:10F7E0006F5261293A20507265616D626C653D25EA
:10F7F00075204865616465723D30782558205061F8
:10F80000796C6F61643D2575204372633D307825C6
:10F810005820496E7665727449513D307825580DEF
:10F820000A0000005061636B657428464C524329FE
:10F830003A20507265616D626C653D3078255820C4
:10F8400053796E634C656E3D307825582053796E40
:10F85000634D617463683D30782558204865616464
:10F8600065723D30782558205061796C6F61643D38
:10F870002575204372633D30782558205768697498
:10F88000656E696E673D307825580D0A00000000EE
:10F890005061636B6574284746534B293A20507278
:10F8A00065616D626C653D307825582053796E63D3
:10F8B0004C656E3D307825582053796E634D6174E8
:10F8C00063683D30782558204865616465723D3035
:10F8D000782558205061796C6F61643D257520430F
:10F8E00072633D307825582057686974656E696E7B
:10F8F000673D307825580D0A000000005061636BA9
:10F90000657428424C45293A20436F6E6E656374D6
:10F91000696F6E53746174653D257520437263464B
:10F9200069656C643D257520426C655061636B654B
:10F9300074547970653D25752057686974656E69E2
:10F940006E673D307825580D0A000000464C524342
:10F950002053796E6320576F7264733A0D0A20202A
:10F96000576F726420313A20253032582530325892
:10F9700025303258253032580D0A2020576F7264D6
:10F9800020323A202530325825303258253032582E
:10F99000253032580D0A2020576F726420333A20E8
:10F9A00025303258253032582530325825303258DB
:10F9B0000D0A00004746534B2053796E6320576F62
:10F9C0007264733A0D0A2020576F726420313A2016
:10F9D00025303258253032582530325825303258AB
:10F9E000253032580D0A2020576F726420323A2099
:10F9F000253032582530325825303258253032588B
:10FA0000253032580D0A2020576F726420333A2077
:10FA1000253032582530325825303258253032586A
:10FA2000253032580D0A00006D6F64653A20275664
:10FA300041524941424C4527202D2076617269612F
:10FA4000626C65206C656E6774682028554152545D
:10FA50002069646C65290D0A20202020202027467B
:10FA60004958454427202D206669786564206C65D7
:10FA70006E6774680D0A00006D723136203C737534
:10FA800062636D643E205B617267735D202D204D63
:10FA90005231362073797374656D20636F6D6D61BB
:10FAA0006E64732E2055736520276D723136206881
:10FAB000656C702720666F722064657461696C7371
:10FAC0000D0A0000726164696F203C636D643E2022
:10FAD0002D2053583132383120726164696F2063B0
:10FAE0006F6E74726F6C20636F6D6D616E64732ED8
:10FAF000205573652027726164696F2068656C709A
:10FB00002720666F722064657461696C730D0A004A
:10FB100043757272656E74206D6F64653A2025734B
:10FB20000D0A4261756472617465733A20424C45F6
:10FB30003D2575207C204C4F52413D2575207C2071
:10FB40004746534B3D2575207C20464C52433D256E
:10FB5000750D0A006D723136000000007261646933
:10FB60006F0000005461736B5F496E6974000000A0
:10FB700090FB00080000002030010000E0100008A9
:10FB8000CCFB000830010020E8340000F07B0008C6
:10FB900081320182100379127A1AAA010110E3E876
:10FBA00003521925024001401305511408C950821F
:10FBB000081A2D101AF1109ADD14419BA95C10123D
:0CFBC000018220CBD4DF280120000000CF
:04000005080000ED02
:00000001FF
